:0400000057EF00F0C6
:100008002B002B002B002B002B002B002B002B0090
:10001800A5652B002B002B002B002B002B002B00A1
:100028002B002B002B002B002B002B002B002B0070
:100038002B002B002B0003622B002B002B002B0026
:10004800A4642B002B002B002B002B002B002B0073
:100058002B002B002B002B002B002B002B002B0040
:100068002B002B002B002B002B002B002B002B0030
:100078002B002B002B002B002B002B002B002B0020
:100088002B002B002B002B002B002B002B002B0010
:100098002B002B002B002B002B002B002B002B0000
:0A00A8002B002B00FF0000EFBBF05F
:10E68E000000000000000000007E81A581BD998180
:10E69E007E7EFFDBFFC3E7FF7E6CFEFEFE7C381046
:10E6AE000010387CFE7C381000383838FEFED6104C
:10E6BE00381010387CFE7C10380000183C3C1800D6
:10E6CE0000FFFFE7C3C3E7FFFF003C664242663C24
:10E6DE0000FFC399BDBD99C3FF0F03057D848484DC
:10E6EE00783C4242423C187E183F213F202060E099
:10E6FE00C03F213F212367E6C018DB3CE7E73CDB48
:10E70E001880E0F8FEF8E08000020E3EFE3E0E029B
:10E71E0000183C7E18187E3C18242424242400243F
:10E72E00007F929272121212003E6338444438CC2B
:10E73E0078000000007E7E7E00183C7E187E3C181D
:10E74E00FF10387C5410101000101010547C38102C
:10E75E000000180CFE0C180000003060FE60300047
:10E76E000000004040407E0000002466FF6624004A
:10E77E00000010387CFEFE000000FEFE7C3810000B
:10E78E00000000000000000000101010101000101B
:10E79E0000242424000000000024247E247E24244F
:10E7AE0000183E403C027C180000626408102646A9
:10E7BE000030483056888876001010200000000087
:10E7CE0000102040404020100020100808081020A3
:10E7DE0000004438FE384400000010107C10100079
:10E7EE000000000000001010200000007E0000005D
:10E7FE00000000000000101000000204081020406D
:10E80E00003C42464A52623C001030501010107CC0
:10E81E00003C42020C30427E003C42021C02423C52
:10E82E000008182848FE081C007E407C0202423C6C
:10E83E00001C20407C42423C007E42040810101016
:10E84E00003C42423C42423C003C42423E020438C2
:10E85E00000010100000101000001010000010102A
:10E86E0020081020402010080000007E00007E00CE
:10E87E000010080402040810003C420204080008BC
:10E88E00003C425E525E403C00182442427E4242B0
:10E89E00007C22223C22227C001C22404040221C72
:10E8AE000078242222222478007E22283828227EF4
:10E8BE00007E222838282070001C2240404E221E46
:10E8CE00004242427E424242003810101010103870
:10E8DE00000E0404044444380062242830282463C3
:10E8EE00007020202020227E006355494141414185
:10E8FE000062524A46424242003C42424242423C3E
:10E90E00007C22223C202070003C4242424A3C03C2
:10E91E00007C22223C282472003C42403C02423CB5
:10E92E00007F49080808081C004242424242423C0D
:10E93E0000414141412214080041414149494936B3
:10E94E000041221408142241004122140808081C18
:10E95E00007F42040810217F0078404040404078FC
:10E96E000080402010080402007808080808087883
:10E97E00001028448200000000000000000000008B
:10E98E00FF101008000000000000003C023E423F55
:10E99E00006020202E31312E0000003C4240423CCF
:10E9AE00000602023A46463B0000003C427E403CD6
:10E9BE00000C1210381010380000003D42423E028A
:10E9CE007C60202C32222262001000301010103891
:10E9DE0000020006020242423C6020242830282613
:10E9EE0000301010101010380000007649494949C7
:10E9FE000000005C624242420000003C4242423C47
:10EA0E000000006C32322C20700000364C4C340466
:10EA1E000E00006C322220700000003E403C027C52
:10EA2E000010107C1010120C000000424242463AB8
:10EA3E0000000041412214080000004149494936B6
:10EA4E0000000044281028440000004242423E02CA
:10EA5E007C00007C0810207C000C10106010100C44
:10EA6E0000101010001010100030080806080830B2
:10EA7E0000324C0000000000001C14141C000000AA
:10EA8E00003C4240423C0C023C0044004444443EA4
:10EA9E00000C003C427E403C003C4238043C443E6C
:10EAAE0000420038043C443E00300038043C443EF2
:10EABE00003C2424243C00000000003C40403C0666
:10EACE001C3C423C427E403C0042003C427E403C6C
:10EADE000030003C427E403C002400180808081C10
:10EAEE00007C823010101038003000180808081C06
:10EAFE0000421824427E4242001818003C427E42D8
:10EB0E00000C007C2038207C000000330C3F443B7E
:10EB1E00001F24447F444447001824003C42423CDA
:10EB2E00000042003C42423C002010003C42423C6D
:10EB3E00001824004242423C002010004242423C57
:10EB4E000000420042423E023C4218244242241837
:10EB5E00004200424242423C0008083E40403E080D
:10EB6E00081824207020427C0044287C107C101051
:10EB7E0000F84C78444F4445E61C12107C1010905F
:10EB8E00600C0038043C443E000C00180808081CB9
:10EB9E00000408003C42423C000004084242423C51
:10EBAE0000324C007C42424200324C0062524A46D5
:10EBBE00003C44443E007E000038444438007C0053
:10EBCE00001000102040423C000000007E4040003B
:10EBDE00000000007E0202000042C448F629438C69
:10EBEE001F42C44AF62A5F82020010001010101055
:10EBFE000000122448241200000048241224480069
:10EC0E0000228822882288228855AA55AA55AA55FC
:10EC1E00AADB77DBEEDB77DBEE1010101010101096
:10EC2E001010101010F01010101010F010F0101036
:10EC3E001014141414F414141400000000FC141412
:10EC4E00140000F010F01010101414F404F4141446
:10EC5E001414141414141414140000FC04F41414D6
:10EC6E00141414F404FC00000014141414FC00001A
:10EC7E00001010F010F000000000000000F0101066
:10EC8E0010101010101F00000010101010FF0000C8
:10EC9E000000000000FF101010101010101F1010B8
:10ECAE001000000000FF00000010101010FF1010E8
:10ECBE001010101F101F1010101414141417141409
:10ECCE0014141417101F00000000001F1017141446
:10ECDE00141414F700FF0000000000FF00F71414D6
:10ECEE001414141710171414140000FF00FF000062
:10ECFE00001414F700F71414141010FF00FF000096
:10ED0E000014141414FF0000000000FF00FF101088
:10ED1E001000000000FF141414141414141F00002B
:10ED2E000010101F101F00000000001F101F1010F9
:10ED3E0010000000001F14141414141414FF1414E3
:10ED4E00141010FF10FF10101010101010F0000013
:10ED5E0000000000001F101010FFFFFFFFFFFFFF5D
:10ED6E00FF00000000FFFFFFFFF0F0F0F0F0F0F00A
:10ED7E00F00F0F0F0F0F0F0F0FFFFFFFFF00000021
:10ED8E00000000314A444A3100003C427C427C4043
:10ED9E0040007E424040404000003F541414141482
:10EDAE00007E42201820427E0000003E4848483037
:10EDBE0000004444447A40408000334C0808080860
:10EDCE00007C1038444438107C1824427E422418AB
:10EDDE000018244242242466001C20183C42423C67
:10EDEE0000006295899562000002043C4A523C4044
:10EDFE00800C10203C20100C003C42424242424209
:10EE0E0000007E007E007E000010107C1010007C42
:10EE1E00001008040810007E000810201008007E64
:10EE2E00000C1212101010101010101010109090E4
:10EE3E00601818007E0018180000324C00324C008A
:10EE4E000030484830000000000000001818000094
:10EE5E000000000000180000000F08080808C8286D
:10EE6E0018784444444400000030481020780000D4
:10EE7E000000003C3C3C3C00000000000000000094
:10EE8E000000000000000000000000000000000074
:10EE9E000000000000000000000000000000000064
:10EEAE000000000000000000000000000000000054
:10EEBE000000000000000000000000000000000044
:10EECE000000000000000000000000000000000034
:10EEDE000000000000000000000000000000000024
:10EEEE000000000000000000000000000000000014
:10EEFE000000000000000000000000000000000004
:10EF0E0000000000000000000000000000000000F3
:10EF1E0000000000000000000000000000000000E3
:10EF2E0000000000000000000000000000000000D3
:10EF3E0000000000000000000000000000000000C3
:10EF4E0000000000000000000000000000000000B3
:10EF5E0000000000000000000000000000000000A3
:10EF6E000000000000000000000000000000000093
:10EF7E000000000000000000000000000000000083
:10EF8E0000000000000000000000005F0000000014
:10EF9E00000007000700000000147F147F1400001B
:10EFAE0000242A7F2A1200000026160834320000A0
:10EFBE0000764955225000000000000503000000B5
:10EFCE0000001C2241000000000041221C00000035
:10EFDE000014083E081400000008083E080800004F
:10EFEE00000050300000000000080808080800006B
:10EFFE000000606000000000002010080402000005
:10F00E00003E5149453E00000000427F4000000096
:10F01E000042615149460000002141454B3100003C
:10F02E00001814127F1000000027454545390000D6
:10F03E00003C4A49493000000001017905030000F7
:10F04E00003649494936000000064949291E00008C
:10F05E0000003636000000000000563600000000AA
:10F06E0000000814224100000014141414140000AF
:10F07E0000412214080000000002015109060000A0
:10F08E00003E4149555E0000007E1111117E0000C8
:10F09E00007F494949360000003E414141220000AF
:10F0AE00007F4141221C0000007F49494941000078
:10F0BE00007F090909010000003E4149493A00005C
:10F0CE00007F0808087F00000000417F410000001B
:10F0DE00002041413F000000007F08142241000043
:10F0EE00007F404040400000007F020C027F000085
:10F0FE00007F0408107F0000003E4141413E0000A9
:10F10E00007F090909060000003E4151215E000002
:10F11E00007F09192946000000464949493100007F
:10F12E000001017F01010000003F4040403F000010
:10F13E00001F2040201F0000003F403C403F0000C9
:10F14E00006314081463000000070870080700002D
:10F15E00006151494543000000007F41410000001D
:10F16E000002040810200000000041417F00000052
:10F17E000004020102040000004040404040000034
:10F18E0000000102040000000020545454780000D6
:10F19E00007F4844443800000038444444200000B6
:10F1AE0000384444487F000000385454541800007E
:10F1BE0000087E090102000000085454543C00006F
:10F1CE00007F0804047800000000447D4000000029
:10F1DE00002040443D000000007F10284400000045
:10F1EE000000417F40000000007C041804780000FD
:10F1FE00007C0804047800000038444444380000C1
:10F20E00007C14141408000000081414187C00006C
:10F21E00007C0804040800000048545454200000E8
:10F22E0000043F4440200000003C4040207C000091
:10F23E00001C2040201C0000003C4038403C0000D8
:10F24E000044281028440000000C5050503C000090
:10F25E00004464544C440000000008364100000095
:10F26E000000007F00000000000041360800000092
:10F27E000000000609090600000010385410101096
:10F28E0000FA9F01A49C01FE9E01B67301D2860175
:10F29E00F48B012E8601EC9F0198A00194A00180B1
:10F2AE009D0140A00148A001DE9F0138A001BE9F34
:10F2BE00018A9001DA8D01AE9F017F2052544320C6
:10F2CE00737572206275732049324331204857207E
:10F2DE003A205243333D53434C2C5243343D534416
:10F2EE00410D0A20524231203D4261766172642006
:10F2FE00466F72636565202C205242323D3D52545A
:10F30E004320466F726365650D0A002053504920F5
:10F31E005243303D4353202C5243313D434C434BDB
:10F32E002C5243353D444F555420202055415254C4
:10F33E00203131353230302062647320205241301A
:10F34E003D204F575320445331384232300D0A007E
:10F35E0020417574726573203A2020636F6E666962
:10F36E00672E682C7461626C655F636861722E68CB
:10F37E002C5254435F4453333233315F30362E6850
:10F38E00202C4F6E655F576972655F323032332EB7
:10F39E0068200D0A00204469726563746F727920CB
:10F3AE003A433A5C4D504C4142585F50726F6A6519
:10F3BE006374735C5F31384632374B34325F486F5B
:10F3CE00726C6F67655F3132784D617837323139E3
:10F3DE005F323032332E580D0A00205049433138F7
:10F3EE004632374B3432202B207465787465206496
:10F3FE006566696C616E7420737572203132206D92
:10F40E0061747269636573204D4158373231390D1D
:10F41E000A002050726F6A656374203A205F31389B
:10F42E004632374B34325F486F726C6F67655F31AF
:10F43E0032784D6178373231395F323032330D0ADE
:10F44E0000203320626C6F63732064652034206D5E
:10F45E006174726963657320387838204D6178372E
:10F46E003231390D0A0020436F6E666967202049DC
:10F47E006E7465726E616C20466F73632036344D08
:10F48E00487A0D0A0020536F75726365203A20206A
:10F49E006D61696E2E63205F323032332D3036301F
:10F4AE00310D0A0020456570726F6D203A202E2EA8
:10F4BE002E0D0A004572726F7220006572726F72A5
:10F4CE000044696D0053616D0056656E004A6575A6
:10F4DE00004D6572004D6172004C756E004465639F
:10F4EE00004E6F76004F63740053657000416F7568
:10F4FE00004A756C004A756E004D61690041767266
:10F50E00004D617200466576004A616E0020200053
:10F51E002020202530336420202020202025303349
:10F52E00642020202020202530336420202020201D
:10F53E0020253033642020202020202530336420E5
:10F54E00202020202025303364202020202020253C
:10F55E0030336420202020253033642020202025C5
:10F56E0030336420202020202025303364202020BA
:10F57E0020202025303364202020202530336420A5
:10F58E000D0A00204D73673D782E2E2E782064656F
:10F59E0020302061A0203633206361726163746570
:10F5AE00726573202C207369203E30202C2041661A
:10F5BE006669636865206C65206D65737361676548
:10F5CE0020782E2E2E782070656E64616E742078F1
:10F5DE0020526570203C43523E0D0A002065742077
:10F5EE006166666963686167652054696D6520723E
:10F5FE0065647569742C20706173206427696E666A
:10F60E006F2074656D7065726174757265732070AC
:10F61E00656E64616E74206C65204D736720416663
:10F62E0066696368C3A9203C43523E0D0A0020421E
:10F63E0075666665722064276166666963686167D0
:10F64E006520427566666572206465707569732003
:10F65E003C4F46465345543D307830303230683E4C
:10F66E00202862616E6B3029203234206C6F6E67F9
:10F67E0073203332626974732021200D0A002041F9
:10F68E005454454E54494F4E203A20506F7373696F
:10F69E0062696C6974E920646520666F72E7616760
:10F6AE006520696E69742052544320696E686962E0
:10F6BE00E9652070656E64616E74206C65732074EC
:10F6CE00657374730D0A002052652D4C6563747555
:10F6DE00726520657420616666696368616765207E
:10F6EE00287369206261766172643D3129646573A5
:10F6FE0020382072656769737472657320205254C6
:10F70E004320445333323331200D0A0020526570AA
:10F71E003D78782064652030312061203939203AD7
:10F72E0052657065746974696F6E206475204D73CF
:10F73E00672070656E64616E7420787820437963FB
:10F74E006C657320203C43523E0D0A00204C274529
:10F75E006570726F6D206475205049432065737417
:10F76E0020207072E92D696E697469616C6973E9A4
:10F77E006520646972656374656D656E7420706171
:10F78E0072206C6520636F64650D0A0020436F6DF7
:10F79E0070696C65206C65202573206120257320AF
:10F7AE005554430D0A206176656320766572736940
:10F7BE006F6E20584338203A20202564206574202F
:10F7CE005041434B2025730D0A0020553B32343BEC
:10F7DE0030383B31373B31383B33363B30342320E6
:10F7EE0020706F757220323420416F757420323064
:10F7FE003137202031384833362030343D4A657554
:10F80E0064690D0A0D0A00204C756D3D78782064F0
:10F81E00652030302061A0203135203A5265676C6A
:10F82E00616765204C756D696E6F736974652065CF
:10F83E006E206D6F6465204A4F555220203C435216
:10F84E003E0D0A0020496E69742052544320466FC3
:10F85E007263656520612053616D6564692032377E
:10F86E002F30352F323032332031313A35393A3567
:10F87E00372076696120205242323D30200D0A0039
:10F88E00204269742042616E6720536F6674205364
:10F89E00504920205243323D436C6B202C52433151
:10F8AE003D446F757420205243303D4353202D3E0E
:10F8BE00204D6178373231393A0D0A0020436F6E90
:10F8CE0066696720657420496E6974204F6E6520E5
:10F8DE00576972652062757320706F75722063614F
:10F8EE007074657572204453313842323020656E23
:10F8FE00205241300D0A002053706565643D7878C2
:10F90E00202076697465737365206465206465666E
:10F91E00696C656D656E7420787820646520303171
:10F92E002061A0203939203C43523E0D0A0020426E
:10F93E00414420504C4D2076616C75657321206DCD
:10F94E007573742062652066726F6D205B31332E85
:10F95E002E203233205D20746F205B2030202E2E1F
:10F96E002038205D000D0A2052617070656C206693
:10F97E006F726D617420646520636465203A202285
:10F98E00553B4A4A3B4D4D3B41413B48483B4D4D13
:10F99E003B6A533B2322200D0A0020424144204360
:10F9AE004F52782076616C7565206D757374206981
:10F9BE006E207468652072616E6765203C2D333051
:10F9CE003020746F202B3330305D00204241564181
:10F9DE003D30206F752031202D3E204261766172C0
:10F9EE006420706F75722074726163616765207038
:10F9FE00726F6772616D6D650D0A00204241442081
:10FA0E0053706565642076616C756521206D757324
:10FA1E0074206265206265747765656E20303220D1
:10FA2E00616E642039380D0A0020402064656369D8
:10FA3E006D616C20232534752020736F697420400E
:10FA4E00446576696365203762697473203D2030A2
:10FA5E005825303258200020424144204C756D20EC
:10FA6E0076616C75652021206D757374206265203A
:10FA7E006265747765656E20303020616E6420316A
:10FA8E00300D0A00206578656D706C6520706F759D
:10FA9E0072203A3330204D616920323032332030BB
:10FAAE0032284D61726469292031354833360D0A8A
:10FABE000020506C616765204C756D696E6F7369BF
:10FACE007465204D696E696D616C6520504C4D3DBD
:10FADE0032333A30313C43523E0D0A00204241440B
:10FAEE00205265702076616C756521206D7573747A
:10FAFE00206265747765656E2020303220616E64F9
:10FB0E002035300D0A0020416A75737465204C75DE
:10FB1E006D696E6F736974E920204D41583732312B
:10FB2E0039206175206D696E696D61200D0A0020A6
:10FB3E00525443205570646174653A20553B3330FE
:10FB4E003B30353B32333B31353B33363B30322362
:10FB5E003C43523E0D0A002052654C65637475722B
:10FB6E00652064657320706172616D657472657372
:10FB7E0020656E2020456570726F6D0D0A00205451
:10FB8E006573742070726573656E63652064657647
:10FB9E006963657320737572204275732049324311
:10FBAE00310D0A002072656D706C69732062756686
:10FBBE00666572207769746820737472696E672047
:10FBCE005445585445200D0A002043726565207037
:10FBDE006172616D65747261676520656E20456541
:10FBEE006570726F6D20504943203A2031002023FA
:10FBFE00312041637469766520736F727469652074
:10FC0E00525443205351573D31487A3A200D0A0041
:10FC1E005F31384632374B34325F486F726C6F67E4
:10FC2E00655F3132784D6178373231395F3230323B
:10FC3E0033000D0A45727265757220737572204A13
:10FC4E006F75722053656D61696E65206A532E2043
:10FC5E000D0A000D0A2070423D4F46465345543D55
:10FC6E002520356420736F69742020302534784840
:10FC7E00200D0A00204D736720646F69742065742F
:10FC8E007265203E30206574203C363320636172ED
:10FC9E0073210D0A0020313846374B34322C464F33
:10FCAE0053432036344D487A2C445333323331206B
:10FCBE0020200D0A00486F726C6F6765203132206C
:10FCCE004D6174726963657348203878382032301C
:10FCDE0032330D0A002061666669636865206E6FB7
:10FCEE006D206465206C276170706C696361746946
:10FCFE006F6E0D0A0020496E697420496E7465722C
:10FD0E0072757074202055415254205258200D0A9D
:10FD1E00002074656D706572617475726520416D39
:10FD2E00622E203D25352E32662563430020436C1E
:10FD3E00656172204D61747269636573204D41581F
:10FD4E0037323139200D0A0020496E6974204D6119
:10FD5E00747269636573204D415837323139200D05
:10FD6E000A00205043463837353420666F72204CD7
:10FD7E004344203278313663617273004563726991
:10FD8E0074757265204453333233312E2E2E204F2C
:10FD9E004B0D0A0020496E69745F493243282920B1
:10FDAE00E0203130304B687A3B0D0A000D0A2048B6
:10FDBE00656C70203A2048656C703C43523E2020A2
:10FDCE000D0A00204C6F6E67205472616D65203DE8
:10FDDE002025356420200D0A002054455854452016
:10FDEE00746F20646973706C6179203A20005049F9
:10FDFE00433138462D4B5F44465020312E362E313E
:10FE0E00323500204364652052544320557064619E
:10FE1E007465203A2000204F6C6420526570203D9E
:10FE2E00202533642025632000504346383537346F
:10FE3E004120386269747320492F4F00204F6C6443
:10FE4E002073706565643D20253364202563004C66
:10FE5E004344203231313920327831366361727346
:10FE6E000020546573742055706461746528290DE3
:10FE7E000A0020457461742070696E20524232204F
:10FE8E003D2000504346383537342038626974734C
:10FE9E0020494F00204F6C64204C756D3D2025335A
:10FEAE0064202563002050726573656E74617469F9
:10FEBE006F6E203A00454550524F4D20353132621B
:10FECE00797465730048454C4C4F205041554C4F4A
:10FEDE0020202000207061756C666A756A6F203074
:10FEEE00312000204F4B20666F72204D73670D0A34
:10FEFE0000202020202020202020202020004F4CD9
:10FF0E0045442053534431333036006E6F6E2072A9
:10FF1E006563656E73E900434F52313D2B303031CE
:10FF2E000D0A00504C4D3D32333A30310D0A00204F
:10FF3E0052656769737472652023004A756E2020BE
:10FF4E003120323032330053706565643D31300DEF
:10FF5E000A00204E6577205265703D2000525443B2
:10FF6E0020445333323331005265703D30300D0A28
:10FF7E00004C756D3D30310D0A0031313A31393A50
:10FF8E003436004E657720504C4D3D002025352EE1
:10FF9E003266256300204F6C64203D2000204E65A4
:10FFAE0077203D20004E657720434F52002043645A
:10FFBE00653A200020474F0D0A00206F6B0D0A0096
:10FFCE0054696D653D00646174653D004D6F6973E4
:10FFDE003D00494E46004E414E00696E66006E6110
:10FFEE006E006C6C73006A533D0054693D006C6684
:02FFFE00000001
:020000040001F9
:10000000600E3901D96F000EDB6F000EDD6F080E38
:10001000DF6F000EDE6F110E0301EB6F3C0EEA6F17
:10002000CB0EE82EFED7EA2FFCD7EB2FFAD7D29EC5
:100030003901909F000E3A01456F000E466F000E89
:10004000476F000E656F000E666F000E676F390117
:10005000909F9191A09FA1911BECC0F098ECCBF0E8
:10006000090E0301EB6F1E0EEA6FE40EE82EFED7B9
:10007000EA2FFCD7EB2FFAD700F069ECCEF0000E98
:100080000101696F000E686F200E0301EA6F000E18
:10009000EB6FD89001016835D96E6935DA6ED8906A
:1000A000D936DA360301EA51D926EB51DA22DE6A73
:1000B000DE6ADE6ADD6A0101684B692B695109E17C
:1000C000180E685DD8A067EF80F069EF80F044EF0C
:1000D00080F0000E696F000E686F400E6825D96EC3
:1000E000050E6921DA6E000EDF6E684B692B6951CF
:1000F00009E1400E685DD8A080EF80F082EF80F0CB
:100100006DEF80F0000E696F000E686F000E6825BD
:10011000D96E040E6921DA6E000EDF6E684B692B12
:10012000695109E1800E685DD8A099EF80F09BEFDE
:1001300080F086EF80F0000E0001FC6F040EFD6F72
:10014000B30E026EFE0E036EFEECC9F0000E01014E
:10015000696F000E686FD8906835D96E6935DA6EB0
:10016000930ED926020EDA226F0078FF02F06F009C
:1001700074FF03F0FEECC9F00101684B692B695173
:1001800009E10A0E685DD8A0C8EF80F0CAEF80F0E0
:10019000ABEF80F069ECCEF0FCC0B0F1FDC0B1F186
:1001A0009A0E0101B26FF70EB36F490EB46FFF0ED6
:1001B000B56F880EB66FFF0EB76F090EB96F380EA8
:1001C000B86FFC0EBA6FFD0EBB6F53ECCAF0FCC0EB
:1001D00008F0FDC009F00DECC8F069ECCEF00101AB
:1001E000728DCBB2F6EF80F0F8EF80F000EF81F087
:1001F000030E0A6EF00E096EFF0E0B6E7DECCAF058
:10020000000E0101696F000E686F000E6825D96E3F
:10021000030E6921DA6E000EDF6E684B692B69519F
:1002200009E17F0E685DD8A018EF81F01AEF81F028
:1002300005EF81F0030E036EF00E026EF9ECCEF0C6
:100240000101776F7729D8A428EF81F02AEF81F098
:10025000F4EF81F0000E02018B6F030E8C6FD70E4E
:10026000026EFB0E036EFEECC9F0000E026E030E72
:10027000036EC30E046EFC0E056E62ECC7F0000E3A
:1002800003011F6F000E0E6E000E0D6E200E0F6E1E
:10029000000E106E030E116E9CECC4F0320E3D0188
:1002A000EA6F000E026E030E036EA30E046EFC0EC8
:1002B000056E62ECC7F0000E03011F6F000E0E6E9C
:1002C000200E0D6E200E0F6E000E106E030E116EBE
:1002D0009CECC4F0330E3D01EA6F000E026E030E7B
:1002E000036E310E046EFF0E056E62ECC7F0000E59
:1002F0000E6E600E0D6E100E0F6E000E106E030E61
:10030000116E9CECC4F0340E3D01EA6F000E026EDB
:10031000030E036E550E046EFF0E056E62ECC7F001
:10032000000E0E6E700E0D6E100E0F6E000E106E23
:10033000030E116E9CECC4F0350E3D01EA6F000E09
:10034000026E030E036E760E046EFF0E056E62ECF7
:10035000C7F0000E0E6E800E0D6E100E0F6E000EAA
:10036000106E030E116E9CECC4F0360E3D01EA6F68
:10037000000E026E030E036E7F0E046EFF0E056EFE
:1003800062ECC7F0000E0E6E900E0D6E100E0F6E2A
:10039000000E106E030E116E9CECC4F0370E3D0182
:1003A000EA6F000E026E030E036E250E046EFF0E42
:1003B000056E62ECC7F0000E0E6EA00E0D6E100EF4
:1003C0000F6E000E106E030E116E9CECC4F0380E12
:1003D0003D01EA6F030E0A6EF00E096E630E0B6E9E
:1003E0007DECCAF069ECCEF05A0E026EF70E036E89
:1003F000FEECC9F0000E0001FC6F040EFD6F650EEF
:10040000026EFB0E036EFEECC9F0000E056E000ED0
:10041000046EFCC006F0FDC007F070ECC5F0020EE3
:100420000301EB6FA00EEA6F920EE82EFED7EA2FC3
:10043000FCD7EB2FFAD700F0FCC008F0FDC009F0A4
:100440000DECC8F0000E056E200E046EFCC006F028
:10045000FDC007F070ECC5F0020E0301EB6FA00EBB
:10046000EA6F920EE82EFED7EA2FFCD7EB2FFAD7D1
:1004700000F0FCC008F0FDC009F00DECC8F069EC1C
:10048000CEF0000E0001FC6F040EFD6F000E056E35
:10049000600E046EFCC006F0FDC007F070ECC5F005
:1004A000FCC008F0FDC009F00DECC8F0000120EE22
:1004B00006F0FC51D926FD51DA22000EDF6E040E43
:1004C000FC25096E000EFD210A6E80ECB2F0095089
:1004D00001016E6F000120EE09F0FC51D926FD519B
:1004E000DA22000EDF6E070EFC25096E000EFD21DC
:1004F0000A6E80ECB2F0095001016F6F020E030129
:10050000EB6FA00EEA6F920EE82EFED7EA2FFCD713
:10051000EB2FFAD700F0000E0001FC6F040EFD6F08
:10052000000E056E700E046EFCC006F0FDC007F0F4
:1005300070ECC5F0FCC008F0FDC009F00DECC8F08F
:10054000000120EE06F0FC51D926FD51DA22DF50E1
:100550000301EA6FD00EEA25026E036AFF0E032242
:10056000000E056E0A0E046EABECCEF002C0DDF19B
:1005700003C0DEF1000120EE07F0FC51D926FD5149
:10058000DA22DF500301EA6FEA510101DD250301A0
:10059000EB6F000E0101DE210301EC6FD00EEB25A5
:1005A0000101DD6FFF0E0301EC210101DE6F020E80
:1005B0000301EB6FA00EEA6F920EE82EFED7EA2F32
:1005C000FCD7EB2FFAD700F0000E0101E06F000E10
:1005D0000001FC6F040EFD6F000E056E800E046EB0
:1005E000FCC006F0FDC007F070ECC5F0FCC008F0E0
:1005F000FDC009F00DECC8F0000120EE04F0FC5144
:10060000D926FD51DA22DF50D00F0A0D6F00CCFF42
:10061000E0F120EE05F0FC51D926FD51DA22DF5041
:100620000101E025D00FE06FE0C1E1F1020E03010E
:10063000EB6FA00EEA6F920EE82EFED7EA2FFCD7E2
:10064000EB2FFAD700F0000E1E6E000E0001FC6FBB
:10065000040EFD6F000E056E900E046EFCC006F0D9
:10066000FDC007F070ECC5F0FCC008F0FDC009F05B
:100670000DECC8F0000120EE04F0FC51D926FD512C
:10068000DA22DF50D00F0A0D6F00CCFF1EF020EEF3
:1006900005F0FC51D926FD51DA22DF501E24D00F7F
:1006A0001E6E1E500F0B1E6E020E0301EB6FA00E8E
:1006B000EA6F920EE82EFED7EA2FFCD7EB2FFAD77F
:1006C00000F0000E0101476F000E466F000E0001A2
:1006D000FC6F040EFD6F000E056EA00E046EFCC0D4
:1006E00006F0FDC007F070ECC5F0FCC008F0FDC0DE
:1006F00009F00DECC8F0000120EE06F0FC51D926FF
:10070000FD51DA22DF500301EA6FD00EEA25026EB6
:10071000036AFF0E0322000E056E640E046EABEC3E
:10072000CEF002C046F103C047F1000120EE07F011
:10073000FC51D926FD51DA22DF500301EA6FEA515C
:100740000A0D6F00CCFFEBF36F00D0FFECF301015B
:1007500046510301EB27010147510301EC23200E11
:10076000EB250101466FFE0E0301EC210101476FED
:10077000000120EE08F0FC51D926FD51DA22DF50AD
:100780000301EA6FEA51010146250301EB6F000EF8
:10079000010147210301EC6FD00EEB250101466FEB
:1007A000FF0E0301EC210101476F000120EE05F06F
:1007B000FC51D926FD51DA222D0EDE18D8A4E3EF24
:1007C00083F0E5EF83F0EAEF83F00101466D471F08
:1007D000D8B0472B010147AFF9EF83F0D40E465D47
:1007E000FE0E4759D8A0F7EF83F0F9EF83F007EF3B
:1007F00084F047BF05EF84F02D0E465D010E47598A
:10080000D8A005EF84F007EF84F00BEF84F0000E22
:10081000476F000E466F46C102F047C103F0000E5D
:1008200003BEFF0E046E056E010E54ECB4F002C060
:1008300010F003C011F004C012F005C013F0000E58
:10084000146E000E156EC80E166E420E176E73EC07
:10085000A7F010C041F211C042F212C043F213C01F
:1008600044F269ECCEF0020E0301EB6FA00EEA6FCA
:10087000920EE82EFED7EA2FFCD7EB2FFAD700F026
:10088000A20E026EFD0E036EFEECC9F00AECCFF074
:100890008C0E026EFB0E036EFEECC9F01EECACF08B
:1008A00069ECCEF0FC0E026EFB0E036EFEECC9F09E
:1008B000C20E026EFF0E036EFEECC9F0400E010187
:1008C0008A6F0E0E176E8AC118F0680EB2ECC6F071
:1008D000C80E026EFF0E036EFEECC9F0090E030196
:1008E000EB6F1E0EEA6FE40EE82EFED7EA2FFCD760
:1008F000EB2FFAD700F08C0E026EF60E036EFEECB4
:10090000C9F0CBB486EF84F088EF84F0A1EF84F0D7
:10091000800E026EFE0E036EFEECC9F0CBA493EFC8
:1009200084F095EF84F09AEF84F0310E1BECCFF059
:100930009DEF84F0300E1BECCFF069ECCEF02AEC8A
:10094000C5F0520E0301EB6F2B0EEA6F000EE82E7E
:10095000FED7EA2FFCD7EB2FFAD700F0010E0101EA
:10096000716FD50E026EF60E036EFEECC9F0000E2E
:100970000101676F000E666F7405D8A4C2EF84F0A2
:10098000C4EF84F0DEEF84F03D0E026EFF0E036EC6
:10099000FEECC9F001016651300F1BECCFF0090EDF
:1009A0001BECCFF0010E1A6E0101665103ECCCF086
:1009B0000101776F69ECCEF0E5EF84F0000E1A6E5E
:1009C000665103ECCCF00101776F0101664B672B98
:1009D000675109E1080E665DD8A0F1EF84F0F3EFEE
:1009E00084F0BCEF84F069ECCEF00DECB8F069EC6B
:1009F000CEF0520E0301EB6F2B0EEA6F000EE82EC5
:100A0000FED7EA2FFCD7EB2FFAD700F0CA0E026E02
:100A1000F80E036EFEECC9F08AECCCF045ECB9F0B0
:100A20009EC02AF19FC02BF1A0C02CF1A1C02DF1D6
:100A3000FCC0B0F1FDC0B1F11F0E0101B26FFD0E9F
:100A4000B36F2AC1B4F12BC1B5F12CC1B6F12DC1E0
:100A5000B7F1000EB96FB00EB86F53ECCAF0FCC01E
:100A600008F0FDC009F00DECC8F069ECCEF0000E06
:100A7000146E000E156EC80E166E420E176E46C12D
:100A800002F047C103F0000E03BEFF0E046E056EB8
:100A9000010E54ECB4F002C010F003C011F004C019
:100AA00012F005C013F073ECA7F010C08EF011C067
:100AB0008FF012C090F013C091F02AC192F02BC1B8
:100AC00093F02CC194F02DC195F0EAECA2F08EC009
:100AD0002AF18FC02BF190C02CF191C02DF1810E25
:100AE0000101B06F050EB16F9A0EB26FFF0EB36FBA
:100AF0002AC1B4F12BC1B5F12CC1B6F12DC1B7F1AA
:100B0000000EB96FB00EB86F53ECCAF069ECCEF0BE
:100B1000520E0301EB6F2B0EEA6F000EE82EFED78C
:100B2000EA2FFCD7EB2FFAD700F00101728D000EEF
:100B3000E16F000E656F000E646F000E3D6F000EDA
:100B40003C6F000E0001FA6F000EFB6F000E0201F9
:100B5000666F000E656F200E0001F86F000EF96FD2
:100B60006F0E026EFE0E036EFEECC9F0000E000169
:100B7000FC6F040EFD6F77ECA0F0FCC002F0FDC02E
:100B800003F0D2ECC9F002C03AF103C03BF1FCC063
:100B900054F1FDC055F154C108F055C109F00DECF8
:100BA000C8F069ECCEF0000E0101B06F030EB16F1A
:100BB000D10EB26FFD0EB36F3AC1B4F13BC1B5F1C6
:100BC00053ECCAF0000E086E030E096E0DECC8F06F
:100BD00069ECCEF054C102F055C103F072ECAFF0F5
:100BE000B20E026EFB0E036EFEECC9F0FCC008F004
:100BF000FDC009F00DECC8F069ECCEF0000E01016B
:100C0000656F000E646FBC92BC9ABC808E0E026E43
:100C1000F80E036EFEECC9F0560E026EFD0E036E6A
:100C2000FEECC9F0A9ECB8F0010E29ECCAF03B0EBD
:100C3000026EFD0E036EFEECC9F0B1ECBFF069EC84
:100C4000CEF0BC8069ECCEF03C0E026EF60E036E68
:100C5000FEECC9F0140E026EFB0E036EFEECC9F042
:100C6000000E066E000E076E000E086E000E096E76
:100C7000000E0A6E000E0B6E000E0C6E000E0D6E56
:100C8000000E0E6E000E0F6E000E106E000E116E36
:100C90000A0E45ECBFF0200E0001F86F000EF96F50
:100CA000000E0101676F000E666F675109E1080EC3
:100CB000665DD8A05EEF86F060EF86F062EF86F0AA
:100CC0005BEF87F066510001F8250301EA6F01012F
:100CD00067510001F9210301EB6F580EEA25D96E27
:100CE000000EEB21DA6EDF50066E01016651000145
:100CF000F8250301EC6F010167510001F92103019F
:100D0000ED6F500EEC25D96E000EED21DA6EDF503E
:100D1000076E010166510001F8250301EE6F010124
:100D200067510001F9210301EF6F480EEE25D96EDE
:100D3000000EEF21DA6EDF50086E010166510001EE
:100D4000F8250301F06F010167510001F92103014A
:100D5000F16F400EF025D96E000EF121DA6EDF50F2
:100D6000096E010166510001F8250301F26F0101CE
:100D700067510001F9210301F36F380EF225D96E96
:100D8000000EF321DA6EDF500A6E01016651000198
:100D9000F8250301F46F010167510001F9210301F6
:100DA000F56F300EF425D96E000EF521DA6EDF50A6
:100DB0000B6E010166510001F8250301F66F010178
:100DC00067510001F9210301F76F280EF625D96E4E
:100DD000000EF721DA6EDF500C6E01016651000142
:100DE000F8250301F86F010167510001F9210301A2
:100DF000F96F200EF825D96E000EF921DA6EDF505A
:100E00000D6E010166510001F8250301FA6F010121
:100E100067510001F9210301FB6F180EFA25D96E05
:100E2000000EFB21DA6EDF500E6E010166510001EB
:100E3000F8250301FC6F010167510001F92103014D
:100E4000FD6F100EFC25D96E000EFD21DA6EDF500D
:100E50000F6E010166510001F8250301FE6F0101CB
:100E600067510001F9210301FF6F080EFE25D96EBD
:100E7000000EFF21DA6EDF50106E01016651000195
:100E8000F825D96E010167510001F921DA6EDF50B2
:100E9000116E0101662945ECBFF0150E0301EA6FE2
:100EA000C60EE82EFED7EA2FFCD700F00101664BF4
:100EB000672B55EF86F069ECCEF0010E0101716FE2
:100EC000010E746F69ECCEF0000E026E030E036E1D
:100ED000FF0E046EFE0E056E62ECC7F0000E026E91
:100EE000030E036E72ECAFF0F2ECB5F0E70E026E9B
:100EF000FD0E036EFEECC9F0FCC008F0FDC009F069
:100F00000DECC8F069ECCEF0000E0101416F000E4F
:100F1000406F000E3F6F000E3E6F000E3D6F000EE3
:100F20003C6F000E656F000E646F000E3D6F000E8B
:100F30003C6F000E0001FA6F000EFB6F000E020105
:100F4000666F000E656F200E0001F86F000EF96FDE
:100F5000FCC054F1FDC055F154C108F055C109F071
:100F60000DECC8F069ECCEF0000E0101B06F030E7D
:100F7000B16FD10EB26FFD0EB36F3AC1B4F13BC188
:100F8000B5F153ECCAF0000E086E030E096E0DECBD
:100F9000C8F054C102F055C103F072ECAFF0000E7E
:100FA0000101416F000E406F000E3D6F000E3C6F5F
:100FB000000E3F6F000E3E6F000E0201646F000EC8
:100FC000636FE30E026EFC0E036EFEECC9F0400E82
:100FD000026E050E036E1E0E046EFC0E056E62ECB4
:100FE000C7F0010E0101E16F000E0001FC6F040E5D
:100FF000FD6F77ECA0F0000E0101746F69ECCEF08C
:10100000FCC002F0FDC003F0D2ECC9F002C03AF11E
:1010100003C03BF1FCC054F1FDC055F1030E026E5C
:10102000FD0E036EFEECC9F039018387848193873E
:10103000B29091919491D28E77ECC6F045ECB9F0D4
:101040009EC02AF19FC02BF1A0C02CF1A1C02DF1B0
:10105000000E146E000E156EC80E166E420E176E40
:1010600046C102F047C103F0000E03BEFF0E046E3E
:10107000056E010E54ECB4F002C010F003C011F084
:1010800004C012F005C013F073ECA7F010C08EF08E
:1010900011C08FF012C090F013C091F02AC192F0ED
:1010A0002BC193F02CC194F02DC195F0EAECA2F085
:1010B0008EC02AF18FC02BF190C02CF191C02DF180
:1010C000810E0101B06F050EB16F9A0EB26FFF0E67
:1010D000B36F2AC1B4F12BC1B5F12CC1B6F12DC14A
:1010E000B7F1000EB96FB00EB86F53ECCAF0000E36
:1010F000F7ECBDF0010141BF87EF88F0415109E1F4
:10110000080E405DD8A087EF88F089EF88F0CAEF1D
:1011100089F0000E416F000E406F3C513A5D3B512B
:10112000800A0301EA6F01013D51800A0301EA5977
:10113000D8B09DEF88F09FEF88F0EDEF88F0CBB24C
:10114000A4EF88F0A6EF88F0AEEF88F0FCC008F0BE
:10115000FDC009F00DECC8F069ECCEF00101E151E1
:10116000D8B4B5EF88F0B7EF88F0B8EF88F0E107B2
:10117000000E3D6F000E3C6F000E0001FC6F040E70
:10118000FD6FFCC054F1FDC055F1000E0101436F2D
:10119000000E426F43BFD6EF88F0435109E10C0EB9
:1011A000425DD8A0D6EF88F0D8EF88F0DAEF88F06B
:1011B000C1EF89F042515425D96E43515521DA6E61
:1011C000BA0E4225E16E050E4321E26E6F007FFFED
:1011D000E7FF424B432BCAEF88F001013C513A5DD7
:1011E0000301EA6F01013D513B590301EB6F010E11
:1011F000EA2501013E6F000E0301EB2101013F6F63
:10120000F40E0301EA6FFF0EEB6F3AC1ECF33BC142
:10121000EDF3EA51EC27EB51ED23EC5101013C5D7C
:101220003D51800A0301EE6FED51800AEE59D8B0AE
:101230001CEF89F01EEF89F054EF89F0000E0101D8
:10124000436F000E426F43BF2FEF89F0435109E116
:101250000C0E425DD8A02FEF89F031EF89F033EF0B
:1012600089F0C1EF89F03C5154250301EA6F010177
:101270003D5155210301EB6F010142510301EA2564
:10128000D96E010143510301EB21DA6EBA0E01015F
:101290004225E16E050E4321E26E6F007FFFE7FFFE
:1012A000424B432B23EF89F0000E0101436F000EE8
:1012B000426F7BEF89F001013C5154250301EA6F35
:1012C00001013D5155210301EB6F01014251030121
:1012D000EA25D96E010143510301EB21DA6EBA0E02
:1012E00001014225E16E050E4321E26E6F007FFF92
:1012F000E7FF424B432B3E51425D4351800A0301BD
:10130000EA6F01013F51800A0301EA59D8A08BEF2F
:1013100089F08DEF89F05BEF89F03EC142F13FC16A
:1013200043F1B2EF89F03E51545D0301EA6F0101D0
:101330003F5155590301EB6F010142510301EA2569
:10134000D96E010143510301EB21DA6EBA0E01019E
:101350004225E16E050E4321E26E6F007FFFE7FF3D
:10136000424B432B010143BFBFEF89F0435109E1D9
:101370000C0E425DD8A0BFEF89F0C1EF89F093EF6A
:1013800089F0BA0E026E050E036E72ECAFF0010129
:101390003C4B3D2B0201634B642BF2ECB5F0CBB21E
:1013A000D4EF89F0D6EF89F0D8EF89F043ECADF0B7
:1013B00080ECBDF0000E0101436F000E426FEDEFB7
:1013C00089F0150E0301EA6FC60EE82EFED7EA2F4C
:1013D000FCD700F00101424B432BDD51425DDE5151
:1013E0004359D8A0F6EF89F0F8EF89F0E1EF89F0E2
:1013F000404B412B7505D8A400EF8AF002EF8AF02C
:101400000AEF94F0800E0001FA6F040EFB6F60008B
:10141000EBF3D9FF6000EFF3DAFF480EDE18D8A433
:1014200014EF8AF016EF8AF068EF8AF020EE03F0EE
:10143000FA51D926FB51DA22700EDE18D8A423EF18
:101440008AF025EF8AF068EF8AF0BA0E026EFD0E80
:10145000036EFEECC9F03D0E026EFB0E036EFEEC59
:10146000C9F0920E026EFA0E036EFEECC9F0BF0ECA
:10147000026EFA0E036EFEECC9F0050E026EF90E56
:10148000036EFEECC9F0910E026EF50E036EFEECDB
:10149000C9F0EA0E026EF50E036EFEECC9F01A0EEC
:1014A000026EF70E036EFEECC9F0150E026EF80E1A
:1014B000036EFEECC9F0D90E026EF90E036EFEEC5F
:1014C000C9F069ECCEF0000E0001FA6F000EFB6F60
:1014D0006000EBF3D9FF6000EFF3DAFF550EDE1882
:1014E000D8A475EF8AF077EF8AF0C1EF8AF020EE8A
:1014F00014F0FA51D926FB51DA22230EDE18D8B4A3
:1015000084EF8AF086EF8AF095EF8AF020EE14F0EF
:10151000FA51D926FB51DA223B0EDE18D8A493EFFC
:101520008AF095EF8AF0C1EF8AF0110E026EFE0E7E
:10153000036EFEECC9F0800E086E040E096E0DEC11
:10154000C8F069ECCEF083ECB1F0B8ECC3F0010167
:101550008851CCECCFF001017E6F8751CCECCFF0FD
:1015600001017F6F8651CCECCFF00101806F835178
:10157000CCECCFF00101816F000E0001FA6F000E7C
:10158000FB6F6000EBF3D9FF6000EFF3DAFF4D0E65
:10159000DE18D8A4CEEF8AF0D0EF8AF068EF8BF097
:1015A00020EE01F0FA51D926FB51DA22730EDE1833
:1015B000D8A4DDEF8AF0DFEF8AF068EF8BF020EE41
:1015C00002F0FA51D926FB51DA22670EDE18D8A4B0
:1015D000ECEF8AF0EEEF8AF068EF8BF020EE03F08C
:1015E000FA51D926FB51DA223D0EDE18D8A4FBEFC2
:1015F0008AF0FDEF8AF068EF8BF0000E0401C36FF4
:10160000000E0501406F400E066E050E076E840E3B
:10161000086E040E096E7CECC8F0400E086E050ED4
:10162000096E0DECC8F069ECCEF0400E026E050EAE
:10163000036ED2ECC9F002C064F103C065F1010190
:10164000655109E1050E645DD8A029EF8BF02BEF01
:101650008BF057EF8BF0F10E026EFE0E036EFEEC78
:10166000C9F0050E0301EB6F0F0EEA6FF10EE82EC5
:10167000FED7EA2FFCD7EB2FFAD70101E051D8B4FF
:1016800044EF8BF046EF8BF063EF8BF0E0C1E1F1BC
:10169000B1ECBFF0000E0101416F000E406F000E73
:1016A0003D6F000E3C6F77ECA0F063EF8BF0820E85
:1016B000026EFC0E036EFEECC9F0000E0101E16F3C
:1016C000000E0501406F000E0001FA6F000EFB6F67
:1016D0006000EBF3D9FF6000EFF3DAFF530EDE1882
:1016E000D8A475EF8BF077EF8BF0DDEF8CF020EE68
:1016F00001F0FA51D926FB51DA22700EDE18D8A477
:1017000084EF8BF086EF8BF0DDEF8CF020EE02F0B3
:10171000FA51D926FB51DA22650EDE18D8A493EFD0
:101720008BF095EF8BF0DDEF8CF020EE03F0FA51AB
:10173000D926FB51DA22650EDE18D8A4A2EF8BF071
:10174000A4EF8BF0DDEF8CF020EE04F0FA51D926F7
:10175000FB51DA22640EDE18D8A4B1EF8BF0B3EFA0
:101760008BF0DDEF8CF020EE05F0FA51D926FB511D
:10177000DA223D0EDE18D8A4C0EF8BF0C2EF8BF05A
:10178000DDEF8CF0800E086E040E096E0DECC8F0D3
:10179000090E1BECCFF0000E0101B06F030EB16F0C
:1017A0004A0EB26FFE0EB36FDDC1B4F1DEC1B5F10A
:1017B000000EB76F090EB66F53ECCAF0000E086E3C
:1017C000030E096E0DECC8F0D00E0301EA6FFF0E98
:1017D000EB6F000120EE07F0FA51D926FB51DA2217
:1017E000DF500301EC6FED6BEA51EC27EB51ED2379
:1017F000ED510AE10A0EEC5DD8A001EF8CF004EF88
:101800008CF0010E05EF8CF0000EEE6FEF6BD00E3A
:10181000F06FFF0EF16F000120EE06F0FA51D926AD
:10182000FB51DA22DF500301F26FF36BF051F22724
:10183000F151F323F3510AE10A0EF25DD8A023EF30
:101840008CF026EF8CF0010E27EF8CF0000EEE25C9
:101850000101626F000E0301EF210101636F0001BE
:1018600020EE06F0FA51D926FB51DA22DF500301AF
:10187000EA6FEA510A0D6F00CCFFEBF36F00D0FF67
:10188000ECF3000120EE07F0FA51D926FB51DA22E1
:10189000DF500301ED6FED51EB27000EEC23F00E4E
:1018A000EB250101646FFD0E0301EC210101656F61
:1018B000020E62196311D8A460EF8CF062EF8CF015
:1018C000D2EF8CF064516511D8B469EF8CF06BEFF6
:1018D0008CF0D2EF8CF0655107E1630E645DD8B0F7
:1018E00074EF8CF076EF8CF0D2EF8CF064C1DDF108
:1018F00065C1DEF1000E0A6E760E096E64C102F05B
:1019000065C103F0000E056E0A0E046E28ECC7F0E8
:101910000250300F0B6E7DECCAF0030E0301EB6F2B
:10192000080EEA6F770EE82EFED7EA2FFCD7EB2FD2
:10193000FAD7000E0A6E770E096E64C102F065C117
:1019400003F0000E056E0A0E046EE6ECC8F00250BD
:10195000300F0B6E7DECCAF0030E0301EB6F080E27
:10196000EA6F770EE82EFED7EA2FFCD7EB2FFAD7D7
:10197000AB0E026EFF0E036EFEECC9F0000E056E9C
:10198000700E046E000E066E030E076E70ECC5F04E
:10199000000E086E030E096E0DECC8F069ECCEF077
:1019A000D8EF8CF0090E026EFA0E036EFEECC9F051
:1019B000000E0001FA6F000EFB6F6000EBF3D9FF21
:1019C0006000EFF3DAFF4C0EDE18D8A4EAEF8CF0DB
:1019D000ECEF8CF026EF8EF020EE01F0FA51D926D4
:1019E000FB51DA22750EDE18D8A4F9EF8CF0FBEF6C
:1019F0008CF026EF8EF020EE02F0FA51D926FB5142
:101A0000DA226D0EDE18D8A408EF8DF00AEF8DF003
:101A100026EF8EF020EE03F0FA51D926FB51DA22A0
:101A20003D0EDE18D8A417EF8DF019EF8DF026EFDC
:101A30008EF0800E086E040E096E0DECC8F0000EDC
:101A40000101B06F030EB16FA20EB26FFE0EB36F45
:101A50001EC0B4F1B56B000EB76F090EB66F53EC34
:101A6000CAF0000E086E030E096E0DECC8F0D00E21
:101A70000301EA6FFF0EEB6F000120EE05F0FA5153
:101A8000D926FB51DA22DF500301EC6FED6BEA51EE
:101A9000EC27EB51ED23ED510AE10A0EEC5DD8A0E5
:101AA00054EF8DF057EF8DF0010E58EF8DF0000ED2
:101AB000EE6FEF6BD00EF06FFF0EF16F000120EEB6
:101AC00004F0FA51D926FB51DA22DF500301F26FFC
:101AD000F36BF051F227F151F323F3510AE10A0EAF
:101AE000F25DD8A076EF8DF079EF8DF0010E7AEFF0
:101AF0008DF0000EEE250101626F000E0301EF2153
:101B00000101636F000120EE04F0FA51D926FB5168
:101B1000DA22DF500301EA6FEA510A0D6F00CCFFB1
:101B2000EBF36F00D0FFECF3000120EE05F0FA516B
:101B3000D926FB51DA22DF500301ED6FED51EB277F
:101B4000000EEC23F00EEB250101646FFD0E030186
:101B5000EC210101656F020E62196311D8A4B3EF85
:101B60008DF0B5EF8DF01BEF8EF0655107E10B0E98
:101B7000645DD8B0BEEF8DF0C0EF8DF01BEF8EF03E
:101B800064510F0B1E6E000E0A6E940E096E64C136
:101B900002F065C103F0000E056E0A0E046E28EC1B
:101BA000C7F00250300F0B6E7DECCAF0030E03013C
:101BB000EB6F080EEA6F770EE82EFED7EA2FFCD700
:101BC000EB2FFAD7000E0A6E950E096E64C102F073
:101BD00065C103F0000E056E0A0E046EE6ECC8F057
:101BE0000250300F0B6E7DECCAF0030E0301EB6F59
:101BF000080EEA6F770EE82EFED7EA2FFCD7EB2F00
:101C0000FAD7AB0E026EFF0E036EFEECC9F0000EAB
:101C1000056E900E046E000E066E030E076E70ECDD
:101C2000C5F0000E086E030E096E0DECC8F069ECED
:101C3000CEF021EF8EF0650E026EFA0E036EFEEC12
:101C4000C9F0000E0001FA6F000EFB6F6000EBF3AD
:101C5000D9FF6000EFF3DAFF520EDE18D8A433EF9D
:101C60008EF035EF8EF078EF8FF020EE01F0FA5124
:101C7000D926FB51DA22650EDE18D8A442EF8EF089
:101C800044EF8EF078EF8FF020EE02F0FA51D92673
:101C9000FB51DA22700EDE18D8A451EF8EF053EF0C
:101CA0008EF078EF8FF020EE03F0FA51D926FB5139
:101CB000DA223D0EDE18D8A460EF8EF062EF8EF0CF
:101CC00078EF8FF0800E086E040E096E0DECC8F0F0
:101CD000090E1BECCFF0000E0101B06F030EB16FC7
:101CE000240EB26FFE0EB36FE0C1B4F1B56B000EFF
:101CF000B76F090EB66F53ECCAF0000E086E030EF4
:101D0000096E0DECC8F0D00E0301EA6FFF0EEB6F09
:101D1000000120EE05F0FA51D926FB51DA22DF50FE
:101D20000301EC6FED6BEA51EC27EB51ED23ED5124
:101D30000AE10A0EEC5DD8A0A0EF8EF0A3EF8EF0C2
:101D4000010EA4EF8EF0000EEE6FEF6BD00EF06F71
:101D5000FF0EF16F000120EE04F0FA51D926FB517D
:101D6000DA22DF500301F26FF36BF051F227F151E9
:101D7000F323F3510AE10A0EF25DD8A0C2EF8EF010
:101D8000C5EF8EF0010EC6EF8EF0000EEE250101BC
:101D9000626F000E0301EF210101636F000120EE6D
:101DA00004F0FA51D926FB51DA22DF500301EA6F21
:101DB000EA510A0D6F00CCFFEBF36F00D0FFECF39C
:101DC000000120EE05F0FA51D926FB51DA22DF504E
:101DD0000301ED6FED51EB27000EEC23F00EEB2528
:101DE0000101646FFD0E0301EC210101656F020E1C
:101DF00062196311D8A4FFEF8EF001EF8FF003EFAB
:101E00008FF064C1E0F1E051D8B409EF8FF00BEF2F
:101E10008FF06BEF8FF0510EE06111EF8FF013EF49
:101E20008FF06BEF8FF0000E0A6E840E096E64C1A6
:101E300002F065C103F0000E056E0A0E046E28EC78
:101E4000C7F00250300F0B6E7DECCAF0030E030199
:101E5000EB6F080EEA6F770EE82EFED7EA2FFCD75D
:101E6000EB2FFAD7000E0A6E850E096E64C102F0E0
:101E700065C103F0000E056E0A0E046EE6ECC8F0B4
:101E80000250300F0B6E7DECCAF0030E0301EB6FB6
:101E9000080EEA6F770EE82EFED7EA2FFCD7EB2F5D
:101EA000FAD7000E056E800E046E000E066E030E4D
:101EB000076E70ECC5F0600E026EFF0E036EFEEC56
:101EC000C9F0000E086E030E096E0DECC8F0E0C1FB
:101ED000E1F173EF8FF0000EE06FEA0E026EFA0E82
:101EE000036EFEECC9F0000E0001FA6F000EFB6FEE
:101EF0006000EBF3D9FF6000EFF3DAFF420EDE186B
:101F0000D8A485EF8FF087EF8FF0F9EF8FF020EEF8
:101F100001F0FA51D926FB51DA22410EDE18D8A47D
:101F200094EF8FF096EF8FF0F9EF8FF020EE02F044
:101F3000FA51D926FB51DA22560EDE18D8A4A3EFA7
:101F40008FF0A5EF8FF0F9EF8FF020EE03F0FA514C
:101F5000D926FB51DA22410EDE18D8A4B2EF8FF059
:101F6000B4EF8FF0F9EF8FF020EE04F0FA51D9269C
:101F7000FB51DA223D0EDE18D8A4C1EF8FF0C3EF7B
:101F80008FF0F9EF8FF0800E086E040E096E0DECE5
:101F9000C8F0000120EE05F0FA51D926FB51DA22F3
:101FA000310EDE18D8B4D7EF8FF0D9EF8FF0E8EF0D
:101FB0008FF020EE05F0FA51D926FB51DA22300ECF
:101FC000DE18D8A4E6EF8FF0E8EF8FF0F2EF8FF095
:101FD00020EE05F0FA51D926FB51DA22DF50D00F5E
:101FE0000101746F69ECCEF0000E0001FA6F000E73
:101FF000FB6F6000EBF3D9FF6000EFF3DAFF500EE8
:10200000DE18D8A406EF90F008EF90F036EF92F0CB
:1020100020EE01F0FA51D926FB51DA224C0EDE18DF
:10202000D8A415EF90F017EF90F036EF92F020EE75
:1020300002F0FA51D926FB51DA224D0EDE18D8A44F
:1020400024EF90F026EF90F036EF92F020EE03F0C0
:10205000FA51D926FB51DA223D0EDE18D8A433EF0F
:1020600090F035EF90F036EF92F0800E026E040E95
:10207000036ED2ECC9F0035009E1090E025CD8A04E
:1020800044EF90F046EF90F036EF92F0800E086E3D
:10209000040E096E0DECC8F0090E1BECCFF0000128
:1020A00020EE06F0FA51D926FB51DA22000EDF6E3F
:1020B00020EE09F0FA51D926FB51DA22000EDF6E2C
:1020C000A30E026EFF0E036EFEECC9F0000E056E4D
:1020D000600E046E000E066E030E076E70ECC5F007
:1020E000000E086E030E096E0DECC8F0090E1BEC15
:1020F000CFF0D00E0301EA6FFF0EEB6F000120EE70
:1021000008F0FA51D926FB51DA22DF500301EC6FB7
:10211000ED6BEA51EC27EB51ED23ED510AE10A0E8C
:10212000EC5DD8A096EF90F099EF90F0010E9AEF49
:1021300090F0000EEE6FEF6BD00EF06FFF0EF16FB0
:10214000000120EE04F0FA51D926FB51DA22DF50CB
:102150000301F26FF36BF051F227F151F323F351C6
:102160000AE10A0EF25DD8A0B8EF90F0BBEF90F054
:10217000010EBCEF90F0000EF46FF56BD00EF66F11
:10218000FF0EF76F000120EE05F0FA51D926FB5142
:10219000DA22DF500301F86FF96BF651F827F75197
:1021A000F923F9510AE10A0EF85DD8A0DAEF90F0B0
:1021B000DDEF90F0010EDEEF90F0000EF427000E40
:1021C000F523D00EFA6FFF0EFB6F000120EE07F033
:1021D000FA51D926FB51DA22DF500301FC6FFD6B67
:1021E000FA51FC27FB51FD23FD510AE10A0EFC5D6B
:1021F000D8A0FDEF90F000EF91F0010E01EF91F00B
:10220000000EF427000EF523EE51F4250101626F54
:102210000301EF51F5210101636F000120EE04F08D
:10222000FA51D926FB51DA22DF500301EA6FEA5155
:102230000A0D6F00CCFFEBF36F00D0FFECF3000151
:1022400020EE05F0FA51D926FB51DA22DF500301C6
:10225000ED6FED51EB27000EEC23F00EEB250101A5
:10226000646FFD0E0301EC210101656F000120EE9A
:1022700007F0FA51D926FB51DA22DF500301EA6F49
:10228000EA510A0D6F00CCFFEBF36F00D0FFECF3C7
:10229000000120EE08F0FA51D926FB51DA22DF5076
:1022A0000301ED6FED51EB27000EEC23F00EEB2553
:1022B0000101606FFD0E0301EC210101616F040E4D
:1022C00062196311D8A467EF91F069EF91F029EFDB
:1022D00092F0655109E10D0E645DD8A072EF91F0A6
:1022E00074EF91F029EF92F0655107E1180E645DEB
:1022F000D8B07DEF91F07FEF91F029EF92F060512F
:102300006111D8B486EF91F088EF91F029EF92F047
:10231000615107E1090E605DD8B091EF91F093EF44
:1023200091F029EF92F064C16EF1000120EE04F00B
:10233000FA51D926FB51DA22DF500101896F000ED4
:102340000A6E640E096E89C10BF07DECCAF00001C3
:1023500020EE05F0FA51D926FB51DA22DF500101B7
:10236000896F000E0A6E650E096E89C10BF07DEC57
:10237000CAF0030E0301EB6F080EEA6F770EE82E2A
:10238000FED7EA2FFCD7EB2FFAD760C16FF100011F
:1023900020EE07F0FA51D926FB51DA22DF50010175
:1023A000896F000E0A6E670E096E89C10BF07DEC15
:1023B000CAF0030E0301EB6F080EEA6F770EE82EEA
:1023C000FED7EA2FFCD7EB2FFAD7000120EE08F05A
:1023D000FA51D926FB51DA22DF500101896F000E34
:1023E0000A6E680E096E89C10BF07DECCAF0030E0F
:1023F0000301EB6F080EEA6F770EE82EFED7EA2F87
:10240000FCD7EB2FFAD7910E026EFF0E036EFEEC97
:10241000C9F0000E056E600E046E000E066E030E0F
:10242000076E70ECC5F0030E0301EB6F080EEA6F48
:10243000770EE82EFED7EA2FFCD7EB2FFAD7000E47
:10244000086E030E096E0DECC8F069ECCEF02FEFAC
:1024500092F03C0E026EF90E036EFEECC9F069ECD0
:10246000CEF0000E0001FA6F000EFB6F6000EBF380
:10247000D9FF6000EFF3DAFF430EDE18D8A443EF74
:1024800092F045EF92F007EF94F0000120EE01F09A
:10249000FA51D926FB51DA224F0EDE18D8A453EF99
:1024A00092F055EF92F007EF94F020EE02F0FA511F
:1024B000D926FB51DA22520EDE18D8A462EF92F030
:1024C00064EF92F007EF94F020EE04F0FA51D92671
:1024D000FB51DA223D0EDE18D8A471EF92F073EFB3
:1024E00092F007EF94F0FAC002F0FBC003F0D2ECD8
:1024F000C9F0035009E1090E025CD8A082EF92F006
:1025000084EF92F007EF94F0BB0E026EFF0E036EA5
:10251000FEECC9F0FAC008F0FBC009F00DECC8F001
:10252000090E1BECCFF0000120EE0AF0FA51D9267B
:10253000FB51DA22000EDF6EA30E026EFF0E036E59
:10254000FEECC9F0000E056EA00E046E000E066EC5
:10255000030E076E70ECC5F0000E086E030E096ED8
:102560000DECC8F0D00E0301EA6FFF0EEB6F000117
:1025700020EE08F0FA51D926FB51DA22DF50030190
:10258000EC6FED6BEA51EC27EB51ED23ED510AE1D5
:102590000A0EEC5DD8A0CFEF92F0D2EF92F0010ED0
:1025A000D3EF92F0000EEE6FEF6BD00EF06FFF0ED8
:1025B000F16F000120EE06F0FA51D926FB51DA2224
:1025C000DF500301F26FF36BF051F227F151F32367
:1025D000F3510AE10A0EF25DD8A0F1EF92F0F4EFA8
:1025E00092F0010EF5EF92F0000EF46FF56BD00E45
:1025F000F66FFF0EF76F000120EE07F0FA51D926B3
:10260000FB51DA22DF500301F86FF96BF651F8271E
:10261000F751F923F9510AE10A0EF85DD8A013EF3A
:1026200093F016EF93F0010E17EF93F0000EF427DE
:10263000000EF523EE51F4250101626F0301EF5105
:10264000F5210101636F030E62196311D8A42BEF0A
:1026500093F02DEF93F002EF94F0050E0001FA25B0
:10266000096E000EFB210A6E80ECB2F009C044F145
:102670000AC045F1010145BF49EF93F02C0E445DBE
:10268000010E4559D8B047EF93F049EF93F0FCEFB6
:1026900093F045AF57EF93F0D50E445DFE0E4559CC
:1026A000D8A055EF93F057EF93F0FCEF93F00001B3
:1026B00020EE03F0FA51D926FB51DA22310EDE1852
:1026C000D8A465EF93F067EF93F002EF94F044C164
:1026D00046F145C147F144C102F045C103F0000E87
:1026E00003BEFF0E046E056E010E54ECB4F002C082
:1026F00010F003C011F004C012F005C013F0000E7A
:10270000146E000E156EC80E166E420E176E73EC28
:10271000A7F010C041F211C042F212C043F213C040
:1027200044F2000E0101696F000E686FA50E682566
:10273000096E000E69210A6E68510001FA25030135
:10274000EA6F010169510001FB210301EB6F050EE6
:10275000EA25D96E000EEB21DA6EDF500B6E7DECB0
:10276000CAF0030E0301EB6F080EEA6F770EE82E36
:10277000FED7EA2FFCD7EB2FFAD70101684B692B64
:10278000695109E1040E685DD8A0C9EF93F0CBEF61
:1027900093F096EF93F0B30E026EFF0E036EFEEC15
:1027A000C9F06000EBF3D9FF6000EFF3DAFFDF5010
:1027B000030F1BECCFF03A0E1BECCFF0000E056EB2
:1027C000A00E046E000E066E030E076E70ECC5F0D0
:1027D000030E0301EB6F080EEA6F770EE82EFED7AB
:1027E000EA2FFCD7EB2FFAD7000E086E030E096E06
:1027F0000DECC8F002EF94F0A80E026EF90E036E15
:10280000FEECC9F0000E0001FA6F000EFB6F000E27
:102810000101756F000E6D6FE3510A0DF350E42551
:10282000F00F706F6F51705DD8A019EF94F01BEF2F
:1028300094F026EF94F06E51705DD8B022EF94F0D2
:1028400024EF94F026EF94F0010E6D6F6F51705DE0
:10285000D8B02DEF94F02FEF94F031EF94F0000EFC
:102860006D6F6D51D8A437EF94F039EF94F056EFB7
:1028700094F0000E066E000E076E000E086E000E3D
:10288000096E000E0A6E000E0B6E000E0C6E000E2E
:102890000D6E000E0E6E000E0F6E000E106E000E0E
:1028A000116E0A0E45ECBFF071EF94F01EC006F0F9
:1028B0001EC007F01EC008F01EC009F01EC00AF0BE
:1028C0001EC00BF01EC00CF01EC00DF01EC00EF09E
:1028D0001EC00FF01EC010F01EC011F00A0E45EC15
:1028E000BFF0BA7877ECA0F01CEF88F057EF00F05B
:1028F000000E0001C76F000EC66FA8C0D8F0A9C0B7
:10290000D9F0AAC0DAF0ABC0DBF0DBBF8CEF94F0FB
:102910008AEF94F0A2EF94F0000EC76F010EC66F1D
:10292000D8C002F0D9C003F0DAC004F0DBC005F073
:1029300056ECCDF002C0D8F003C0D9F004C0DAF0F4
:1029400005C0DBF0000E0001DF6F000EDE6F30C14E
:10295000CAF031C1CBF0C651C711D8A4B2EF94F080
:10296000B4EF94F0BCEF94F0010134A5BAEF94F009
:10297000BCEF94F0D7EF94F00001C651C711D8A472
:10298000C4EF94F0C6EF94F0CCEF94F0000EB36F68
:102990002B0EB26FD0EF94F0000EB36F2D0EB26F0E
:1029A000B2C080F3DE4BDF2BCA07D8A0CB07D8C05C
:1029B00002F0D9C003F0DAC004F0DBC005F089EC06
:1029C000BCF002040310D8A4E8EF94F0EAEF94F00E
:1029D00034EF95F0BF0E0001AD6FFF0EAE6FAC513E
:1029E000AF6FB06BAD51AF27AE51B023B05107E11F
:1029F0001A0EAF5DD8B0FFEF94F001EF95F00FEF36
:102A000095F0800EDE25066E030EDF21076EE00EC8
:102A1000086EFF0E096E7CECC8F01BEF95F0800E7F
:102A2000DE25066E030EDF21076EE80E086EFF0E30
:102A3000096E7CECC8F00001FD0ECA27FF0ECB2307
:102A4000A6C012F0A7C013F0800E146E030E156E10
:102A5000CAC016F0CBC017F053ECC1F012C0A6F0FC
:102A600013C0A7F08AEF9AF0D8C002F0D9C003F0E3
:102A7000DAC004F0DBC005F089ECBCF002500310B2
:102A8000D8A445EF95F047EF95F07AEF95F0BF0E9B
:102A90000001AD6FFF0EAE6FAC51AF6FB06BAD51BB
:102AA000AF27AE51B023B05107E11A0EAF5DD8B0D9
:102AB0005CEF95F05EEF95F06CEF95F0800EDE2503
:102AC000066E030EDF21076EE40E086EFF0E096E20
:102AD0007CECC8F01BEF95F0800EDE25066E030E31
:102AE000DF21076EEC0E086EFF0E096E7CECC8F05D
:102AF0001BEF95F0000E0001E06F000EE16F800EFD
:102B0000E26F3F0EE36F000EDD6F000EDC6FD8C08A
:102B100002F0D9C003F0DAC004F0DBC005F0000E0B
:102B2000066E000E076E000E086E000E096E70EC49
:102B3000C2F0D8B09EEF95F0A0EF95F025EF96F09B
:102B4000BFEF95F0E0C010F0E1C011F0E2C012F06C
:102B5000E3C013F0000E146E000E156E200E166EFC
:102B6000410E176E4BECA5F010C0E0F011C0E1F083
:102B700012C0E2F013C0E3F00001DC4BDD2BD8C043
:102B80008EF0D9C08FF0DAC090F0DBC091F0000E6B
:102B9000146E000E156E200E166E410E176EE0C0FC
:102BA00010F0E1C011F0E2C012F0E3C013F04BEC02
:102BB000A5F010C092F011C093F012C094F013C0B1
:102BC00095F006ECBCF00001D8B0E9EF95F0EBEF22
:102BD00095F0A2EF95F00BEF96F0E0C010F0E1C099
:102BE00011F0E2C012F0E3C013F0000E146E000EFC
:102BF000156E200E166E410E176E73ECA7F010C006
:102C0000E0F011C0E1F012C0E2F013C0E3F0000107
:102C1000DC07D8A0DD07D8C08EF0D9C08FF0DAC0AD
:102C200090F0DBC091F0E0C092F0E1C093F0E2C020
:102C300094F0E3C095F006ECBCF00001D8A023EFBF
:102C400096F025EF96F0EDEF95F0ACC008F0096A2C
:102C5000E0ECCBF008500001CD6FCDC0CCF0670E9A
:102C6000CD19D8A436EF96F038EF96F060EF96F0D5
:102C7000010132513311D8A440EF96F042EF96F0A3
:102C800046EF96F0000E336F010E326F33BF53EFF5
:102C900096F0335106E13205D8B051EF96F053EF7C
:102CA00096F05AEF96F0000E0001C96F060EC86F3D
:102CB0006AEF96F032C1C8F033C1C9F06AEF96F0FE
:102CC000010133BF66EF96F068EF96F053EF96F090
:102CD0005AEF96F0670E0001CD19D8A472EF96F066
:102CE00074EF96F0A3EF96F0DDAF82EF96F0FC0E56
:102CF000DC5DFF0EDD59D8A080EF96F082EF96F0F4
:102D0000A1EF96F0FF0EAD6FFF0EAE6FC8C0AFF033
:102D1000C9C0B0F0AD51AF27AE51B023DC51AF5DAB
:102D2000B051800AB16FDD51800AB159D8A09BEF34
:102D300096F09DEF96F0A1EF96F0660ECC6FA3EFA4
:102D400096F0650ECC6FC8C0BEF0C9C0BFF0670E6C
:102D5000CD19D8A4AEEF96F0B0EF96F0C0EF96F094
:102D6000660ECC19D8A4B7EF96F0B9EF96F0C2EF83
:102D700096F0DDBFC0EF96F0BEEF96F0C2EF96F092
:102D8000BE4BBF2B660ECC19D8A4C9EF96F0CBEF83
:102D900096F0EBEF96F0DDBFD2EF96F0D0EF96F025
:102DA000DEEF96F0000EE06F000EE16F800EE26F36
:102DB0003F0EE36F000EDD6F000EDC6F670ECD1966
:102DC000D8B4E5EF96F0E7EF96F0EBEF96F0DC5134
:102DD000BE27DD51BF23000ED76F000ED66FD8C0BF
:102DE000CEF0D9C0CFF0DAC0D0F0DBC0D1F0E0C077
:102DF000C0F0E1C0C1F0E2C0C2F0E3C0C3F07CEFBC
:102E000097F0CEC010F0CFC011F0D0C012F0D1C0FA
:102E100013F0E0C014F0E1C015F0E2C016F0E3C01A
:102E200017F073ECA7F010C08EF011C08FF012C035
:102E300090F013C091F067ECAEF08EC0D2F08FC06E
:102E4000D3F090C0D4F091C0D5F0D2C002F0D3C07E
:102E500003F0D4C004F0D5C005F083ECBBF002C091
:102E6000C4F003C0C5F0CEC09EF0CFC09FF0D0C06C
:102E7000A0F0D1C0A1F0E0C014F0E1C015F0E2C0B4
:102E800016F0E3C017F0D2C010F0D3C011F0D4C0D8
:102E900012F0D5C013F04BECA5F010C0A2F011C099
:102EA000A3F012C0A4F013C0A5F0BCECCBF09EC000
:102EB000CEF09FC0CFF0A0C0D0F0A1C0D1F0E0C054
:102EC00010F0E1C011F0E2C012F0E3C013F0000E08
:102ED000146E000E156E200E166E410E176E73ECFA
:102EE000A7F010C0E0F011C0E1F012C0E2F013C092
:102EF000E3F00001D64BD72BBE51D65DD751800AE7
:102F0000AD6FBF51800AAD59D8A089EF97F08BEF14
:102F100097F001EF97F0E0C010F0E1C011F0E2C0CF
:102F200012F0E3C013F0000E146E000E156EA00E2A
:102F3000166E400E176E4BECA5F010C0D2F011C00B
:102F4000D3F012C0D4F013C0D5F0CEC08EF0CFC0F5
:102F50008FF0D0C090F0D1C091F0D2C092F0D3C029
:102F600093F0D4C094F0D5C095F006ECBCF000010D
:102F7000D8B0BDEF97F0BFEF97F0C9EF97F0000E14
:102F8000D26F000ED36F000ED46F000ED56FF2EF2C
:102F900097F0CEC002F0CFC003F0D0C004F0D1C093
:102FA00005F0D2C006F0D3C007F0D4C008F0D5C0F9
:102FB00009F070ECC2F0D8A0E0EF97F0E2EF97F0E4
:102FC000F2EF97F00001C4B1E8EF97F0EAEF97F065
:102FD000F2EF97F0000ED26F000ED36F000ED46F99
:102FE000000ED56FD8C08EF0D9C08FF0DAC090F047
:102FF000DBC091F0D2C092F0D3C093F0D4C094F073
:10300000D5C095F0EAECA2F08EC0CEF08FC0CFF024
:1030100090C0D0F091C0D1F0CEC08EF0CFC08FF074
:10302000D0C090F0D1C091F0000E146E000E156E5D
:10303000200E166E410E176EC0C010F0C1C011F008
:10304000C2C012F0C3C013F04BECA5F010C092F058
:1030500011C093F012C094F013C095F006ECBCF0D0
:103060000001D8A036EF98F038EF98F060EF98F0B4
:10307000DC4BDD2BC0C010F0C1C011F0C2C012F09B
:10308000C3C013F0000E146E000E156E200E166EE7
:10309000410E176E4BECA5F010C0C0F011C0C1F08E
:1030A00012C0C2F013C0C3F0660E0001CC19D8A440
:1030B0005CEF98F05EEF98F060EF98F0BE4BBF2B9E
:1030C000C0C0E0F0C1C0E1F0C2C0E2F0C3C0E3F0B4
:1030D000650ECC19D8B46FEF98F071EF98F077EFD8
:1030E00098F0DCC0BCF0DDC0BDF07BEF98F0000EC6
:1030F000BD6F000EBC6F000EBB6F000EBA6F000EEE
:10310000B96F000EB86F000ED76F000ED66F78EF54
:1031100099F0CEC010F0CFC011F0D0C012F0D1C0E5
:1031200013F0E0C014F0E1C015F0E2C016F0E3C007
:1031300017F073ECA7F010C08EF011C08FF012C022
:1031400090F013C091F067ECAEF08EC0D2F08FC05B
:10315000D3F090C0D4F091C0D5F0D2C002F0D3C06B
:1031600003F0D4C004F0D5C005F083ECBBF002C07E
:10317000C4F003C0C5F0010134B9C1EF98F0C3EF4A
:1031800098F0E1EF98F00001C451C511D8A4CBEF3D
:1031900098F0CDEF98F0E1EF98F0670ECD19D8A434
:1031A000D4EF98F0D6EF98F0E1EF98F0BDBFDDEFE7
:1031B00098F0DBEF98F0E1EF98F0B84BB92B2CEFDB
:1031C00099F00001BA51BB11D8A4E9EF98F0EBEFE8
:1031D00098F015EF99F0BDBFF2EF98F0F0EF98F08E
:1031E00015EF99F0800EDE25D96E030EDF21DA6E21
:1031F0002E0EDF6EDE4BDF2BCA07D8A0CB07000EEA
:10320000BB6F010EBA6F15EF99F0800EDE25D96EF7
:10321000030EDF21DA6E300EDF6EDE4BDF2BCA07C6
:10322000D8A0CB07B807D8A0B907B851B911D8A40E
:103230001CEF99F01EEF99F005EF99F0800EDE2556
:10324000D96E030EDF21DA6EC451300FDF6EDE4B14
:10325000DF2BCA07D8A0CB07CEC09EF0CFC09FF00F
:10326000D0C0A0F0D1C0A1F0E0C014F0E1C015F0D2
:10327000E2C016F0E3C017F0D2C010F0D3C011F0D6
:10328000D4C012F0D5C013F04BECA5F010C0A2F0E2
:1032900011C0A3F012C0A4F013C0A5F0BCECCBF099
:1032A0009EC0CEF09FC0CFF0A0C0D0F0A1C0D1F0A2
:1032B000E0C010F0E1C011F0E2C012F0E3C013F082
:1032C000000E146E000E156E200E166E410E176E57
:1032D00073ECA7F010C0E0F011C0E1F012C0E2F012
:1032E00013C0E3F00001BC07D8A0BD07D64BD72B15
:1032F000BE51D65DD751800AAD6FBF51800AAD591E
:10330000D8B085EF99F087EF99F095EF99F0DFBF8E
:1033100093EF99F0DF5109E14B0EDE5DD8A093EFFA
:1033200099F095EF99F089EF98F0BA51BB11D8A4B4
:103330009CEF99F09EEF99F0B1EF99F0010134A95B
:10334000A4EF99F0A6EF99F0B1EF99F0800E00018B
:10335000DE25D96E030EDF21DA6E2E0EDF6EDE4B18
:10336000DF2B800E0001DE25D96E030EDF21DA6E21
:10337000000EDF6E650ECC19D8A4C1EF99F0C3EF33
:1033800099F020EF95F0000ED76F4F0ED66F800E9C
:10339000D625D96E030ED721DA6E000EDF6E000E31
:1033A000C76F000EC66FDDBFDAEF99F0D8EF99F066
:1033B000E2EF99F0000EC76F010EC66FDC6DDD1FE6
:1033C000D8B0DD2B000EC96F020EC86F13EF9AF054
:1033D000D607D8A0D707800ED625D96E030ED721E1
:1033E000DA6EDCC002F0DDC003F0000E056E0A0EDE
:1033F000046E18ECC2F00250300FDF6EDCC002F039
:10340000DDC003F0000E056E0A0E046EB6ECC1F0CE
:1034100002C0DCF003C0DDF00001C807D8A0C90776
:10342000CA07D8A0CB07DC51DD11D8A41AEF9AF057
:103430001CEF9AF0E8EF99F0C9BF29EF9AF0C95153
:1034400006E1C805D8B027EF9AF029EF9AF0E8EF27
:1034500099F0D607D8A0D707C651C711D8A433EF23
:103460009AF035EF9AF03BEF9AF0000EB56F2B0E05
:10347000B46F3FEF9AF0000EB56F2D0EB46F800E53
:10348000D625D96E030ED721DA6E6000D3F2DFFFA6
:10349000CA07D8A0CB07D607D8A0D707BF0EAD6FF5
:1034A000FF0EAE6FAC51AF6FB06BAD51AF27AE51E9
:1034B000B023B05109E11A0EAF5DD8A062EF9AF0C7
:1034C00064EF9AF06AEF9AF0000EB76F650EB66F70
:1034D0006EEF9AF0000EB76F450EB66F800ED625D0
:1034E000D96E030ED721DA6E6000DBF2DFFFCA0768
:1034F000D8A0CB07800EDE25066E030EDF21076EF7
:10350000800ED625086E030ED721096E7CECC8F01C
:1035100020EF95F0120060009BF3D9FF60009FF34D
:10352000DAFF6F007BFFF6FF6F0077FFF7FF000EFB
:10353000F86E0800F550250AD8A4A1EF9AF0A3EF81
:103540009AF053EFA0F060009BF3D9FF60009FF367
:10355000DAFFDE2A000EDD22000E0101316F000EBF
:10356000306F30C134F131C135F132693369000E49
:103570009D6F000E9C6F12EF9BF001013481600083
:103580009BF3D9FF60009FF3DAFFDE2A000EDD22F5
:1035900012EF9BF001013483BFEF9AF001013485F3
:1035A000BFEF9AF001013487BFEF9AF0010134892F
:1035B000BFEF9AF0000E01019D6F010E9C6F12EF9C
:1035C0009BF060009BF3D9FF60009FF3DAFF6F0070
:1035D0007BFFF6FF6F0077FFF7FF000EF86E080025
:1035E000F5500001EA6FEB6BEB51000AD8B4FBEF2A
:1035F0009AF0DAEF9AF0EA51200AD8B4D2EF9AF0B2
:10360000030AD8B4D6EF9AF0080AD8B4CEEF9AF0ED
:10361000060AD8B4BDEF9AF01D0AD8B4CAEF9AF0E2
:10362000DAEF9AF09C519D11D8B419EF9BF01BEF83
:103630009BF0E1EF9AF034A120EF9BF022EF9BF09A
:1036400023EF9BF0349360009BF3D9FF60009FF35E
:10365000DAFF6F007BFFF6FF6F0077FFF7FF000ECA
:10366000F86E0800F5502A0AD8A439EF9BF03BEF1A
:103670009BF06EEF9BF060009BF3D9FF60009FF31F
:10368000DAFFDE2A000EDD226000A3F3D9FF60001E
:10369000A7F3DAFF6F007CFFEAF0020EDE266F0070
:1036A0007CFFEBF0000EDD226000ABF3D9FF600081
:1036B000AFF3DAFF6F0078FF30F16F0074FF31F184
:1036C00031BF67EF9BF065EF9BF0B1EF9BF034816A
:1036D000306D311FD8B0312BB1EF9BF060009BF300
:1036E000D9FF60009FF3DAFF6F0078FF09F06F00E9
:1036F00074FF0AF080ECB2F009C030F10AC031F179
:103700008BEF9BF060009BF3D9FF60009FF3DAFF23
:10371000DE2A000EDD22D00E0001EA6FFF0EEB6FF5
:1037200060009BF3D9FF60009FF3DAFF6F007BFF1F
:10373000F6FF6F0077FFF7FF000EF86E0800F550F8
:10374000EC6FED6BEA51EC27EB51ED23ED5109E104
:103750000A0EEC5DD8A0AFEF9BF0B1EF9BF082EFCB
:103760009BF060009BF3D9FF60009FF3DAFF6F00CE
:103770007BFFF6FF6F0077FFF7FF000EF86E080083
:10378000F5502E0AD8A4C7EF9BF0C9EF9BF059EF74
:103790009CF0000E0101336F000E326F60009BF34E
:1037A000D9FF60009FF3DAFFDE2A000EDD22600001
:1037B0009BF3D9FF60009FF3DAFF6F007BFFF6FFFA
:1037C0006F0077FFF7FF000EF86E0800F5502A0A29
:1037D000D8A4EDEF9BF0EFEF9BF016EF9CF06000AC
:1037E0009BF3D9FF60009FF3DAFFDE2A000EDD2293
:1037F0006000A3F3D9FF6000A7F3DAFF6F007CFF3E
:10380000EAF0020EDE266F007CFFEBF0000EDD22F8
:103810006000ABF3D9FF6000AFF3DAFF6F0078FF11
:1038200032F16F0074FF33F159EF9CF060009BF3AD
:10383000D9FF60009FF3DAFF6F0078FF09F06F0097
:1038400074FF0AF080ECB2F009C032F10AC033F123
:1038500033EF9CF060009BF3D9FF60009FF3DAFF29
:10386000DE2A000EDD22D00E0001EA6FFF0EEB6FA4
:1038700060009BF3D9FF60009FF3DAFF6F007BFFCE
:10388000F6FF6F0077FFF7FF000EF86E0800F550A7
:10389000EC6FED6BEA51EC27EB51ED23ED5109E1B3
:1038A0000A0EEC5DD8A057EF9CF059EF9CF02AEF80
:1038B0009CF060009BF3D9FF60009FF3DAFF6F007C
:1038C0007BFFF6FF6F0077FFF7FF000EF86E080032
:1038D000F550086E096AE0ECCBF008500101AC6FBE
:1038E000AC51D8B476EF9CF078EF9CF0C4EF9CF02C
:1038F00060009BF3D9FF60009FF3DAFF6F0078FF51
:10390000EAF06F0074FFEBF0010E0001EA27000EF1
:10391000EB236000ABF3F6FF6000AFF3F7FF000EA0
:10392000F86E0800F550086E096AE0ECCBF008501C
:103930000101AD6FAD51D8B4A0EF9CF0A2EF9CF0A7
:10394000C4EF9CF060009BF3D9FF60009FF3DAFFA7
:103950006F0078FFEAF06F0074FFEBF0020E0001D9
:10396000EA27000EEB236000ABF3F6FF6000AFF335
:10397000F7FF000EF86E0800F550086E096AE0ECDB
:10398000CBF008500101AE6F60009BF3D9FF6000DF
:103990009FF3DAFF6F007BFFF6FF6F0077FFF7FF03
:1039A000000EF86E0800F550630AD8A4DAEF9CF018
:1039B000DCEF9CF00BEF9DF060009BF3D9FF600003
:1039C0009FF3DAFFDE2A000EDD226000A3F3D9FFA9
:1039D0006000A7F3DAFF6F007CFFEAF0020EDE263C
:1039E0006F007CFFEBF0000EDD226000ABF3D9FF2F
:1039F0006000AFF3DAFFDF50AF6FE4C00BF0E5C05B
:103A00000CF0AFC10DF06DECBEF00BC0E4F00CC0DB
:103A1000E5F076EFA0F060009BF3D9FF60009FF324
:103A2000DAFF6F007BFFF6FF6F0077FFF7FF000EF6
:103A3000F86E0800F550640AD8B421EF9DF023EF2A
:103A40009DF03BEF9DF060009BF3D9FF60009FF37A
:103A5000DAFF6F007BFFF6FF6F0077FFF7FF000EC6
:103A6000F86E0800F550690AD8A439EF9DF03BEFD5
:103A70009DF085EF9DF060009BF3D9FF60009FF300
:103A8000DAFFDE2A000EDD226000A3F3D9FF60001A
:103A9000A7F3DAFF6F007CFFEAF0020EDE266F006C
:103AA0007CFFEBF0000EDD226000ABF3D9FF60007D
:103AB000AFF3DAFF6F0078FF92F16F0074FF93F1BC
:103AC000000E93BFFF0E946F956F966F976F986F70
:103AD000996FE4C081F0E5C082F092C183F093C198
:103AE00084F094C185F095C186F096C187F097C1A6
:103AF00088F098C189F099C18AF041ECA9F081C0A1
:103B0000E4F082C0E5F076EFA0F0660EAC19D8A420
:103B10008CEF9DF08EEF9DF0E1EF9DF060009BF348
:103B2000D9FF60009FF3DAFF6F007BFFF6FF6F00A5
:103B300077FFF7FF000EF86E08006F00D4FFAFF1BB
:103B400060009BF3D9FF60009FF3DAFFDE2A000ECE
:103B5000DD226000A3F3D9FF6000A7F3DAFF6F0056
:103B60007CFFEAF0040EDE266F007CFFEBF0000E17
:103B7000DD226000ABF3D9FF6000AFF3DAFF6F0026
:103B800078FFA8F16F0078FFA9F16F0078FFAAF124
:103B90006F0078FFABF1E4C0A6F0E5C0A7F0A8C1C4
:103BA000A8F0A9C1A9F0AAC1AAF0ABC1ABF0AFC1FE
:103BB000ACF078EC94F0A6C0E4F0A7C0E5F076EFA6
:103BC000A0F0AC0E026E010E036EFC0E046EFF0E32
:103BD000056E000E076E020E066E64ECB7F0025022
:103BE0000310D8A4F6EF9DF0F8EF9DF08CEF9EF057
:103BF00060009BF3D9FF60009FF3DAFF6F0078FF4E
:103C0000EAF06F0074FFEBF0010E0001EA27000EEE
:103C1000EB236000ABF3F6FF6000AFF3F7FF000E9D
:103C2000F86E08006F00D4FFAFF1BF0EEA6FFF0E11
:103C3000EB6F60009BF3D9FF60009FF3DAFF6F002A
:103C40007BFFF6FF6F0077FFF7FF000EF86E0800AE
:103C5000F550EC6FED6BEA51EC27EB51ED23ED5194
:103C600007E11A0EEC5DD8B038EF9EF03AEF9EF007
:103C70005EEF9EF06000A3F3D9FF6000A7F3DAFFC8
:103C80006F007CFFEAF0040EDE266F007CFFEBF095
:103C9000000EDD226000ABF3D9FF6000AFF3DAFF66
:103CA0006F0078FFA8F16F0078FFA9F16F0078FF2F
:103CB000AAF16F0078FFABF180EF9EF06000A3F3F4
:103CC000D9FF6000A7F3DAFF6F007CFFEAF0040E73
:103CD000DE266F007CFFEBF0000EDD226000ABF310
:103CE000D9FF6000AFF3DAFF6F0078FFA8F16F0033
:103CF00078FFA9F16F0078FFAAF16F0078FFABF1B0
:103D0000020E60009BF3D9FF60009FF3DAFFDE260E
:103D1000000EDD22CBEF9DF060009BF3D9FF600029
:103D20009FF3DAFF6F007BFFF6FF6F0077FFF7FF6F
:103D3000000EF86E0800F550730AD8B4A2EF9EF09A
:103D4000A4EF9EF0C3EF9EF060009BF3D9FF6000EC
:103D50009FF3DAFF6F0078FF02F06F0074FF03F04B
:103D6000F00E046EFF0E056E000E076E030E066E5B
:103D700064ECB7F002500310D8A4C1EF9EF0C3EF7B
:103D80009EF01DEF9FF060009BF3D9FF60009FF352
:103D9000DAFF6F007BFFF6FF6F0077FFF7FF000E83
:103DA000F86E0800F550730AD8B4D9EF9EF0DBEF37
:103DB0009EF0E2EF9EF0000E01019F6F030E9E6FDA
:103DC000E7EF9EF0000E01019F6F010E9E6F6000F5
:103DD0009BF3D9FF60009FF3DAFF9E51DE269F51CF
:103DE000DD226000A3F3D9FF6000A7F3DAFF6F00C4
:103DF0007CFFEAF0020EDE266F007CFFEBF0000E87
:103E0000DD226000ABF3D9FF6000AFF3DAFF6F0093
:103E100078FF9AF16F0074FF9BF1E4C00BF0E5C0EE
:103E20000CF09AC10DF09BC10EF078ECB3F00BC012
:103E3000E4F00CC0E5F076EFA0F060009BF3D9FF52
:103E400060009FF3DAFF6F007BFFF6FF6F0077FFE4
:103E5000F7FF000EF86E0800F550750AD8A433EF8E
:103E60009FF035EF9FF081EF9FF060009BF3D9FF4B
:103E700060009FF3DAFFDE2A000EDD226000A3F36C
:103E8000D9FF6000A7F3DAFF6F007CFFEAF0020EB3
:103E9000DE266F007CFFEBF0000EDD226000ABF34E
:103EA000D9FF6000AFF3DAFF6F0078FFECF06F002E
:103EB00074FFEDF0ECC0A0F1EDC0A1F10101A26B27
:103EC000A36BA46BA56BA66BA76BE4C081F0E5C0E8
:103ED00082F0A0C183F0A1C184F0A2C185F0A3C18A
:103EE00086F0A4C187F0A5C188F0A6C189F0A7C15A
:103EF0008AF07BECB0F081C0E4F082C0E5F076EFB0
:103F0000A0F060009BF3D9FF60009FF3DAFF6F0021
:103F10007BFFF6FF6F0077FFF7FF000EF86E0800DB
:103F2000F550780AD8B497EF9FF099EF9FF0B1EF72
:103F30009FF060009BF3D9FF60009FF3DAFF6F00F2
:103F40007BFFF6FF6F0077FFF7FF000EF86E0800AB
:103F5000F550580AD8A4AFEF9FF0B1EF9FF011EFE2
:103F6000A0F060009BF3D9FF60009FF3DAFF6F00C1
:103F70007BFFF6FF6F0077FFF7FF000EF86E08007B
:103F80006F00D4FFAFF160009BF3D9FF60009FF397
:103F9000DAFFDE2A000EDD226000A3F3D9FF600005
:103FA000A7F3DAFF6F007CFFEAF0020EDE266F0057
:103FB0007CFFEBF0000EDD226000ABF3D9FF600068
:103FC000AFF3DAFF6F0078FFECF06F0074FFEDF0F5
:103FD000ECC0A0F1EDC0A1F10101A26BA36BA46B39
:103FE000A56BA66BA76BE4C081F0E5C082F0A0C111
:103FF00083F0A1C184F0A2C185F0A3C186F0A4C161
:1040000087F0A5C188F0A6C189F0A7C18AF0AFC129
:104010008BF0C0ECAAF081C0E4F082C0E5F076EF4E
:10402000A0F060009BF3D9FF60009FF3DAFF6F0000
:104030007BFFF6FF6F0077FFF7FF000EF86E0800BA
:10404000F550250AD8A427EFA0F029EFA0F043EF00
:10405000A0F060009BF3D9FF60009FF3DAFFDE2A37
:10406000000EDD22000E036E250E026EE4C004F089
:10407000E5C005F0D9ECBEF0000E0001E56F010EC1
:10408000E46F76EFA0F060009BF3D9FF60009FF330
:10409000DAFFDE2A000EDD22000E0001E56F000EC1
:1040A000E46F76EFA0F060009BF3D9FF60009FF310
:1040B000DAFF6F007BFFF6FF6F0077FFF7FF000E60
:1040C000F86E0800F550026E036AE4C004F0E5C023
:1040D00005F0D9ECBEF060009BF3D9FF60009FF3C0
:1040E000DAFFDE2A000EDD223CEFA0F01200000E07
:1040F0000001FC6F040EFD6F0101E151D8A483EFB4
:10410000A0F085EFA0F018EFA2F0000E0F6E000EE9
:104110000E6E000E0E24D96E040E0F20DA6E000E05
:10412000DF6E0E4A0F2A0FBE9FEFA0F00F5009E17D
:10413000600E0E5CD8A09FEFA0F0A1EFA0F089EF79
:10414000A0F0000E0001FC6F040EFD6F000E0101D7
:10415000526F040E536F60004BF5D9FF60004FF5AE
:10416000DAFF200EDF6E010E5225026E000E532183
:10417000036EE30E046E010E056E000E076E090E4F
:10418000066E53ECC4F001017405D8A4CAEFA0F088
:10419000CCEFA0F0DBEFA0F0CE0E026EFF0E036EB0
:1041A000FEECC9F052C108F053C109F00DECC8F0A3
:1041B0003B0E1BECCFF0010120EE09F05251D92645
:1041C0005351DA22200EDF6E0A0E5225506F000E78
:1041D0005321516F50C102F051C103F08551020DBE
:1041E000A70EF324D96E020EF420DA6E6F0078FF6A
:1041F00004F06F0074FF05F062ECC7F050C102F0EC
:1042000051C103F0D2ECC9F002C00EF003C00FF0B0
:1042100001017405D8A40FEFA1F011EFA1F020EF78
:10422000A1F0F40E026EFF0E036EFEECC9F050C159
:1042300008F051C109F00DECC8F03B0E1BECCFF0BB
:104240000E5001015025D96E0F505121DA6E200E0B
:10425000DF6E0E5050250C6E0F5051210D6E010E69
:104260000C244A6F000E0D204B6F60002BF5D9FF18
:1042700060002FF5DAFF600093FBDFFF20EE01F016
:104280004A51D9264B51DA22600097FBDFFF20EE1E
:1042900002F04A51D9264B51DA22000EDF6E740526
:1042A000D8A455EFA1F057EFA1F066EFA1F0D40E1E
:1042B000026EFF0E036EFEECC9F04AC108F04BC15E
:1042C00009F00DECC8F03B0E1BECCFF0010120EE25
:1042D00002F04A51D9264B51DA22200EDF6E030E2E
:1042E0004A254E6F000E4B214F6F4EC102F04FC159
:1042F00003F08151020DD00EF324D96E030EF42089
:10430000DA6E6F0078FF04F06F0074FF05F062EC66
:10431000C7F04EC102F04FC103F0D2ECC9F002C0A9
:104320000EF003C00FF001017405D8A49AEFA1F0BC
:104330009CEFA1F0ABEFA1F0DA0E026EFF0E036E60
:10434000FEECC9F04EC108F04FC109F00DECC8F009
:104350003B0E1BECCFF00E5001014E25D96E0F50D5
:104360004F21DA6E200EDF6E0E504E254C6F0F502F
:104370004F214D6F810E026E050E036ED2ECC9F017
:1043800002C00EF003C00FF04CC102F04DC103F0AB
:10439000810E046E050E056E0EC006F00FC007F00C
:1043A00053ECC4F04CC102F04DC103F0D2ECC9F0A3
:1043B00002C00EF003C00FF00E5001014C25D96E63
:1043C0000F504D21DA6E200EDF6E0E504C250C6E14
:1043D0000F504D210D6E010E0C24D96E000E0D20D4
:1043E000DA6E000EDF6E7405D8A4F9EFA1F0FBEFD2
:1043F000A1F009EFA2F0F80E026EFF0E036EFEECC4
:10440000C9F04CC108F04DC109F00DECC8F069ECE1
:10441000CEF0000E0501406FFCC002F0FDC003F0BD
:10442000D2ECC9F002C03AF103C03BF1CDEFA2F0EB
:10443000000E05017F6F000E0001FC6F040EFD6F82
:10444000000E0F6E000E0E6E6000F3F3D9FF6000D9
:10445000F7F3DAFF000EDF6E0E4A0F2A0FBE3AEFB7
:10446000A2F00F5009E1600E0E5CD8A03AEFA2F066
:104470003CEFA2F024EFA2F0000E0101526F040EF7
:10448000536F60004BF5D9FF60004FF5DAFF200E47
:10449000DF6E010E5225026E000E5321036EE30EF5
:1044A000046E010E056E000E076E090E066E53ECCB
:1044B000C4F001017405D8A460EFA2F062EFA2F08D
:1044C0006CEFA2F0010E5225086E000E5321096E0A
:1044D0000DECC8F069ECCEF052C102F053C103F00C
:1044E000D2ECC9F002C00EF003C00FF00E50000174
:1044F000FC250101526F0F500001FD210101536F96
:1045000060004BF5D9FF60004FF5DAFF200EDF6E3B
:10451000400E026E050E036ED2ECC9F002C00EF022
:1045200003C00FF0010E01015225026E000E53214F
:10453000036E400E046E050E056E0EC006F00FC031
:1045400007F053ECC4F00E50010152250C6E0F50D1
:1045500053210D6E010E0C24D96E000E0D20DA6E63
:10456000000EDF6EFCC002F0FDC003F0D2ECC9F01B
:1045700002C03AF103C03BF101017405D8A4C3EFB6
:10458000A2F0C5EFA2F0CDEFA2F0FCC008F0FDC094
:1045900009F00DECC8F069ECCEF001013BBFDAEF99
:1045A000A2F03B5109E1600E3A5DD8A0DAEFA2F02B
:1045B000DCEFA2F0E0EFA2F0000E3B6F5F0E3A6F6F
:1045C000000120EE60F0FC51D926FD51DA22000EE8
:1045D000DF6E120000019151800B9A6F915191256D
:1045E0009C6F90AFF6EFA2F0F8EFA2F0F9EFA2F017
:1045F0009C819C51D8B4FFEFA2F001EFA3F016EF1D
:10460000A3F09C29D8A407EFA3F009EFA3F011EFC2
:10461000A3F0000E8E6F000E8F6F000E906F000ED5
:10462000916F908F000E916F1EEFA3F0000E8E6FB2
:10463000000E8F6F000E906F000E916F9551800BE2
:104640009B6F9A519B19D8B428EFA3F02AEFA3F0DF
:104650002BEFA3F09A8D955195259B6F94AF33EF77
:10466000A3F035EFA3F036EFA3F09B819B51D8B4B4
:104670003CEFA3F03EEFA3F053EFA3F09B29D8A4A7
:1046800044EFA3F046EFA3F04EEFA3F0000E926FBD
:10469000000E936F000E946F000E956F948F000EB6
:1046A000956F5BEFA3F0000E926F000E936F000EFC
:1046B000946F000E956F9C519B5DD8B062EFA3F094
:1046C00064EFA3F08BEFA3F09AAD69EFA3F06BEF6B
:1046D000A3F06DEFA3F0800E9A1B9CC09DF09BC0D1
:1046E0009CF09DC09BF08EC09DF092C08EF09DC04E
:1046F00092F08FC09DF093C08FF09DC093F090C05A
:104700009DF094C090F09DC094F091C09DF095C034
:1047100091F09DC095F0000E9D6F9C519BC096F04E
:10472000976B965F000E975B97BFA0EFA3F0975132
:1047300009E11A0E965DD8A0A0EFA3F0A2EFA3F0B6
:10474000D9EFA3F08E518F1190119111D8A4ABEF36
:10475000A3F0AEEFA3F0010EAFEFA3F0000E9D6F3C
:10476000000E8E6F000E8F6F000E906F000E916F17
:104770009BC09CF0E2EFA3F09DA1C1EFA3F0C3EFBB
:10478000A3F0C9EFA3F0D8909D3101099D6FCBEF45
:10479000A3F0D8909D338EA1D0EFA3F0D2EFA3F079
:1047A000D3EFA3F09D8F9135913390338F338E33B8
:1047B0009C2B9B519C5DD8A0E0EFA3F0E2EFA3F00F
:1047C000BCEFA3F09ABDE7EFA3F0E9EFA3F029EF68
:1047D000A4F09C51D8A4EFEFA3F0F1EFA3F0FBEF0E
:1047E000A3F0000E8E6F000E8F6F000E906F000E04
:1047F000916F4AEFA5F092518E2793518F239451D8
:1048000090239551912391A108EFA4F00AEFA4F011
:10481000B6EFA4F09DA10FEFA4F011EFA4F017EFF5
:10482000A4F0D8909D3101099D6F19EFA4F0D890A4
:104830009D338EA11EEFA4F020EFA4F021EFA4F091
:104840009D8F9135913390338F338E339C2BB6EF00
:10485000A4F092518E5D93518F599451905991517A
:10486000800A966F9551800A9659D8B03AEFA4F015
:104870003CEFA4F067EFA4F08E51925D966F8F51DC
:104880009359976F90519459986F91519559996F89
:10489000FF0E96258E6FFF0E97218F6FFF0E9821CA
:1048A000906FFF0E9921916F800E9A1B9D6D9D5107
:1048B000D8A45DEFA4F05FEFA4F06FEFA4F0010EB9
:1048C0008E27000E8F23902391236FEFA4F0925137
:1048D0008E5F93518F5B9451905B9551915B8E519C
:1048E0008F1190119111D8A478EFA4F07AEFA4F071
:1048F000AFEFA4F09D51D8A480EFA4F082EFA4F014
:10490000AFEFA4F0000E8E6F000E8F6F000E906F51
:10491000000E916F4AEFA5F0D8908E378F37903701
:1049200091379DAF96EFA4F098EFA4F099EFA4F023
:104930008E819DA19EEFA4F0A0EFA4F0A4EFA4F0BF
:10494000D8809D37A6EFA4F0D8909D379C51D8B45D
:10495000ACEFA4F0AEEFA4F0AFEFA4F09C0790AFE3
:10496000B4EFA4F0B6EFA4F08CEFA4F0000E9B6FB0
:104970009DAFBDEFA4F0BFEFA4F0D7EFA4F09DC0B2
:1049800096F07F0E9617D8B4C8EFA4F0CAEFA4F043
:10499000CEEFA4F0010E9B6FD7EFA4F08EA1D3EF62
:1049A000A4F0D5EFA4F0D7EFA4F0CAEFA4F09B5188
:1049B000D8B4DDEFA4F0DFEFA4F00AEFA5F0010E0C
:1049C0008E27000E8F239023912391A1EAEFA4F06C
:1049D000ECEFA4F00AEFA5F08EC096F08FC097F030
:1049E00090C098F091C099F09935993398339733E6
:1049F000963396C08EF097C08FF098C090F099C013
:104A000091F09C29D8B407EFA5F009EFA5F00AEFC3
:104A1000A5F09C2B9C29D8B410EFA5F012EFA5F0BF
:104A20001AEFA5F09C51D8A418EFA5F01AEFA5F045
:104A30002CEFA5F0000E8E6F000E8F6F000E906FA2
:104A4000000E916F9C51D8A428EFA5F02AEFA5F095
:104A50002CEFA5F0000E9A6F9CA131EFA5F033EF7B
:104A6000A5F036EFA5F0908F37EFA5F0909FD89086
:104A70009C31916F9AAF3FEFA5F041EFA5F042EF67
:104A8000A5F0918F8EC08EF08FC08FF090C090F007
:104A900091C091F012001350800B0001816F1350F0
:104AA0001324876F12AE57EFA5F059EFA5F05AEF18
:104AB000A5F087818751D8B460EFA5F062EFA5F02B
:104AC00075EFA5F08729D8A468EFA5F06AEFA5F0E7
:104AD00072EFA5F0000E106E000E116E000E126E39
:104AE000000E136E128E7DEFA5F0000E106E000EFC
:104AF000116E000E126E000E136E1750800B811B8C
:104B000017501724826F16AE88EFA5F08AEFA5F034
:104B10008BEFA5F082818251D8B491EFA5F093EF8D
:104B2000A5F0A6EFA5F08229D8A499EFA5F09BEFF8
:104B3000A5F0A3EFA5F0000E146E000E156E000E8A
:104B4000166E000E176E168EAEEFA5F0000E146EE8
:104B5000000E156E000E166E000E176E8251D8B440
:104B6000B4EFA5F0B6EFA5F0BEEFA5F08751D8A43D
:104B7000BCEFA5F0BEEFA5F0C8EFA5F0000E106EDB
:104B8000000E116E000E126E000E136E72EFA7F083
:104B9000165010026F00CCFF8CF06F00D0FF8DF02C
:104BA0008C51836F846B856B866B8D51886F896B9D
:104BB0008A6B8B6B155011026F00CCFF8CF06F006D
:104BC000D0FF8DF08C518327000E8423852386230C
:104BD0008D518827000E89238A238B2314501202BB
:104BE0006F00CCFF8CF06F00D0FF8DF08C518327CD
:104BF000000E8423852386238D518827000E892368
:104C00008A238B2385C086F084C085F083C084F01E
:104C1000836B145011026F00CCFF8CF06F00D0FF3B
:104C20008DF08C5183278D518423000E8523000E37
:104C30008623155010026F00CCFF8CF06F00D0FF60
:104C40008DF08C5183278D518423000E8523000E17
:104C5000862385C086F084C085F083C084F0836B92
:104C6000145010026F00CCFF8CF06F00D0FF8DF05D
:104C70008C5183278D518423000E8523000E8623BB
:104C8000165011026F00CCFF8CF06F00D0FF8DF03A
:104C90008C5188278D518923000E8A23000E8B2387
:104CA000155012026F00CCFF8CF06F00D0FF8DF01A
:104CB0008C5188278D518923000E8A23000E8B2367
:104CC000165012026F00CCFF8CF06F00D0FF8DF0F9
:104CD0008C51186E8D51196E1A6A1B6A1AC01BF01E
:104CE00019C01AF018C019F0186A185088271950FE
:104CF00089231A508A231B508B2383C018F084C049
:104D000019F085C01AF086C01BF0190E8DEFA6F0C1
:104D1000D8901B321A3219321832E82E88EFA6F0DA
:104D200018508827195089231A508A231B508B2327
:104D300085C086F084C085F083C084F0836B825187
:104D400087C018F0196A1826000E1922820E18243E
:104D50008C6FFF0E19208D6FC3EFA6F0D8908837A7
:104D600089378A378B3786AFB8EFA6F0BAEFA6F04F
:104D7000BBEFA6F08881D890833784378537863794
:104D80008C07D8A08D078AAFC8EFA6F0CAEFA6F0AF
:104D9000AEEFA6F0000E826F86AFD1EFA6F0D3EF94
:104DA000A6F0F7EFA6F0FF0E8315186EFF0E841520
:104DB000196EFF0E85151A6E7F0E86151B6E185024
:104DC00019101A101B10D8B4E8EFA6F0EAEFA6F0FD
:104DD000EEEFA6F0010E826FF7EFA6F088A1F3EFD9
:104DE000A6F0F5EFA6F0F7EFA6F0EAEFA6F08251F5
:104DF000D8B4FDEFA6F0FFEFA6F023EFA7F0010E69
:104E00008827000E89238A238B238BA10AEFA7F022
:104E10000CEFA7F023EFA7F088C018F089C019F0B5
:104E20008AC01AF08BC01BF01B341B321A321932A5
:104E3000183218C088F019C089F01AC08AF01BC057
:104E40008BF08C4B8D2B8DBF2EEFA7F08D5108E191
:104E50008C29D8A02EEFA7F030EFA7F03AEFA7F0FB
:104E6000000E886F000E896F800E8A6F7F0E8B6F29
:104E700068EFA7F08DBF47EFA7F08D5106E18C05D5
:104E8000D8B045EFA7F047EFA7F053EFA7F0000E1B
:104E9000886F000E896F000E8A6F000E8B6F000EF8
:104EA000816F68EFA7F08CC087F0FF0E8817FF0EA8
:104EB00089177F0E8A17000E8B1787A162EFA7F064
:104EC00064EFA7F065EFA7F08A8FD89087318B6FDA
:104ED00081518B1388C010F089C011F08AC012F084
:104EE0008BC013F012001350800B0001856F13501C
:104EF00013248C6F12AE7FEFA7F081EFA7F082EF43
:104F0000A7F08C818C51D8B488EFA7F08AEFA7F076
:104F10009FEFA7F08C29D8A490EFA7F092EFA7F00D
:104F20009AEFA7F0000E106E000E116E000E126EBA
:104F3000000E136E128E000E136EA7EFA7F0000E78
:104F4000106E000E116E000E126E000E136E1750D2
:104F5000800B851B175017248D6F16AEB2EFA7F08C
:104F6000B4EFA7F0B5EFA7F08D818D51D8B4BBEFAA
:104F7000A7F0BDEFA7F0D2EFA7F08D29D8A4C3EF1B
:104F8000A7F0C5EFA7F0CDEFA7F0000E146E000E4E
:104F9000156E000E166E000E176E168E000E176E32
:104FA000DAEFA7F0000E146E000E156E000E166EEE
:104FB000000E176E1450151016101710D8A4E3EF3A
:104FC000A7F0E5EFA7F0FDEFA7F0000E106E000EC2
:104FD000116E000E126E000E136E800E12127F0EF6
:104FE00013128551131210C010F011C011F012C02D
:104FF00012F013C013F040EFA9F08C51D8A403EFC6
:10500000A8F005EFA8F00FEFA8F0000E106E000E4C
:10501000116E000E126E000E136E40EFA9F08D514E
:105020008CC018F0196A185E000E195A7F0E1824E9
:10503000866F000E1920876F10C081F011C082F0BA
:1050400012C083F013C084F0000E106E000E116EBB
:10505000000E126E000E136E000E886F000E896F28
:10506000000E8A6F000E8B6F000E8D6F70EFA8F030
:105070008D51D8B43EEFA8F040EFA8F057EFA8F05C
:10508000D8908137823783378437D89010361136DD
:10509000123613368BAF4FEFA8F051EFA8F052EF56
:1050A000A8F01080D890883789378A378B3714500A
:1050B000815D155082591650835917508459D8A0D4
:1050C00064EFA8F066EFA8F06FEFA8F08B8D145096
:1050D000815F1550825B1650835B1750845B8D2B6C
:1050E000190E8D6576EFA8F078EFA8F038EFA8F0EC
:1050F0008151821183118411D8B481EFA8F083EF1C
:10510000A8F09BEFA8F088819BEFA8F0D89010360C
:105110001136123613368BAF90EFA8F092EFA8F04D
:1051200093EFA8F01080D890883789378A378B376B
:105130008607D8A0870712AEA0EFA8F0A2EFA8F0CC
:1051400086EFA8F0000E8D6F8BAFA9EFA8F0ABEF44
:10515000A8F0CFEFA8F0FF0E8815186EFF0E891586
:10516000196EFF0E8A151A6E7F0E8B151B6E185066
:1051700019101A101B10D8B4C0EFA8F0C2EFA8F095
:10518000C6EFA8F0010E8D6FCFEFA8F010A0CBEF07
:10519000A8F0CDEFA8F0CFEFA8F0C2EFA8F08D51A6
:1051A000D8B4D5EFA8F0D7EFA8F0FBEFA8F0010E28
:1051B0001026000E11221222132213A0E2EFA8F0F3
:1051C000E4EFA8F0FBEFA8F010C018F011C019F040
:1051D00012C01AF013C01BF01B341B321A321932E2
:1051E000183218C010F019C011F01AC012F01BC00C
:1051F00013F0864B872B87BF06EFA9F0875108E194
:105200008629D8A006EFA9F008EFA9F013EFA9F0BE
:10521000000E876F8669000E106E000E116E000E74
:10522000126E000E136E87BF20EFA9F0875106E1C2
:105230008605D8B01EEFA9F020EFA9F02EEFA9F057
:10524000000E876F000E866F000E106E000E116E3E
:10525000000E126E000E136E000E856F86C08CF06D
:105260008CA135EFA9F037EFA9F03AEFA9F0128E33
:105270003BEFA9F0129ED8908C31136EF1EFA7F09E
:10528000120083C09BF084C09CF085C09DF086C056
:105290009EF087C09FF088C0A0F089C0A1F08AC0AE
:1052A000A2F00001A2BF57EFA9F05AEFA9F0010E3A
:1052B0005BEFA9F0000E996F9A6B99519A11D8B4CF
:1052C00064EFA9F066EFA9F076EFA9F0A21FA11F85
:1052D000A01F9F1F9E1F9D1F9C1F9B6D000E9C2348
:1052E0009D239E239F23A023A123A223010133BF3B
:1052F0007CEFA9F07EEFA9F07FEFA9F0349333BFE4
:105300008CEFA9F0335106E13205D8B08AEFA9F04D
:105310008CEFA9F093EFA9F0000E0001966F010E3B
:10532000956F97EFA9F032C195F033C196F030C177
:1053300097F031C198F0000199519A11D8A4A3EFC8
:10534000A9F0A5EFA9F0ADEFA9F0010134A5ABEFED
:10535000A9F0ADEFA9F0B1EFA9F000019707D8A02F
:105360009807000E0001A46F4F0EA36F000E0301FB
:10537000CF6F39EFAAF00001A307D8A0A407800ED1
:10538000A325D96E030EA421DA6E9BC002F09CC047
:1053900003F09DC004F09EC005F09FC006F0A0C0C1
:1053A00007F0A1C008F0A2C009F00A0E0A6E000EB4
:1053B0000B6E000E0C6E000E0D6E000E0E6E000ECB
:1053C0000F6E000E106E000E116EB2ECB6F002C041
:1053D0008BF003C08CF004C08DF005C08EF006C0C9
:1053E0008FF007C090F008C091F009C092F08BC018
:1053F00014F08DC015F06AECCCF01450300FDF6E55
:1054000000019507D8A096079707D8A098079BC0DA
:1054100002F09CC003F09DC004F09EC005F09FC048
:1054200006F0A0C007F0A1C008F0A2C009F00A0E63
:105430000A6E000E0B6E000E0C6E000E0D6E000E4E
:105440000E6E000E0F6E000E106E000E116E2EEC22
:10545000B5F002C09BF003C09CF004C09DF005C0F5
:105460009EF006C09FF007C0A0F008C0A1F009C0E0
:10547000A2F00001A4BF45EFAAF0A45108E1A305E2
:10548000D8A045EFAAF047EFAAF078EFAAF09B5119
:105490009C119D119E119F11A011A111A211D8A4C0
:1054A00054EFAAF056EFAAF0BBEFA9F096BF63EF56
:1054B000AAF0965106E19505D8B061EFAAF063EF26
:1054C000AAF0BBEFA9F098BF6EEFAAF0985108E1DF
:1054D0009705D8A06EEFAAF070EFAAF078EFAAF0C7
:1054E000010134B376EFAAF078EFAAF0BBEFA9F090
:1054F000000199519A11D8A480EFAAF082EFAAF086
:105500008AEFAAF0010134A588EFAAF08AEFAAF089
:10551000AAEFAAF00001A307D8A0A40799519A11F5
:10552000D8A495EFAAF097EFAAF09DEFAAF0000E8D
:10553000946F2B0E936FA1EFAAF0000E946F2D0EB7
:10554000936F800EA325D96E030EA421DA6E60003E
:105550004FF2DFFF81C012F082C013F0800E000115
:10556000A325146E030EA421156E97C016F098C0E3
:1055700017F053ECC1F012C081F013C082F012009A
:10558000010133BFC6EFAAF0C8EFAAF0C9EFAAF035
:10559000349333BFD6EFAAF0335106E13205D8B0C9
:1055A000D4EFAAF0D6EFAAF0DDEFAAF0000E0001CA
:1055B000956F010E946FE1EFAAF032C194F033C100
:1055C00095F030C196F031C197F0010134A9EBEFAD
:1055D000AAF0EDEFAAF0F2EFAAF00001FE0E962776
:1055E000FF0E972383C098F084C099F085C09AF08D
:1055F00086C09BF087C09CF088C09DF089C09EF05B
:105600008AC09FF0000E0001A16F4F0EA06F000E28
:105610000301CF6FA8EFABF00001A007D8A0A1074E
:105620000F0E9815A26FA36BA3BF20EFABF0A35191
:1056300009E10A0EA25DD8A020EFABF022EFABF09B
:105640002AEFABF0570EA225A26F000EA321A36F85
:1056500030EFABF0300EA225A26F000EA321A36F96
:10566000BF0E8C6FFF0E8D6F8B518E6F8F6B8C51B9
:105670008E278D518F238F5107E11A0E8E5DD8B082
:1056800044EFABF046EFABF069EFABF09F0E8C6FE1
:10569000FF0E8D6F200EA2118E6F000EA3118F6F63
:1056A0008C518E278D518F238F5107E11A0E8E5DFD
:1056B000D8B05DEFABF05FEFABF069EFABF0A2C03D
:1056C00008F0A3C009F026ECCCF008C0A2F009C095
:1056D000A3F0800E0001A025D96E030EA121DA6E81
:1056E00060008BF2DFFF9407D8A095079607D8A03B
:1056F000970798C08CF099C08DF09AC08EF09BC02F
:105700008FF09CC090F09DC091F09EC092F09FC021
:1057100093F0050E95EFABF0D8909333923391331D
:1057200090338F338E338D338C33E82E8CEFABF088
:105730008CC098F08DC099F08EC09AF08FC09BF00D
:1057400090C09CF091C09DF092C09EF093C09FF0DD
:105750000001A1BFB5EFABF0A15109E1020EA05DC0
:10576000D8A0B5EFABF0B7EFABF0E8EFABF09851E6
:1057700099119A119B119C119D119E119F11D8A4F2
:10578000C4EFABF0C6EFABF00CEFABF095BFD3EFCF
:10579000ABF0955106E19405D8B0D1EFABF0D3EF63
:1057A000ABF00CEFABF097BFDEEFABF0975108E139
:1057B0009605D8A0DEEFABF0E0EFABF0E8EFABF092
:1057C000010134B3E6EFABF0E8EFABF00CEFABF078
:1057D000010134A9EEEFABF0F0EFABF008EFACF065
:1057E0000001A007D8A0A107800EA025D96E030E46
:1057F000A121DA6E60002FF2DFFFA007D8A0A10779
:10580000800EA025D96E030EA121DA6E300EDF6E58
:1058100081C012F082C013F0800E0001A025146E2A
:10582000030EA121156E96C016F097C017F053EC29
:10583000C1F012C081F013C082F01200000E00010E
:10584000FC6F040EFD6F3D017599738F000E010111
:10585000DC6F020EDB6FDBC102F0DCC103F0AAECEF
:10586000CDF00009D8B437EFACF039EFACF028EF49
:10587000ADF00101DC35DC310001F66F0101DB31F7
:10588000646FF6C065F1FCC0B0F1FDC0B1F1370E38
:10589000B26FFA0EB36FDBC1B4F1DCC1B5F164C114
:1058A000B6F165C1B7F153ECCAF0D1EFACF0FCC072
:1058B00010F0FDC011F0700E126EFD0E136ED4ECE0
:1058C000CEF020EFADF0000E026E030E036E910ECF
:1058D000046EFE0E056E62ECC7F0FCC002F0FDC067
:1058E00003F0D2ECC9F002C0D9F103C0DAF1010132
:1058F000D9510001FC25066E0101DA510001FD219C
:10590000076E000E086E030E096E7CECC8F020EFE7
:10591000ADF0FCC010F0FDC011F05D0E126EFE0E79
:10592000136ED4ECCEF020EFADF0FCC010F0FDC053
:1059300011F0370E126EFE0E136ED4ECCEF020EF87
:10594000ADF0FCC010F0FDC011F00C0E126EFF0E99
:10595000136ED4ECCEF020EFADF0FCC010F0FDC023
:1059600011F0C30E126EFE0E136ED4ECCEF020EFCB
:10597000ADF0FCC010F0FDC011F06B0E126EFF0E0A
:10598000136ED4ECCEF020EFADF0FCC010F0FDC0F3
:1059900011F0190E126EFF0E136ED4ECCEF020EF44
:1059A000ADF064C1F6F065C1F7F00001F751000AEF
:1059B000D8B4DDEFACF0C5EFACF0F651200AD8B4A6
:1059C00057EFACF0010AD8B457EFACF0030AD8B4E3
:1059D00057EFACF0010AD8B457EFACF0040AD8B4D2
:1059E00057EFACF00F0AD8B463EFACF0010AD8B4AB
:1059F00063EFACF0030AD8B463EFACF01D0AD8B47F
:105A000089EFACF00F0AD8B495EFACF0010AD8B426
:105A100095EFACF0030AD8B495EFACF0010AD8B416
:105A200095EFACF0070AD8B4A1EFACF06B0AD8B48C
:105A3000ADEFACF03F0AD8B4B9EFACF0C5EFACF0C5
:105A4000FCC008F0FDC009F00DECC8F069ECCEF028
:105A5000020E0101DB25DB6F000EDC21DC6FDCBFF9
:105A60003BEFADF0DC5109E1FC0EDB5DD8A03BEF74
:105A7000ADF03DEFADF02BEFACF03D01739F7589BC
:105A800069ECCEF01200200E0001F86F000EF96FE5
:105A9000000EFC6F040EFD6F69ECCEF0000E0F6E71
:105AA000000E0E6E0E500001F825D96E0F50F92130
:105AB000DA6EDF50ECECC0F002C008F003C009F071
:105AC0000DECC8F00E500001F8250C6E0F50F921B6
:105AD0000D6E080E0C24D96E000E0D20DA6EDF500C
:105AE000ECECC0F002C008F003C009F00DECC8F007
:105AF0000E500001F8250C6E0F50F9210D6E100E9E
:105B00000C24D96E000E0D20DA6EDF50ECECC0F0E4
:105B100002C008F003C009F00DECC8F00E500001FF
:105B2000F8250C6E0F50F9210D6E180E0C24D96E4D
:105B3000000E0D20DA6EDF50ECECC0F002C008F071
:105B400003C009F00DECC8F00E500001F8250C6EF2
:105B50000F50F9210D6E200E0C24D96E000E0D2071
:105B6000DA6EDF50ECECC0F002C008F003C009F0C0
:105B70000DECC8F00E500001F8250C6E0F50F92105
:105B80000D6E280E0C24D96E000E0D20DA6EDF503B
:105B9000ECECC0F002C008F003C009F00DECC8F056
:105BA0000E500001F8250C6E0F50F9210D6E300ECD
:105BB0000C24D96E000E0D20DA6EDF50ECECC0F034
:105BC00002C008F003C009F00DECC8F00E5000014F
:105BD000F8250C6E0F50F9210D6E380E0C24D96E7D
:105BE000000E0D20DA6EDF50ECECC0F002C008F0C1
:105BF00003C009F00DECC8F00E500001F8250C6E42
:105C00000F50F9210D6E400E0C24D96E000E0D20A0
:105C1000DA6EDF50ECECC0F002C008F003C009F00F
:105C20000DECC8F00E500001F8250C6E0F50F92154
:105C30000D6E480E0C24D96E000E0D20DA6EDF506A
:105C4000ECECC0F002C008F003C009F00DECC8F0A5
:105C50000E500001F8250C6E0F50F9210D6E500EFC
:105C60000C24D96E000E0D20DA6EDF50ECECC0F083
:105C700002C008F003C009F00DECC8F00E5000019E
:105C8000F8250C6E0F50F9210D6E580E0C24D96EAC
:105C9000000E0D20DA6EDF50ECECC0F002C008F010
:105CA00003C009F00DECC8F069ECCEF00E4A0F2AE3
:105CB0000FBE64EFAEF00F5009E1080E0E5CD8A0E5
:105CC00064EFAEF066EFAEF052EFADF0120039C205
:105CD0009EF03AC29FF03BC2A0F03CC2A1F08EC041
:105CE0009EF08FC09FF090C0A0F091C0A1F0810EF7
:105CF0000001926FFF0E936F9EC094F09FC095F0CD
:105D0000A0C096F0A1C097F0180E8CEFAEF0D8901E
:105D10009733963395339433E82E87EFAEF0945152
:105D200092259C6F000E93219D6F9DBFA1EFAEF059
:105D30009D5109E1170E9C5DD8A0A1EFAEF0A3EF35
:105D4000AEF0ADEFAEF08EC08EF08FC08FF090C091
:105D500090F091C091F071EFAFF09DBFB2EFAEF057
:105D6000B4EFAEF025EFAFF09CC092F0FF0E936F52
:105D7000FF0E946F7F0E956F000E966F9267C3EFC4
:105D8000AEF0CBEFAEF09635963395339433933334
:105D9000922FBEEFAEF093C098F094C099F095C0EA
:105DA0009AF096C09BF0000198519E15926F995100
:105DB0009F15936F9A51A015946F9B51A115956FE4
:105DC0009251931194119511D8A4E9EFAEF0EBEF35
:105DD000AEF0EDEFAEF0A3EFAEF09EC092F09FC03C
:105DE00093F0A0C094F0A1C095F0200EFDEFAEF0AE
:105DF000D8909533943393339233E82EF8EFAEF086
:105E00009251931194119511D8B409EFAFF00BEFA3
:105E1000AFF013EFAFF098519E2799519F239A51FD
:105E2000A0239B51A123981D926F991D936F9A1DDA
:105E3000946F9B1D956F92519E1793519F1794518C
:105E4000A0179551A11769EFAFF09EC092F09FC0C7
:105E500093F0A0C094F0A1C095F0200E35EFAFF004
:105E6000D8909533943393339233E82E30EFAFF0DC
:105E70009251931194119511D8A441EFAFF043EFD3
:105E8000AFF04DEFAFF0000E9E6F000E9F6F000E53
:105E9000A06F000EA16F69EFAFF0D8909E35926FA2
:105EA0009F35936FA035946FA135956F92519311E3
:105EB00094119511D8B45FEFAFF061EFAFF069EFD7
:105EC000AFF0000E9E6F000E9F6F800EA06FBF0E92
:105ED000A16F9EC08EF09FC08FF0A0C090F0A1C0B7
:105EE00091F01200200E086E000E096E000E0F6E6B
:105EF000000E0E6E0E500224D96E0F500320DA6E83
:105F0000DF500A6E55EFB0F0000E116E000E106EED
:105F1000C80E1024D96E020E1120DA6EDF500D6EFD
:105F20000EC004F00FC005F0D89004360536D890A6
:105F300004360536D89004360536105004240B6E0E
:105F4000115005200C6E0B500824D96E0C500920FE
:105F5000DA6E600037F0DFFF104A112A11BEBAEF87
:105F6000AFF0115009E1080E105CD8A0BAEFAFF005
:105F7000BCEFAFF088EFAFF06AEFB0F0000E116E3B
:105F8000000E106EC00E1024D96E020E1120DA6EB3
:105F9000DF500D6E0EC004F00FC005F0D89004362F
:105FA0000536D89004360536D8900436053610509C
:105FB00004240B6E115005200C6E0B500824D96E72
:105FC0000C500920DA6E600037F0DFFF104A112A0A
:105FD00011BEF4EFAFF0115009E1080E105CD8A02B
:105FE000F4EFAFF0F6EFAFF0C2EFAFF06AEFB0F062
:105FF0003B0E0A18D8A4FFEFAFF001EFB0F003EFAB
:10600000B0F0200E0A6E0A50080D6F00CCFF06F0AB
:106010006F00D0FF07F0000E116E000E106E8F0E95
:10602000046EE60E056E0650042607500522105039
:10603000042611500522600013F0F6FF600017F0EF
:10604000F7FF000EF86E08006F00D4FF0DF00EC0D1
:1060500004F00FC005F0D89004360536D890043609
:106060000536D89004360536105004240B6E1150B6
:1060700005200C6E0B500824D96E0C500920DA6EE6
:10608000600037F0DFFF104A112A11BE51EFB0F067
:10609000115009E1080E105CD8A051EFB0F053EF99
:1060A000B0F00FEFB0F06AEFB0F00A50046E056A7E
:1060B0000550000AD8B45FEFB0F0F8EFAFF004502D
:1060C000B00AD8B484EFAFF0010AD8B4BEEFAFF095
:1060D000F8EFAFF00E4A0F2A0FBE78EFB0F00F5076
:1060E00009E10C0E0E5CD8A078EFB0F07AEFB0F0BA
:1060F0007AEFAFF01200010133BF81EFB0F083EF10
:10610000B0F084EFB0F0349333BF91EFB0F033517F
:1061100006E13205D8B08FEFB0F091EFB0F098EF14
:10612000B0F0000E0001946F010E936F9CEFB0F081
:1061300032C193F033C194F030C195F031C196F083
:1061400083C097F084C098F085C099F086C09AF01B
:1061500087C09BF088C09CF089C09DF08AC09EF0EB
:10616000000E0001A06F4F0E9F6F000E0301CF6F56
:1061700032EFB1F000019F07D8A0A007800E9F2545
:10618000D96E030EA021DA6E97C002F098C003F01A
:1061900099C004F09AC005F09BC006F09CC007F0BF
:1061A0009DC008F09EC009F00A0E0A6E000E0B6E2C
:1061B000000E0C6E000E0D6E000E0E6E000E0F6EB9
:1061C000000E106E000E116E84ECC0F002C08BF059
:1061D00003C08CF004C08DF005C08EF006C08FF0B7
:1061E00007C090F008C091F009C092F000018B51F7
:1061F000300FDF6E9307D8A094079507D8A09607B5
:1062000097C002F098C003F099C004F09AC005F05E
:106210009BC006F09CC007F09DC008F09EC009F02E
:106220000A0E0A6E000E0B6E000E0C6E000E0D6E46
:10623000000E0E6E000E0F6E000E106E000E116E30
:1062400008ECBDF002C097F003C098F004C099F0CC
:1062500005C09AF006C09BF007C09CF008C09DF0F6
:1062600009C09EF000019F51A011D8B43AEFB1F0DF
:106270003CEFB1F06DEFB1F09751981199119A116F
:106280009B119C119D119E11D8A449EFB1F04BEFC9
:10629000B1F0BAEFB0F094BF58EFB1F0945106E10D
:1062A0009305D8B056EFB1F058EFB1F0BAEFB0F0B7
:1062B00096BF63EFB1F0965108E19505D8A063EF62
:1062C000B1F065EFB1F06DEFB1F0010134B36BEFF8
:1062D000B1F06DEFB1F0BAEFB0F081C012F082C052
:1062E00013F0800E00019F25146E030EA021156E81
:1062F00095C016F096C017F053ECC1F012C081F0B3
:1063000013C082F01200000E0001826F020E816F36
:10631000000E846F000E836F800E01015825D96E28
:10632000040E5921DA6E000EDF6E595107E1160E88
:10633000585DD8B09EEFB1F0A0EFB1F073EFB2F0BE
:10634000595109E1130E585DD8A0A9EFB1F0ABEF98
:10635000B1F073EFB2F0000E0001866F020E856F90
:10636000E5EFB1F0800E8525D96E040E8621DA6E38
:106370003B0EDE18D8A4BFEFB1F0C1EFB1F0E3EFF0
:10638000B1F0800E8525D96E040E8621DA6E000EDE
:10639000DF6E800E8125026E040E8221036E6EEC8C
:1063A000BAF0000E00018325D96E020E8421DA6E48
:1063B00060000BF0DFFF834B842B010E8525816F7E
:1063C000000E8621826F854B862B010158510001FA
:1063D000855D0101595100018659D8A0F2EFB1F055
:1063E000F4EFB1F0B2EFB1F0800E8125026E040E31
:1063F0008221036E6EECBAF0000E00018325D96E87
:10640000020E8421DA6E60000BF0DFFF00C284F11F
:10641000020101511F0B0101836F02C282F103C20D
:1064200086F104C287F102010551070B0101856F56
:106430008351CCECCFF00101816F0C0E816523EF0D
:10644000B2F025EFB2F027EFB2F0000E816F070E29
:1064500085652DEFB2F02FEFB2F037EFB2F0000EFE
:10646000856F400E026EFC0E036EFEECC9F0000E4E
:1064700001018A6F000E886F88C18BF187518EEC05
:10648000CDF001018C6F86518EECCDF001018D6F46
:1064900085C18EF184518EECCDF001018F6F835157
:1064A0008EECCDF00101906F82518EECCDF00101A8
:1064B000916F000E926F8A0E0001FA6F010EFB6F52
:1064C000FAC017F0FBC018F0000E1A6E080E196E15
:1064D000680E18ECC9F08A0E026EFD0E036EFEEC1B
:1064E000C9F07FEFB2F0730E026EF90E036EFEEC90
:1064F000C9F0D80E026EF70E036EFEECC9F0120062
:10650000000E126E000E116E000E106E000E0F6E59
:106510008CEFB2F0094A0A2A600027F0F6FF60000B
:106520002BF0F7FF000EF86E1F0EF76403D0080083
:10653000F55007D06F00DBFFE9FF6F00DFFFEAFFD8
:10654000EF50200AD8B4A7EFB2F0A9EFB2F08AEF6B
:10655000B2F0F70E0B6EFF0E0C6E600027F0F6FF28
:1065600060002BF0F7FF000EF86E1F0EF76403D0EB
:106570000800F55007D06F00DBFFE9FF6F00DFFF79
:10658000EAFFEF500D6E0E6A0B500D260C500E22D6
:106590000E5009E1050E0D5CD8A0D1EFB2F0D3EF9B
:1065A000B2F08AEFB2F0DDEFB2F0000E106E010E25
:1065B0000F6E094A0A2A32EFB3F0600027F0F6FFA7
:1065C00060002BF0F7FF000EF86E1F0EF76403D08B
:1065D0000800F55007D06F00DBFFE9FF6F00DFFF19
:1065E000EAFFEF500B6E0C6A0C50000AD8B4FBEFB8
:1065F000B2F032EFB3F00B502B0AD8B4D9EFB2F0AF
:10660000060AD8B4D5EFB2F032EFB3F011C002F001
:1066100012C003F0000E056E0A0E046EABECCEF055
:10662000600027F0F6FF60002BF0F7FF000EF86E19
:106630001F0EF76403D00800F55007D06F00DBFF92
:10664000E9FF6F00DFFFEAFFEF500B6E0B50025EB9
:10665000000E035A300E0224116E000E0320126E3B
:10666000D9EFB2F0D00E0B6EFF0E0C6E600027F06B
:10667000F6FF60002BF0F7FF000EF86E1F0EF764B8
:1066800003D00800F55007D06F00DBFFE9FF6F0073
:10669000DFFFEAFFEF500D6E0E6A0B500D260C5017
:1066A0000E220E5009E10A0E0D5CD8A05AEFB3F08D
:1066B0005CEFB3F006EFB3F00F501010D8A463EF07
:1066C000B3F065EFB3F073EFB3F011C00BF012C08D
:1066D0000CF00B1E0C1E0B4A0C2A0BC009F00CC050
:1066E0000AF077EFB3F011C009F012C00AF01200FF
:1066F00020EED0F210EE81F0060E6F006FFFE3FF88
:10670000E806FBE20DC08CF00EC08DF000018C514C
:106710008D11D8A48EEFB3F090EFB3F094EFB3F0F7
:10672000810E8C6F000E8D6F8CC002F08DC003F057
:10673000D2ECC9F002C090F003C091F032C18EF0EB
:1067400033C18FF000018FBFA8EFB3F0AAEFB3F011
:10675000BFEFB3F090518E5D8F51800A0F6E915153
:10676000800A0F58D8A0B7EFB3F0B9EFB3F0BBEF82
:10677000B3F0BFEFB3F08EC090F08FC091F090C037
:106780008EF091C08FF030C18AF031C18BF00101E1
:1067900034B1CDEFB3F0CFEFB3F0EEEFB3F0DEEF07
:1067A000B3F0000E036E200E026E0BC004F00CC09E
:1067B00005F0D9ECBEF00001904B912B00018A51FD
:1067C000905D9151800A0F6E8B51800A0F58D8A0AE
:1067D000ECEFB3F0EEEFB3F0D1EFB3F0000E000149
:1067E000896F000E886F19EFB4F0600033F2F6FF86
:1067F000600037F2F7FF000EF86E1F0EF76403D04B
:106800000800F55007D06F00DBFFE9FF6F00DFFFE6
:10681000EAFFEF500F6E0F50026E036A0BC004F0D8
:106820000CC005F0D9ECBEF000018C4B8D2B884BD1
:10683000892B8E51885D8951800A0F6E8F51800A95
:106840000F58D8A026EFB4F028EFB4F0F5EFB3F06E
:10685000010134A12EEFB4F030EFB4F04FEFB4F0FB
:106860003FEFB4F0000E036E200E026E0BC004F07A
:106870000CC005F0D9ECBEF00001904B912B00014B
:106880008A51905D9151800A0F6E8B51800A0F588A
:10689000D8A04DEFB4F04FEFB4F032EFB4F090C0A9
:1068A0000BF091C00CF012000A6E0A50D8B45BEFE6
:1068B000B4F05DEFB4F07FEFB4F005BE64EFB4F078
:1068C00062EFB4F07FEFB4F002C006F003C007F04F
:1068D00004C008F005C009F0061E071E081E091EA8
:1068E000062A000E07220822092206C00CF007C063
:1068F0000DF008C00EF009C00FF087EFB4F002C031
:106900000CF003C00DF004C00EF005C00FF00250F3
:10691000031004100510D8A490EFB4F092EFB4F077
:106920009CEFB4F0000E026E000E036E000E046EBB
:10693000000E056E2DEFB5F0960E0B6EA6EFB4F0BF
:106940000B2AD8900F320E320D320C32000E0C147E
:10695000066E000E0D14076E000E0E14086EFE0E6D
:106960000F14096E0650071008100910D8A4BBEFC9
:10697000B4F0BDEFB4F0A0EFB4F0CBEFB4F00B2A5D
:10698000010E0C26000E0D220E220F22D8900F327F
:106990000E320D320C32000E0C14066E000E0D1469
:1069A000076E000E0E14086EFF0E0F14096E0650CF
:1069B000071008100910D8A4E0EFB4F0E2EFB4F02B
:1069C000BFEFB4F0EAEFB4F00B06D8900C360D36FA
:1069D0000E360F360EBEEFEFB4F0F1EFB4F0F9EF74
:1069E000B4F0020E0B60F7EFB4F0F9EFB4F0E4EF9F
:1069F000B4F00BB0FEEFB4F000EFB5F001EFB5F07E
:106A00000E9ED8900B320BC006F0076A086A096A1E
:106A100006C009F0086A076A066A06500C12075099
:106A20000D1208500E1209500F120A50D8B41BEF65
:106A3000B5F01DEFB5F025EFB5F005BE24EFB5F0CC
:106A400022EFB5F025EFB5F00F8E0CC002F00DC0AF
:106A500003F00EC004F00FC005F01200000E136E1C
:106A600011BE37EFB5F035EFB5F049EFB5F0111EB7
:106A7000101E0F1E0E1E0D1E0C1E0B1E0A6C000E8D
:106A80000B220C220D220E220F2210221122010EA7
:106A9000136E09BE50EFB5F04EEFB5F062EFB5F0F2
:106AA000091E081E071E061E051E041E031E026C7C
:106AB000000E0322042205220622072208220922B0
:106AC000010E131A20EE14F0070EDE6AE806FDE24E
:106AD0000A500B100C100D100E100F10101011108A
:106AE000D8B475EFB5F077EFB5F0C9EFB5F0010E9A
:106AF000126E85EFB5F0D8900A360B360C360D368F
:106B00000E360F3610361136122A11AE8AEFB5F056
:106B10008CEFB5F07BEFB5F0D890143615361636FD
:106B20001736183619361A361B360A50025C0B50C7
:106B300003580C5004580D5005580E5006580F506D
:106B400007581050085811500958D8A0AAEFB5F0AE
:106B5000ACEFB5F0BDEFB5F00A50025E0B50035A32
:106B60000C50045A0D50055A0E50065A0F50075A31
:106B70001050085A1150095A1480D890113210320E
:106B80000F320E320D320C320B320A32122E8CEFD3
:106B9000B5F01350D8B4CFEFB5F0D1EFB5F0E1EFC9
:106BA000B5F01B1E1A1E191E181E171E161E151EC6
:106BB000146C000E152216221722182219221A22EE
:106BC0001B2214C002F015C003F016C004F017C059
:106BD00005F018C006F019C007F01AC008F01BC075
:106BE00009F01200200E0001F86F000EF96F000E80
:106BF000146E000E136E13500001F825816F1450AF
:106C0000F921826F580E8125D96E000E8221DA6E2D
:106C1000DF50066E1350F825836F1450F921846FEE
:106C2000500E8325D96E000E8421DA6EDF50076E78
:106C30001350F825856F1450F921866F480E85256D
:106C4000D96E000E8621DA6EDF50086E1350F825DB
:106C5000876F1450F921886F400E8725D96E000E7A
:106C60008821DA6EDF50096E1350F825896F1450B1
:106C7000F9218A6F380E8925D96E000E8A21DA6EC5
:106C8000DF500A6E1350F8258B6F1450F9218C6F6A
:106C9000300E8B25D96E000E8C21DA6EDF500B6E14
:106CA0001350F8258D6F1450F9218E6F280E8D2505
:106CB000D96E000E8E21DA6EDF500C6E1350F8255F
:106CC0008F6F1450F921906F200E8F25D96E000E12
:106CD0009021DA6EDF500D6E1350F825916F14502D
:106CE000F921926F180E9125D96E000E9221DA6E5D
:106CF000DF500E6E1350F825936F1450F921946FE6
:106D0000100E9325D96E000E9421DA6EDF500F6EAF
:106D10001350F825956F1450F921966F080E95259C
:106D2000D96E000E9621DA6EDF50106E1350F825E2
:106D3000D96E1450F921DA6EDF50116E132845EC2C
:106D4000BFF0134A142A14BEAFEFB6F0145009E195
:106D5000080E135CD8A0AFEFB6F0B1EFB6F0FBEFC2
:106D6000B5F01200000E136E09BEBBEFB6F0B9EF1E
:106D7000B6F0CDEFB6F0091E081E071E061E051E52
:106D8000041E031E026C000E0322042205220622AA
:106D9000072208220922010E136E11BED4EFB6F0AD
:106DA000D2EFB6F0E4EFB6F0111E101E0F1E0E1E4D
:106DB0000D1E0C1E0B1E0A6C000E0B220C220D2247
:106DC0000E220F22102211220A500B100C100D104F
:106DD0000E100F1010101110D8B4F1EFB6F0F3EF41
:106DE000B6F03BEFB7F0010E126E01EFB7F0D8909E
:106DF0000A360B360C360D360E360F361036113677
:106E0000122A11AE06EFB7F008EFB7F0F7EFB6F0C1
:106E10000A50025C0B5003580C5004580D50055892
:106E20000E5006580F500758105008581150095866
:106E3000D8A01DEFB7F01FEFB7F02FEFB7F00A5053
:106E4000025E0B50035A0C50045A0D50055A0E5056
:106E5000065A0F50075A1050085A1150095AD89024
:106E6000113210320F320E320D320C320B320A3226
:106E7000122E08EFB7F01350D8B441EFB7F043EF3C
:106E8000B7F053EFB7F0091E081E071E061E051EB9
:106E9000041E031E026C000E032204220522062299
:106EA00007220822092202C002F003C003F004C036
:106EB00004F005C005F006C006F007C007F008C0E2
:106EC00008F009C009F0120002C009F003C00AF07E
:106ED00004C00BF005C00CF00606D8A00706062873
:106EE00006E10728D8A477EFB7F079EFB7F086EF7F
:106EF000B7F0000E036E000E026E0CEFB8F0094AF8
:106F00000A2A0B4A0C2A0606D8A00706600027F0BA
:106F1000F6FF60002BF0F7FF000EF86E1F0EF7640F
:106F200003D00800F55007D06F00DBFFE9FF6F00CA
:106F3000DFFFEAFFEF500009D8B4A1EFB7F0A3EFED
:106F4000B7F0E7EFB7F060002FF0F6FF600033F026
:106F5000F7FF000EF86E0800F5500009D8B4B3EF43
:106F6000B7F0B5EFB7F0E7EFB7F006500710D8B4B9
:106F7000BCEFB7F0BEEFB7F0E7EFB7F060002FF06F
:106F8000F6FF600033F0F7FF000EF86E08006F00A8
:106F9000D4FF08F0600027F0F6FF60002BF0F7FF49
:106FA000000EF86E1F0EF76403D00800F55007D0EE
:106FB0006F00DBFFE9FF6F00DFFFEAFFEF5008180B
:106FC000D8B4E5EFB7F0E7EFB7F07FEFB7F06000C8
:106FD00027F0F6FF60002BF0F7FF000EF86E1F0E93
:106FE000F76403D00800F55007D06F00DBFFE9FF1E
:106FF0006F00DFFFEAFFEF50086E60002FF0F6FF32
:10700000600033F0F7FF000EF86E0800F550085CE2
:10701000026E036AD8A003061200B8ECC3F0000E9B
:107020000101E36FE40E026E020E036E8451E4EC84
:10703000CCF02F0E0201E66FE70E026E020E036E19
:1070400001018351E4ECCCF02F0E0201E96FEA0E4E
:10705000026E020E036E01018251E4ECCCF0000ED0
:107060000201EC6F01018551020DA70EF324D96EC8
:10707000020EF420DA6E6F0078FF02F06F0074FFEA
:1070800003F0FEECC9F0200E1BECCFF0000E026EF8
:10709000030E036E01018451E4ECCCF0000E086E87
:1070A000030E096E0DECC8F0200E1BECCFF00101B1
:1070B0008351CCECCFF00101816F8151020DD00ED4
:1070C000F324D96E030EF420DA6E6F0078FF02F01D
:1070D0006F0074FF03F0FEECC9F0200E1BECCFF044
:1070E000000E026E030E036E01018251E4ECCCF03F
:1070F000000E086E030E096E0DECC8F0200E1BEC9E
:10710000CFF0E30E026E010E036E01018651E4EC36
:10711000CCF03A0E0101E56FE60E026E010E036E31
:107120008751E4ECCCF03A0E0101E86FE90E026EF3
:10713000010E036E8851E4ECCCF0000E0101EB6F00
:10714000E30E086E010E096E0DECC8F069ECCEF08E
:107150001200090E146E1E0E136EE40EE82EFED7FA
:10716000132EFCD7142EFAD700D0BC80000E066E6A
:10717000000E076E000E086E000E096E000E0A6EFD
:10718000000E0B6E000E0C6E000E0D6E000E0E6EDD
:10719000000E0F6E000E106E000E116E0F0E45ECFD
:1071A000BFF0070E066E070E076E070E086E070E7D
:1071B000096E070E0A6E070E0B6E070E0C6E070E99
:1071C0000D6E070E0E6E070E0F6E070E106E070E79
:1071D000116E0B0E45ECBFF0000E066E000E076E32
:1071E000000E086E000E096E000E0A6E000E0B6E89
:1071F000000E0C6E000E0D6E000E0E6E000E0F6E69
:10720000000E106E000E116E090E45ECBFF0000E60
:10721000066E000E076E000E086E000E096E000E60
:107220000A6E000E0B6E000E0C6E000E0D6E000E40
:107230000E6E000E0F6E000E106E000E116E0A0E16
:1072400045ECBFF0010E066E010E076E010E086ED2
:10725000010E096E010E0A6E010E0B6E010E0C6E10
:10726000010E0D6E010E0E6E010E0F6E010E106EF0
:10727000010E116E0C0E45ECBFF0D00E136ECA0E4F
:10728000E82EFED7132EFCD7120020EEA2F0080E37
:10729000DE6AE806FDE2A8ECCCF0CC0EC3ECCDF043
:1072A000440EC3ECCDF0D00E1C6ECA0EE82EFED7F5
:1072B0001C2EFCD7A8ECCCF0CC0EC3ECCDF0BE0E4F
:1072C000C3ECCDF0000E0001B36FA20EB325D96E52
:1072D000DA6A000EDA2202ECCDF0DF6E0001B32B89
:1072E000010EB36576EFB9F078EFB9F065EFB9F05C
:1072F000A8ECCCF00001A251026E036A046A056A90
:10730000010E54ECB4F002C092F003C093F004C03C
:1073100094F005C095F0000E146E000E156E800EF0
:10732000166E430E176E0001A351026E036A046AC3
:10733000056A010E54ECB4F002C010F003C011F065
:1073400004C012F005C013F04BECA5F010C08EF095
:1073500011C08FF012C090F013C091F0EAECA2F0CF
:107360008EC0AFF08FC0B0F090C0B1F091C0B2F05D
:10737000AFC010F0B0C011F0B1C012F0B2C013F045
:10738000000E146E000E156E800E166E3D0E176EFA
:107390004BECA5F010C0ABF011C0ACF012C0ADF0DA
:1073A00013C0AEF0ABC09EF0ACC09FF0ADC0A0F07B
:1073B000AEC0A1F0120095ECCFF00009D8B4E3EF15
:1073C000B9F0E5EFB9F021EFBAF0F2EFB9F0F6EC71
:1073D000CFF06DEFBAF04CECD0F06DEFBAF0000EDC
:1073E0006DEFBAF018C10DF019C10EF020EE09F1E1
:1073F00002D805EFBAF00500FA6EDE50FD6EDE50E1
:10740000FE6EDE50FF6EFA5012000F6E106A1050C2
:10741000000AD8B40EEFBAF0EFEFB9F00F50010A3E
:10742000D8B4EFEFB9F0030AD8B4E7EFB9F0010A26
:10743000D8B4EBEFB9F0070AD8B4EFEFB9F0EFEF3B
:10744000B9F08AECCFF00009D8B429EFBAF02BEFED
:10745000BAF06CEFBAF001012951030B0009D8B45E
:1074600034EFBAF036EFBAF042EFBAF0010E0F6E19
:107470002951030B106E0F50105E29511018FC0B90
:107480001018296F60008FF4D9FF600093F4DAFFC1
:10749000DF50116E234B242B2507D8A0260725513A
:1074A0002611D8A456EFBAF058EFBAF060EFBAF050
:1074B000FAECC5F00F6E0F50136E146A64EFBAF059
:1074C000000E146E030E136E13C012F0115009EC6F
:1074D000D0F012506DEFBAF0030E120072EFBAF056
:1074E000024A032A60000BF0D9FF60000FF0DAFFB8
:1074F000200EDE18D8B47FEFBAF081EFBAF070EF4B
:10750000BAF060000BF0D9FF60000FF0DAFF090E4F
:10751000DE18D8B48EEFBAF090EFBAF070EFBAF090
:10752000000E076E000E066E60000BF0D9FF6000C3
:107530000FF0DAFF2D0EDE18D8A4A1EFBAF0A3EFFA
:10754000BAF0A8EFBAF0062A024A032ACBEFBAF043
:1075500060000BF0D9FF60000FF0DAFF2B0EDE1891
:10756000D8A4B5EFBAF0B7EFBAF0CBEFBAF0024A51
:10757000032ACBEFBAF060000BF0D9FF60000FF0E8
:10758000DAFFDF50046E07500A0DF3500424D00FC9
:10759000076EB7EFBAF060000BF0D9FF60000FF094
:1075A000DAFF2F0EDF64D7EFBAF0D9EFBAF0E7EFCA
:1075B000BAF060000BF0D9FF60000FF0DAFF390E6F
:1075C000DF64E5EFBAF0E7EFBAF0BBEFBAF00650D0
:1075D000D8B4EDEFBAF0EFEFBAF0FCEFBAF0075025
:1075E000046E056A041E051E044A052A04C002F042
:1075F00005C003F0FFEFBAF007C002F0036A120003
:10760000E40EF66E9E0EF76E010EF86E01EEA1F11D
:1076100010EE19F009006F00D7FFEEFFE550E150C2
:10762000F9E1CA0EF66E9E0EF76E010EF86E00EED0
:10763000D0F310EE1AF009006F00D7FFEEFFE5500F
:10764000E150F9E14A0EF66E930EF76E010EF86EF8
:1076500000EE93F210EE5AF009006F00D7FFEEFF34
:10766000E550E150F9E1CE0EF66E9F0EF76E010E79
:10767000F86E00EEDDF110EE0FF009006F00D7FF9D
:10768000EEFFE550E150F9E101EEBAF110EE00F342
:10769000EE6AE550E150FCE1E250FAE101EE00F162
:1076A000A10EEE6AE806FDE101EE00F010EE00F139
:1076B000EE6AE550E150FCE1E250FAE100EE00F341
:1076C000D00EEE6AE806FDE100EE00F2930EEE6ADF
:1076D000E806FDE10101EC6B00EE00F1920EEE6AAE
:1076E000E806FDE10001FD6BFC6BFB6BFA6BF96BCF
:1076F000F86B1E6A080ED56E000ED66E000ED76EA1
:10770000000100EF80F0043405340B6E0B50D8A458
:107710008CEFBBF08EEFBBF098EFBBF0000E026E6B
:10772000000E036E000E046E000E056E05EFBCF039
:1077300002C006F003C007F004C008F005C009F05D
:10774000200EA8EFBBF0D89009320832073206327B
:10775000E82EA3EFBBF006500A6E048EFF0E021651
:10776000FF0E0316FF0E0416000E0516960E0B5E96
:107770000BBEBFEFBBF0BDEFBBF0D5EFBBF00B50C6
:10778000800A970FD8B0C7EFBBF0C9EFBBF0CBEFC3
:10779000BBF08EEFBBF0D8900532043203320232D8
:1077A0000B3ECBEFBBF0EDEFBBF01F0E0B64DBEF3E
:1077B000BBF0DDEFBBF0E5EFBBF08EEFBBF0D89098
:1077C00002360336043605360B060B50D8A4EBEF11
:1077D000BBF0EDEFBBF0DFEFBBF00A50D8B4F3EF36
:1077E000BBF0F5EFBBF0FDEFBBF0051E041E031E62
:1077F000026C000E03220422052202C002F003C024
:1078000003F004C004F005C005F01200000E0001F2
:107810008E15966F000E8F15976F800E9015986FCE
:107820007F0E9115996F9651971198119911D8A4BF
:107830001CEFBCF01EEFBCF026EFBCF0000E8E6F0C
:10784000000E8F6F000E906F000E916F000E92155C
:10785000966F000E9315976F800E9415986F7F0E9C
:107860009515996F9651971198119911D8A43BEFDE
:10787000BCF03DEFBCF045EFBCF0000E926F000E87
:10788000936F000E946F000E956F91AF4AEFBCF0AE
:107890004CEFBCF055EFBCF08E6D8F1FD8B08F2B26
:1078A000901FD8B0902B800E915795AF5AEFBCF037
:1078B0005CEFBCF065EFBCF0926D931FD8B0932BDA
:1078C000941FD8B0942B800E9557000E8E1B000E7F
:1078D0008F1B000E901B800E911B000E921B000E42
:1078E000931B000E941B800E951B92518E5D93513D
:1078F0008F599451905995519159D8B082EFBCF05D
:1079000084EFBCF087EFBCF0D89088EFBCF0D88053
:1079100012003DC20CF03EC20DF03FC20EF040C25C
:107920000FF002C00CF003C00DF004C00EF005C053
:107930000FF00CC006F00DC007F00EC008F00FC02D
:1079400009F0180EA9EFBCF0D890093208320732BE
:107950000632E82EA4EFBCF006500A6E0B6A0A50FD
:107960000B10D8A4B6EFBCF0B8EFBCF0D8EFBCF069
:10797000D8900C34066E0D34076E0E34086E0F343A
:10798000096E0650071008100910D8A4CAEFBCF001
:10799000CCEFBCF0D2EFBCF0000E036E020E026E14
:1079A00007EFBDF0000E036E030E026E07EFBDF091
:1079B0000A280B10D8A4DFEFBCF0E1EFBCF003EF16
:1079C000BDF00CC006F00DC007F00EC008F00FC0EF
:1079D00009F0090ED8900636073608360936E82E23
:1079E000EAEFBCF00650071008100910D8B4FBEFFE
:1079F000BCF0FEEFBCF0010EFFEFBCF0000E026E1B
:107A0000036A07EFBDF0000E036E040E026E120053
:107A100020EE12F0070EDE6AE806FDE20A500B10B7
:107A20000C100D100E100F1010101110D8B41BEF09
:107A3000BDF01DEFBDF06FEFBDF0010E1A6E2BEF24
:107A4000BDF0D8900A360B360C360D360E360F3692
:107A5000103611361A2A11AE30EFBDF032EFBDF0FC
:107A600021EFBDF0D890123613361436153616367F
:107A70001736183619360A50025C0B5003580C5052
:107A800004580D5005580E5006580F500758105006
:107A9000085811500958D8A050EFBDF052EFBDF072
:107AA00063EFBDF00A50025E0B50035A0C50045AAB
:107AB0000D50055A0E50065A0F50075A1050085ACA
:107AC0001150095A1280D890113210320F320E32F2
:107AD0000D320C320B320A321A2E32EFBDF012C0C8
:107AE00002F013C003F014C004F015C005F016C076
:107AF00006F017C007F018C008F019C009F012000E
:107B000000F06F00A0FF7AF16F0080FF7BF10001B1
:107B1000D8907837703768376037583750374837DC
:107B200040373837303728372037D8907937713792
:107B30006937613759375137493741373937313725
:107B400029372137D8907A3772376A3762375A37F0
:107B500052374A3742373A3732372A372237D890A6
:107B60007B3773376B3763375B3753374B37433765
:107B70003B3733372B372337D8907C3774376C3704
:107B800064375C3754374C3744373C3734372C37FD
:107B90002437D8907D3775376D3765375D37553762
:107BA0004D3745373D3735372D372537D8907E3718
:107BB00076376E3766375E3756374E3746373E373D
:107BC00036372E372637D8907F3777376F37673776
:107BD0005F3757374F3747373F3737372F372737D5
:107BE0006000EFF5E0FF6000EBF5E8FF1200000138
:107BF000866FB8ECC3F0000E0101E36F000E0201C6
:107C0000E46FE30E026E010E036E01018651E4EC97
:107C1000CCF03A0E0101E56FE60E026E010E036E26
:107C20008751E4ECCCF03A0E0101E86FE90E026EE8
:107C3000010E036E8851E4ECCCF0000E0101EB6FF5
:107C4000E40E026E020E036E8451E4ECCCF02F0EB3
:107C50000201E66FE70E026E020E036E0101835110
:107C6000E4ECCCF02F0E0201E96FEA0E026E020E78
:107C7000036E01018251E4ECCCF0000E0201EC6FC6
:107C800001018351CCECCFF00101816F8851CCEC24
:107C9000CFF001017E6F00018605D8A452EFBEF03F
:107CA00054EFBEF06CEFBEF0E40E086E020E096EEB
:107CB0000DECC8F01B0E026EF50E036EFEECC9F063
:107CC000E30E086E010E096E0DECC8F01B0E026E7D
:107CD000F50E036EFEECC9F01200010130513111B6
:107CE000D8A475EFBEF077EFBEF07DEFBEF030C1E7
:107CF00011F031C112F083EFBEF0FF0E3025116E8E
:107D0000FF0E3121126E34A188EFBEF08AEFBEF073
:107D100093EFBEF00DC002F0036A0BC004F00CC07C
:107D200005F0D9ECBEF012BE98EFBEF09AEFBEF0AF
:107D30009CEFBEF0A0EFBEF0000E126E000E116EB2
:107D4000000E106E000E0F6EB2EFBEF0000E036E4E
:107D5000200E026E0BC004F00CC005F0D9ECBEF092
:107D60000F4A102A11500F5C1050800A0E6E1250EC
:107D7000800A0E58D8A0BFEFBEF0C1EFBEF0A6EF4C
:107D8000BEF0010134B1C7EFBEF0C9EFBEF0D2EFD3
:107D9000BEF00DC002F0036A0BC004F00CC005F089
:107DA000D9ECBEF0010E0F240B6E000E10200C6EED
:107DB000120004500510D8B4E0EFBEF0E2EFBEF0C0
:107DC000EBEFBEF004500510D8A4E9EFBEF0EBEFE6
:107DD000BEF0F0EFBEF0025052ECD0F044EFBFF036
:107DE00020EE09F00450D9260550DA22DE50DE10CC
:107DF000D8B4FDEFBEF0FFEFBEF01AEFBFF020EEFB
:107E000009F00450D9260550DA2210EE03F0045090
:107E1000E1260550E222DE50E65CE650800A0A6E5A
:107E2000DE50800A0A58D8B018EFBFF01AEFBFF042
:107E300044EFBFF020EE03F00450D9260550DA22BB
:107E40006F0078FF06F06F0074FF07F0600013F01A
:107E5000D9FF600017F0DAFF6F0078FF08F06F00BD
:107E600074FF09F006500824D96E07500920DA6E15
:107E700060000BF0DFFF20EE03F00450D926055020
:107E8000DA22DE2A000EDD221200126EBC901A0EDB
:107E9000E82EFED700D01250B1ECC8F01150B1EC72
:107EA000C8F000F000F01250B1ECC8F01050B1EC86
:107EB000C8F000F000F01250B1ECC8F00F50B1EC77
:107EC000C8F000F000F01250B1ECC8F00E50B1EC68
:107ED000C8F000F000F01250B1ECC8F00D50B1EC59
:107EE000C8F000F000F01250B1ECC8F00C50B1EC4A
:107EF000C8F000F000F01250B1ECC8F00B50B1EC3B
:107F0000C8F000F000F01250B1ECC8F00A50B1EC2B
:107F1000C8F000F000F01250B1ECC8F00950B1EC1C
:107F2000C8F000F000F01250B1ECC8F00850B1EC0D
:107F3000C8F000F000F01250B1ECC8F00750B1ECFE
:107F4000C8F000F000F01250B1ECC8F00650B1ECEF
:107F5000C8F000F000F01A0EE82EFED700D0BC806A
:107F60001200000E146E000E136E000E066E000E50
:107F7000076E000E086E000E096E000E0A6E000EEF
:107F80000B6E000E0C6E000E0D6E000E0E6E000ECF
:107F90000F6E000E106E000E116E132845ECBFF030
:107FA0006A0EE82EFED700D0134A142A14BEE2EF60
:107FB000BFF0145009E1080E135CD8A0E2EFBFF047
:107FC000E4EFBFF0B5EFBFF0000E066E000E076ED7
:107FD000000E086E000E096E000E0A6E000E0B6E8B
:107FE000000E0C6E000E0D6E000E0E6E000E0F6E6B
:107FF000000E106E000E116E000E45ECBFF0000E6C
:10800000066E000E076E000E086E000E096E000E62
:108010000A6E000E0B6E000E0C6E000E0D6E000E42
:108020000E6E000E0F6E000E106E000E116E0A0E18
:1080300045ECBFF01200000EBA6EBB68BC68000EC3
:108040003A01606F000E506F000E406F000EC26E5E
:10805000C368800EC46E000E156FBC80BC92BC9AC3
:10806000000E816F5169FC0E416F6169000E006F57
:10807000000E016F000E026F000E046FC298BA88E6
:10808000000E5A6F000E5B6F000E086F000E096F36
:10809000000E0A6F000E0B6F000E0C6F000E0D6FBE
:1080A000000E0E6F000E0F6FC384C382070E426F67
:1080B000070E526F180E626F4369800E536F63692B
:1080C000446954696469080E846F000E476F000E9E
:1080D000466F000E456F000E576F000E566F000E74
:1080E000556F000E676F000E666F000E656F210EF4
:1080F000136F220E146F130E166F170EE56F130E0B
:10810000E16F140EE26F12000A500B100C100D10EC
:108110000E100F1010101110D8B491EFC0F093EFA3
:10812000C0F0DBEFC0F0010E126EA1EFC0F0D890EE
:108130000A360B360C360D360E360F361036113623
:10814000122A11AEA6EFC0F0A8EFC0F097EFC0F072
:108150000A50025C0B5003580C5004580D5005583F
:108160000E5006580F500758105008581150095813
:10817000D8A0BDEFC0F0BFEFC0F0CFEFC0F00A5005
:10818000025E0B50035A0C50045A0D50055A0E5003
:10819000065A0F50075A1050085A1150095AD890D1
:1081A000113210320F320E320D320C320B320A32D3
:1081B000122EA8EFC0F002C002F003C003F004C00A
:1081C00004F005C005F006C006F007C007F008C0BF
:1081D00008F009C009F01200046E800E056E000E52
:1081E000076E000E066E3DEFC1F001017151D8A47B
:1081F000FCEFC0F0FEEFC0F01CEFC1F0045005141E
:108200000009D8B406EFC1F008EFC1F012EFC1F0D9
:10821000DB0E0624D96E020E0720DA6E310EDF6EF9
:1082200038EFC1F0DB0E0624D96E020E0720DA6E9D
:10823000300EDF6E38EFC1F0045005140009D8B4D9
:1082400024EFC1F026EFC1F030EFC1F0DB0E0624C1
:10825000D96E020E0720DA6E2A0EDF6E38EFC1F0FB
:10826000DB0E0624D96E020E0720DA6E2E0EDF6EAC
:10827000D8900530056E064A072A07BE49EFC1F0BF
:10828000075009E1080E065CD8A049EFC1F04BEF9A
:10829000C1F0F5EFC0F0000E0201E36FDB0E026EDD
:1082A000020E036E1200010134A159EFC1F05BEF21
:1082B000C1F065EFC1F014C00BF015C00CF012C096
:1082C0000DF013C00EF048ECCCF017BE6AEFC1F011
:1082D0006CEFC1F072EFC1F016C01BF017C01CF0BC
:1082E00076EFC1F0000E1C6E000E1B6E000E1A6EB3
:1082F000000E196E88EFC1F0000E036E200E026EA4
:1083000012C004F013C005F0D9ECBEF0194A1A2AC5
:108310001B50195C1A50800A186E1C50800A18589D
:10832000D8A095EFC1F097EFC1F07CEFC1F001014B
:1083300034B19DEFC1F09FEFC1F0A9EFC1F014C0BF
:108340000BF015C00CF012C00DF013C00EF048EC8D
:10835000CCF014C002F015C003F0D2ECC9F01B50F1
:108360000224126E1C500320136E1200000E076EC2
:1083700005BEBFEFC1F0BDEFC1F0C5EFC1F0046CA9
:10838000051ED8B0052A010E076E03BECCEFC1F062
:10839000CAEFC1F0D2EFC1F0026C031ED8B0032ABD
:1083A000010E071A000E096E000E086E045005102B
:1083B000D8B4DDEFC1F0DFEFC1F007EFC2F0010E7E
:1083C000066EE7EFC1F0D89004360536062A05AEF2
:1083D000ECEFC1F0EEEFC1F0E3EFC1F0D89008365A
:1083E00009360450025C05500358D8A0FAEFC1F0DA
:1083F000FCEFC1F001EFC2F00450025E0550035AD9
:108400000880D89005320432062EEEEFC1F00750F6
:10841000D8B40DEFC2F00FEFC2F013EFC2F0086C4A
:10842000091ED8B0092A08C002F009C003F01200E2
:10843000000E076E03BE21EFC2F01FEFC2F027EF60
:10844000C2F0026C031ED8B0032A010E076E05BEEF
:108450002EEFC2F02CEFC2F032EFC2F0046C051E1A
:10846000D8B0052A04500510D8B439EFC2F03BEF5C
:10847000C2F05FEFC2F0010E066E43EFC2F0D8907B
:1084800004360536062A05AE48EFC2F04AEFC2F0C0
:108490003FEFC2F00450025C05500358D8A053EFE0
:1084A000C2F055EFC2F059EFC2F00450025E055021
:1084B000035AD89005320432062E4AEFC2F0075014
:1084C000D8B465EFC2F067EFC2F06BEFC2F0026C98
:1084D000031ED8B0032A02C002F003C003F012004A
:1084E000000E02140A6E000E03140B6E800E0414AC
:1084F0000C6E7F0E05140D6E0A500B100C100D1033
:10850000D8A485EFC2F087EFC2F08FEFC2F0000E63
:10851000026E000E036E000E046E000E056E000E5D
:1085200006140A6E000E07140B6E800E08140C6EF3
:108530007F0E09140D6E0A500B100C100D10D8A4EC
:10854000A4EFC2F0A6EFC2F0AEEFC2F0000E066ECE
:10855000000E076E000E086E000E096E065002181F
:108560000FE1075003180CE10850041809E1095005
:108570000518D8B4BEEFC2F0C0EFC2F0C3EFC2F02E
:10858000D890C4EFC2F0D8801200026E010E036EC4
:10859000010129B7CEEFC2F0D0EFC2F015EFC3F062
:1085A00002C022F129952987FC0E29170F0E276F8B
:1085B000010E216FF40E206F2989A00E006FA00E0E
:1085C000016F010E026F000E126F000E136FA00EEE
:1085D000036FA00E046F010E056F000E146F000EE6
:1085E000156FA00E066FA00E076F010E086F000E2C
:1085F000166F000E176FA00E096FA00E0A6F010E06
:108600000B6F000E186F000E196F9C0E0C6FA00EF2
:108610000D6F010E0E6F000E1A6F000E1B6F28EC0F
:10862000D0F03BECCEF0000E036E035012000101BF
:1086300029893BEFC3F03BECD0F0080E68EFC3F0A4
:108640003BECD0F0070E68EFC3F0010125290EECDA
:10865000D0F0040E68EFC3F0070E01012719D8B45B
:1086600034EFC3F036EFC3F038EFC3F03EECD0F098
:108670000F0E68EFC3F012C10DF013C10EF002D857
:108680004CEFC3F00500FA6E0051FD6E0151FE6E15
:108690000251FF6EFA5012000F6E106A1050000A5D
:1086A000D8B455EFC3F02CEFC3F00F50010AD8B483
:1086B0002CEFC3F0030AD8B420EFC3F0010AD8B4FA
:1086C0001BEFC3F0070AD8B425EFC3F02CEFC3F0BB
:1086D0001200A0ECCFF00009D8A471EFC3F073EF43
:1086E000C3F076EFC3F0040EB7EFC3F001012951D8
:1086F000030B0009D8B47FEFC3F081EFC3F08DEF17
:10870000C3F0010E116E2951030B126E1150125E4F
:1087100029511218FC0B1218296F2507D8A026071B
:1087200025512611D8B497EFC3F099EFC3F0A7EF06
:10873000C3F038ECD0F060008FF4D9FF600093F400
:10874000DAFFDF6E0101234B242B73EFC3F017EC2C
:10875000C3F0136E38ECD0F060008FF4D9FF6000E6
:1087600093F4DAFFDF6E0101234B242B1350120028
:10877000000E1D6E000E1C6E8A0E1C24D96E010E9A
:108780001D20DA6E000EDF6E1C4A1D2A1DBED2EFC0
:10879000C3F01D5009E10A0E1C5CD8A0D2EFC3F053
:1087A000D4EFC3F0BCEFC3F08A0E0001FA6F010EE4
:1087B000FB6F000E176EFAC018F0FBC019F0000E28
:1087C0001B6E070E1A6E680EB5ECC5F08AC188F1F3
:1087D0008BC187F101018C513F0B866F8DC185F1F3
:1087E000070E8565F6EFC3F0F8EFC3F0FAEFC3F0BC
:1087F000000E856F8EC184F18F511F0B836F90C166
:1088000082F1000E916F000E926F12003901A3A742
:108810000CEFC4F00EEFC4F052EFC4F093A713EFC7
:10882000C4F015EFC4F052EFC4F06F00A0F789F167
:108830000D0E01018919D8B420EFC4F022EFC4F065
:108840002DEFC4F0575109E1800E565DD8A02BEFF3
:10885000C4F02DEFC4F043EFC4F0010E756F800E2D
:108860005625D96E040E5721DA6E000EDF6E56C102
:1088700058F157C159F1000E576F000E566F39016C
:10888000939752EFC4F0800E5625D96E040E5721EF
:10889000DA6E600027F6DFFF564B572B56C158F1B2
:1088A00057C159F1110002C008F003C009F079EF77
:1088B000C4F00606D8A00706600013F0D9FF6000D8
:1088C00017F0DAFF044A052A600023F0E1FF600098
:1088D00027F0E2FF084A092A6F007FFFE7FFE75011
:1088E000D8A475EFC4F077EFC4F079EFC4F08EEF41
:1088F000C4F006500710D8A480EFC4F082EFC4F093
:1089000059EFC4F08EEFC4F0600023F0D9FF60008F
:1089100027F0DAFF000EDF6E084A092A0606D8A003
:108920000706062806E10728D8A499EFC4F09BEFB4
:10893000C4F084EFC4F01200000E176E000E166E25
:1089400010C014F011C015F016500D24096E175008
:108950000E200A6E600053F0D9FF600057F0DAFF76
:10896000DF500B6E7DECCAF0600053F0D9FF600061
:1089700057F0DAFFDF50D8A4C0EFC4F0C2EFC4F064
:10898000C4EFC4F0E2EFC4F0020E136EA00E126E3C
:10899000920EE82EFED7122EFCD7132EFAD700D057
:1089A000144A152A164A172A0F50126E136A1250CB
:1089B000165C13501758D8A0E0EFC4F0E2EFC4F0F3
:1089C000A4EFC4F01200076E025003100410D8B4D4
:1089D000ECEFC4F0EEEFC4F00FEFC5F00750030D5D
:1089E000000EF324D96E010EF420DA6E60000BF055
:1089F000DEFF60000FF0DEFF600013F0DEFF0750C7
:108A0000020D120EF324D96E010EF420DA6E60000E
:108A100017F0DEFF60001BF0DDFF29EFC5F0075007
:108A2000030D000EF324D96E010EF420DA6EA00EB1
:108A3000DE6EA00EDE6E010EDE6E0750020D120E0F
:108A4000F324D96E010EF420DA6E000EDE6E000EF5
:108A5000DD6E1200000E1D6E010E1C6E8A0E1C24AF
:108A6000D96E010E1D20DA6E000EDF6E1C4A1D2A23
:108A70001DBE44EFC5F01D5009E1090E1C5CD8A0D5
:108A800044EFC5F046EFC5F02EEFC5F0520E026E72
:108A9000F80E036EFEECC9F0000E01018A6F570E4E
:108AA0008B6F590E8C6F110E8D6F060E8E6F270E09
:108AB0008F6F050E906F230E916F000E926F8A0ECE
:108AC0000001FA6F010EFB6FFAC017F0FBC018F03F
:108AD000000E1A6E080E196E680E18ECC9F012001E
:108AE000000E0C6E000E0B6E0B500424026E0C5028
:108AF0000520036EF9ECCEF00A6E0B500624D96EF9
:108B00000C500720DA6E60002BF0DFFF0A50D8A46B
:108B10008CEFC5F08EEFC5F090EFC5F0ACEFC5F06F
:108B2000020E096EA00E086E920EE82EFED7082ED9
:108B3000FCD7092EFAD700D00B4A0C2A0CBEAAEF9C
:108B4000C5F00C5009E1200E0B5CD8A0AAEFC5F0CF
:108B5000ACEFC5F074EFC5F00B500624D96E0C5085
:108B60000720DA6E000EDF6E12000001816F18C060
:108B700084F019C085F01AC082F01BC083F0000198
:108B80008151C5ECC2F00009D8B4C9EFC5F0CBEFF4
:108B9000C5F0BFEFC5F0420E086E960E096E010ECD
:108BA0000A6E820E0B6E000E0C6E57ECCFF0170E95
:108BB000026E000E036E000E056E010E046EE7ECF1
:108BC000CEF0000E086E000E096E000E0A6E000E4A
:108BD0000B6E000E0C6E49ECCFF018ECD0F080EC70
:108BE000CEF0E806D8B4F7EFC5F0F9EFC5F0EFEF37
:108BF000C5F01200010129890FEFC6F03BECD0F05F
:108C0000070E38EFC6F0010125290EECD0F0030E57
:108C100038EFC6F03EECD0F00A0E38EFC6F012C1C5
:108C20000DF013C10EF002D820EFC6F00500FA6E69
:108C30000051FD6E0151FE6E0251FF6EFA5012009E
:108C40000F6E106A1050000AD8B429EFC6F00AEF70
:108C5000C6F00F50010AD8B40AEFC6F0030AD8B420
:108C6000FEEFC5F0060AD8B403EFC6F00AEFC6F06F
:108C70001200186E000E196E1850C5ECC2F00009F3
:108C8000D8B445EFC6F047EFC6F03CEFC6F0160E7D
:108C9000086E9C0E096E010E0A6E190E0B6E000E08
:108CA0000C6E57ECCFF0170E026E000E036E000E26
:108CB000056E010E046EE7ECCEF0000E086E000E9D
:108CC000096E000E0A6E000E0B6E000E0C6E49EC63
:108CD000CFF018ECD0F080ECCEF0E806D8B473EF0B
:108CE000C6F075EFC6F06BEFC6F0195012003901EF
:108CF000A3A77DEFC6F07FEFC6F082EFC6F06F004E
:108D0000A0F789F1000E036E000E026E800E0224A1
:108D1000D96E040E0320DA6E000EDF6E024A032ABB
:108D2000035009E17F0E025CD8A099EFC6F09BEFDB
:108D3000C6F086EFC6F0000E0101756F3D01F289A5
:108D4000000EF96F000EFA6F000E0401806F000E26
:108D50000101596F000E586F000E896F3901938D14
:108D600093871200196E1950C5ECC2F00009D8B4EF
:108D7000BCEFC6F0BEEFC6F0B3EFC6F0B60E086E9D
:108D80009B0E096E010E0A6E180E0B6E000E0C6E15
:108D900057ECCFF0170E026E000E036E000E056E3C
:108DA000010E046EE7ECCEF0000E086E000E096EA8
:108DB000000E0A6E000E0B6E000E0C6E49ECCFF02A
:108DC00018ECD0F080ECCEF0E806D8B4EAEFC6F0AC
:108DD000ECEFC6F0E2EFC6F0120028ECD0F0020E85
:108DE0000101286F00EFC7F0F6ECCFF027EFC7F0D6
:108DF0004CECD0F027EFC7F0DFECCFF027EFC7F057
:108E000014C10DF015C10EF020EE03F102D813EFDE
:108E1000C7F00500FA6EDE50FD6EDE50FE6EDE50CD
:108E2000FF6EFA5012000F6E106A1050000AD8B48C
:108E30001CEFC7F0FCEFC6F00F50020AD8B4F4EFF5
:108E4000C6F0010AD8B4F8EFC6F0FCEFC6F0120085
:108E5000000E076E000E066E04500510D8B433EFF6
:108E6000C7F035EFC7F05DEFC7F0010E086E3DEFBC
:108E7000C7F0D89004360536082A05AE42EFC7F091
:108E800044EFC7F039EFC7F0D890063607360450E4
:108E9000025C05500358D8A050EFC7F052EFC7F05E
:108EA00057EFC7F00450025E0550035A0680D89071
:108EB00005320432082E44EFC7F006C002F007C0A6
:108EC00003F01200600013F0F6FF600017F0F7FFE8
:108ED000000EF86E08006F00D4FF6BF189EFC7F049
:108EE000600013F0F6FF600017F0F7FF000EF86E59
:108EF00008006F00D4FF6BF160000BF0D9FF600039
:108F00000FF0DAFF6000AFF5DFFF024A032A044AE0
:108F1000052A01016B51D8A490EFC7F092EFC7F07A
:108F200070EFC7F060000BF0D9FF60000FF0DAFFC0
:108F3000000EDF6E1200F0C0F4F0F1C0F5F0000E8C
:108F400001012F6F000E2E6FBDEFC7F0EEC0E4F0F1
:108F5000EFC0E5F0F40E0001E66F000EE76FF2C01F
:108F6000E8F0F3C0E9F08BEC9AF00001E451010164
:108F70002E270001E55101012F236000D3F3F6FFF6
:108F80006000D7F3F7FF000EF86E0800F5500009F7
:108F9000D8A4CDEFC7F0CFEFC7F0A6EFC7F02EC132
:108FA000EEF02FC1EFF01200F8ECCAF001012951E8
:108FB000030B0009D8B4DFEFC7F0E1EFC7F0EEEF25
:108FC000C7F095ECCFF00009D8B4E9EFC7F0EBEFAC
:108FD000C7F0EEEFC7F0100E0101276F0101275116
:108FE000030D8F0EF324F66EF20EF420F76EF86A7E
:108FF000000EF82202D80AEFC8F00500FA6E090048
:10900000F550FD6E0900F550FE6E0900F550FF6E3B
:10901000FA5012000101276F1200000E0B6E000EB5
:109020000A6E36EFC8F03901A3A919EFC8F01BEF9B
:10903000C8F013EFC8F00A500824D96E0B5009206D
:10904000DA6EDF503D01EA6F0A4A0B2A0BBE32EF9F
:10905000C8F00B5009E1810E0A5CD8A032EFC8F0CD
:1090600034EFC8F036EFC8F044EFC8F00A500824D7
:10907000D96E0B500920DA6EDF50D8A442EFC8F049
:1090800044EFC8F013EFC8F01200FC0E01012917DD
:10909000020E286F299554EFC8F04AECD0F07BEF10
:1090A000C8F00F0E7BEFC8F016C10DF017C10EF01F
:1090B00020EE06F102D867EFC8F00500FA6EDE5028
:1090C000FD6EDE50FE6EDE50FF6EFA5012000F6E27
:1090D000106A1050000AD8B470EFC8F051EFC8F011
:1090E0000F50020AD8B44DEFC8F0010AD8B44DEFC2
:1090F000C8F051EFC8F0120008C00CF009C00DF024
:1091000006C00EF007C00FF00C500A6E0D500B6E2B
:109110000C4A0D2A60002BF0F6FF60002FF0F7FFDD
:10912000000EF86E60003BF0D9FF60003FF0DAFF00
:109130000E4A0F2A1F0EF76403D00800F55007D01F
:109140006F00DBFFE9FF6F00DFFFEAFFEF50DF6E2C
:10915000DF50D8A4AEEFC8F0B0EFC8F084EFC8F08D
:109160001200026EBC9202C005F0000E046E000EEA
:10917000036E05AEBEEFC8F0C0EFC8F0C3EFC8F095
:10918000BC8AC4EFC8F0BC9A1A0EE82EFED700D0F5
:1091900005500524056EBC821A0EE82EFED700D0BD
:1091A000BC921A0EE82EFED700D0034A042A04BE51
:1091B000E3EFC8F0045009E1080E035CD8A0E3EF28
:1091C000C8F0E5EFC8F0B9EFC8F012000450051080
:1091D000D8B4EDEFC8F0EFEFC8F013EFC9F0010E0F
:1091E000066EF7EFC8F0D89004360536062A05AEAD
:1091F000FCEFC8F0FEEFC8F0F3EFC8F00450025CDB
:1092000005500358D8A007EFC9F009EFC9F00DEFDA
:10921000C9F00450025E0550035AD890053204325A
:10922000062EFEEFC8F002C002F003C003F01200E9
:109230001B6E1B50C5ECC2F00009D8B422EFC9F078
:1092400024EFC9F019EFC9F017C002F018C003F0FD
:1092500019C004F01AC005F0E7ECCEF0000E086E5D
:10926000000E096E000E0A6E000E0B6E000E0C6EE4
:1092700049ECCFF018ECD0F080ECCEF0E806D8B492
:0E92800044EFC9F046EFC9F03CEFC9F0120010
:109290003901A4A14EEFC9F050EFC9F076EFC9F043
:1092A00094A155EFC9F057EFC9F076EFC9F001016D
:1092B00048514911D8A45FEFC9F061EFC9F068EFD8
:1092C000C9F0B29039019491010172836BEFC9F03A
:1092D0004807D8A04907CF0EB16E2C0EB06E000E15
:1092E0000201786F010E776F3901A49111003901E5
:1092F000A3A17DEFC9F07FEFC9F081EFC9F0A4EF22
:10930000C9F0A2AF86EFC9F088EFC9F08AEFC9F0C3
:10931000A4EFC9F03D0179A590EFC9F092EFC9F033
:1093200094EFC9F0A4EFC9F079AF99EFC9F09BEFC2
:10933000C9F09DEFC9F0A4EFC9F076A9A2EFC9F07A
:10934000A4EFC9F077EFC9F01200E8F3A3F320F41B
:1093500093F474F45EF3B2F44FF419F3C9F2C2F467
:10936000E7F4E3F4DFF4DBF4D7F4D3F4CFF4203103
:10937000324835376D6E00F8202020202E2E2070C8
:1093800050770404040407286E756C6C2900E2FE13
:10939000D3FE30303030303030300030302F30308D
:1093A0002F30300002C004F003C005F0DAEFC9F03E
:1093B000024A032A60000BF0F6FF60000FF0F7FF8F
:1093C000000EF86E1F0EF76403D00800F55007D0AA
:1093D0006F00DBFFE9FF6F00DFFFEAFFEF500009DE
:1093E000D8A4F5EFC9F0F7EFC9F0D8EFC9F00450F1
:1093F000025C026E05500358036E120016EFCAF0AD
:109400003901A3A906EFCAF008EFCAF000EFCAF0CD
:1094100060000BF0F6FF60000FF0F7FF000EF86E33
:1094200008006F00D7FFEAFD024A032A60000BF034
:10943000F6FF60000FF0F7FF000EF86E0800F55021
:109440000009D8A426EFCAF028EFCAF000EFCAF04E
:109450001200056E000E0101396F000E386F40EFEB
:10946000CAF0520E036E2B0E026E000EE82EFED7CF
:10947000022EFCD7032EFAD700D00101384B392B2E
:109480000550026E036A0250385D3951800A046E3D
:109490000350800A0458D8A050EFCAF052EFCAF027
:1094A00031EFCAF01200B40E0101CC6F010ECD6F86
:1094B000B0C1CEF1B1C1CFF1000ED26F000ED16FAD
:1094C000000ED86F000ED76FCE0E0001EE6F010EAA
:1094D000EF6FB2C1F0F0B3C1F1F0CC0EF26F010E3C
:1094E000F36F9BECC7F00101D151B025D96ED25179
:1094F000B121DA6E000EDF6E1200000ED2BE010E38
:109500000C6E0A50030B3901E16F600027F0E0F99F
:1095100060002FF0E3F93F0EE517E585D29E550E6A
:10952000E66FAA0EE66FE58397EFCAF000F0390107
:10953000E5B39DEFCAF09FEFCAF096EFCAF0E5954C
:109540000CB002D0D29E01D0D28E1200010E086E55
:10955000200E02180310D8B4B0EFCAF0B2EFCAF070
:10956000CBEFCAF0F70E046EFF0E056E02C006F0D8
:1095700003C007F00450062605500722075009E1F2
:10958000050E065CD8A0C7EFCAF0C9EFCAF0CBEF52
:10959000CAF0000E086E08C002F0036A1200156ED1
:1095A000010E166E010129B5D8EFCAF0DAEFCAF044
:1095B000F6EFCAF02985000E166E25510EECD0F09C
:1095C0001550D8B4E6EFCAF0E8EFCAF0EFEFCAF0F2
:1095D000040E0101276F52ECCEF0F4EFCAF0030E37
:1095E0000101276F7FECCFF02BECCFF0165012006B
:1095F000C1ECCFF00009D8B400EFCBF002EFCBF014
:1096000006EFCBF047ECD0F020EFCBF0ABECCFF097
:109610000009D8B40EEFCBF010EFCBF014EFCBF085
:1096200041ECD0F020EFCBF0B6ECCFF00009D8B48D
:109630001CEFCBF01EEFCBF020EFCBF044ECD0F0E2
:10964000120020EE02F00D50D9260E50DA226F00E3
:1096500078FF02F06F0074FF03F0600037F0D9FF6D
:1096600060003BF0DAFF6F0078FF04F06F0074FFDA
:1096700005F0E7ECCEF0000E086E000E096E000E4D
:109680000A6E000E0B6E000E0C6E57ECCFF0020E41
:029690001200C6
:109694003901A1A150EFCBF052EFCBF06EEFCBF03C
:1096A40091A157EFCBF059EFCBF06EEFCBF02A0E30
:1096B400016E8E0EE82EFED7012EFCD7CBA065EFEF
:1096C400CBF067EFCBF06CEFCBF0000E0201686FCC
:1096D400010E676F3901A19102018F4B902B11008C
:1096E40003BE7DEFCBF0035008E10204D8A07DEF68
:1096F400CBF07FEFCBF08CEFCBF0C290CA901A0E78
:10970400E82EFED700D0C280C00E00D0E82EFDD7D0
:1097140097EFCBF0C290CA90E00E00D0E82EFDD7B0
:10972400C2800A0EE82EFED700D01200000E3D01C2
:10973400EC6F000EED6F000EEE6F000EEF6F000E7B
:10974400F06F000EF16FB00EF26F800EF36F000E2B
:10975400F46F8A0EF56F000EF66F000EF76F000EB1
:10976400F86F000EF96F000EFA6FF28BF28939016F
:1097740093971200000E0001A21B000EA31B000E03
:10978400A41B800EA51B9EC08EF09FC08FF0A0C0AE
:1097940090F0A1C091F0A2C092F0A3C093F0A4C035
:1097A40094F0A5C095F0EAECA2F08EC09EF08FC0B4
:1097B4009FF090C0A0F091C0A1F01200BF0E0A6EFD
:1097C400FF0E0B6E08C00CF009C00DF00A500C26F9
:1097D4000B500D220D5007E11A0E0C5CD8B0F5EFBA
:1097E400CBF0F7EFCBF0FEEFCBF0200E0810086EB5
:1097F4000950096E02EFCCF008C008F009C009F066
:1098040012001B6E1BC017F0680E39ECC6F0010184
:109814006A6F1A04D8A411EFCCF013EFCCF023EF45
:10982400CCF0000E026E030E036E6A51E4ECCCF031
:10983400000E086E030E096E0DECC8F0090E1BEC49
:10984400CFF001016A5112009F0E0A6EFF0E0B6EDB
:1098540008C00CF009C00DF00A500C260B500D2264
:109864000D5007E11A0E0C5CD8B03BEFCCF03DEF85
:10987400CCF043EFCCF05F0E0814086E096A47EF92
:10988400CCF008C008F009C009F01200000E116EF7
:10989400000E106E59EFCCF00FC002F0036A0DC039
:1098A40004F00EC005F0D9ECBEF0104A112A105095
:1098B4000B24D96E11500C20DA6EDF500F6E0F504E
:1098C400D8A467EFCCF069EFCCF04EEFCCF01200E7
:1098D40015BE77EFCCF0155006E11404D8B075EF3F
:1098E400CCF077EFCCF085EFCCF014C016F015C0B7
:1098F40017F0161E171E164A172A16C014F017C0A2
:1099040015F089EFCCF014C014F015C015F0120056
:10991400C290CA900B0E026E620EE82EFED7022E83
:10992400FCD700D0C280C00E00D0E82EFDD7CAB04C
:109934009EEFCCF0A0EFCCF0A7EFCCF0E40E00D07B
:1099440000D0E82EFCD700D000D01200C290CA90FC
:109954000B0E026E620EE82EFED7022EFCD700D04C
:10996400C280C00E00D0E82EFDD7CAB0BCEFCCF048
:10997400BEEFCCF0C5EFCCF0E40E00D000D0E82E62
:10998400FCD700D000D012009F0E046EFF0E056EAF
:10999400200E0210066E000E0310076E04500626F9
:1099A4000550072207500AE11A0E065CD8A0DDEF25
:1099B400CCF0E0EFCCF0010EE1EFCCF0000E026E43
:1099C400036A1200046E04380F0B300F60000BF0B2
:1099D400D9FF60000FF0DAFFDF6E20EE01F00250D5
:1099E400D9260350DA2204500F0B300FDF6E20EE1D
:1099F40002F00250D9260350DA22000EDF6E120064
:109A0400000E036E000E046ED890033296ECCEF076
:109A14000009D8B410EFCDF012EFCDF013EFCDF074
:109A2400038E042A070E04641AEFCDF01CEFCDF068
:109A340006EFCDF0035012009F0E046EFF0E056E6C
:109A440002C006F003C007F00450062605500722A2
:109A540007500AE11A0E065CD8A033EFCDF036EFBA
:109A6400CDF0010E37EFCDF0000E026E036A120046
:109A7400BF0E046EFF0E056E02C006F003C007F0B1
:109A8400045006260550072207500AE11A0E065C08
:109A9400D8A04FEFCDF052EFCDF0010E53EFCDF043
:109AA400000E026E036A1200025003100410051027
:109AB400D8B45FEFCDF061EFCDF069EFCDF0000EDB
:109AC400021A000E031A000E041A800E051A02C0B0
:109AD40002F003C003F004C004F005C005F0120056
:109AE400D00E046EFF0E056E02C006F003C007F030
:109AF400045006260550072207500AE10A0E065CA8
:109B0400D8A087EFCDF08AEFCDF0010E8BEFCDF02A
:109B1400000E026E036A12000C6E0CC002F0036A9F
:109B2400000E056E0A0E046E18ECC2F002C00AF0B4
:109B340003C00BF00CC002F0036A000E056E0A0E9F
:109B4400046EB6ECC1F00250100DF3500A2412005A
:109B54003D01799560000BF06EFD000E6C6F738B08
:109B640079A5B7EFCDF0B9EFCDF0B2EFCDF074AB8E
:109B7400BEEFCDF0C1EFCDF0010EC2EFCDF0000E7F
:109B84001200056E000E066E05C004F0010E0416E8
:109B94000450026E036A72ECCBF0D8900532062AA8
:109BA400070E0664D8EFCDF0DAEFCDF0C6EFCDF0B6
:109BB40012000DC002F00EC003F0000E056E010E7F
:109BC400046EE7ECCEF0000E086E000E096E000E77
:109BD4000A6E000E0B6E000E0C6E57ECCFF0040EE6
:109BE40012000DC002F00EC003F0000E056E020E4E
:109BF400046EE7ECCEF0000E086E000E096E000E47
:109C04000A6E000E0B6E000E0C6E57ECCFF0020EB7
:109C140012000DC002F00EC003F0000E056E010E1E
:109C2400046EE7ECCEF0000E086E000E096E000E16
:109C34000A6E000E0B6E000E0C6E57ECCFF0020E87
:109C440012000DC002F00EC003F0000E056E020EED
:109C5400046EE7ECCEF0000E086E000E096E000EE6
:109C64000A6E000E0B6E000E0C6E57ECCFF0040E55
:109C740012003D0173BF41EFCEF043EFCEF051EF40
:109C8400CEF0000E796F000E7A6F000E766F6C695D
:109C9400510E3A016A6F510E6B6F3D01738F1200C2
:109CA40001012951FC0B0209296F25052611D8A4AD
:109CB4005EEFCEF060EFCEF062EFCEF017ECC3F0C3
:109CC400D8800101223509ECD0F0040E12003901CC
:109CD400A3A96FEFCEF071EFCEF069EFCEF00D0EC9
:109CE4003D01EA6F3901A3A97AEFCEF07CEFCEF003
:109CF40074EFCEF00A0E3D01EA6F1200010E026EFF
:109D0400010129B588EFCEF08AEFCEF094EFCEF0C2
:109D14002997226928ECD0F03AECCFF003ECD0F08C
:109D240028C102F002501200C290CA90050EE82E1B
:109D3400FED700F0C2801A0EE82EFED700D0000E27
:109D4400CAB0010E026EB00E00D0E82EFDD702504C
:109D54001200025004026F00CCFF06F06F00D0FF27
:109D640007F002500502F350072603500402F35093
:109D7400072606C002F007C003F012002FECD0F053
:109D84002CECD0F00009D8B4CAEFCEF0CCEFCEF072
:109D9400D2EFCEF0000E0EECD0F0000E09ECD0F0B5
:109DA400000E120010C002F011C003F0D2ECC9F092
:109DB40002501024066E03501120076E12C008F0E2
:109DC40013C009F07CECC8F01200010129A9EDEFE1
:109DD400CEF0EFEFCEF0F8EFCEF002C023F103C0E7
:109DE40024F104C025F105C026F12999120003507D
:109DF400030B3901E16F60000BF0E0F93F0EE5174A
:109E0400E58100F000F000F000F03901E3511200A8
:109E1400030E3D017B6F040E736F800E746F000E92
:109E2400756F000E6C6F7599200E6E6F7995739F28
:109E34001200026E1FEFCFF000F03901A3A925EF45
:109E4400CFF027EFCFF01EEFCFF060000BF0EAFD6C
:109E5400120031EFCFF077ECC9F0D4ECC7F0010178
:109E640029B537EFCFF039EFCFF02DEFCFF0120057
:109E7400390193939395929F93913D017A917A95A9
:109E84007A9F7A9D7A93769376957691120008C09C
:109E940002F009C003F00AC004F00BC005F00CC0C6
:109EA40006F0020EE3ECC4F0120008C002F009C090
:109EB40003F00AC004F00BC005F00CC006F0000E5D
:109EC400E3ECC4F01200C9F417F513F50FF50BF524
:109ED40007F503F5FFF4FBF4F7F4F3F4EFF4EBF414
:109EE40020444546494C454D454E54204D4154521D
:099EF40049434520382A382000BA
:109EFE0001012951FC0B0209296F2251222509EC7F
:109F0E00D0F0030E12003D0178BB90EFCFF093EF2F
:109F1E00CFF0010E94EFCFF0000E12003D0174BB96
:109F2E009BEFCFF09EEFCFF0010E9FEFCFF0000E24
:109F3E0012003D0178B1A6EFCFF0A9EFCFF0010EE0
:109F4E00AAEFCFF0000E12003D0179B5B1EFCFF0C0
:109F5E00B4EFCFF0010EB5EFCFF0000E12003D01C1
:109F6E0076B9BCEFCFF0BFEFCFF0010EC0EFCFF060
:109F7E00000E12003D0179BFC7EFCFF0CAEFCFF050
:109F8E00010ECBEFCFF0000E1200036E03C002F0F5
:109F9E000F0E021603380F0B0A0DF3500224120097
:109FAE0013ECD0F001012995020E286F0F0E12004E
:109FBE0013ECD0F001012995000E286F0F0E120040
:0F9FCE006300FF06060130303A30303A30300081
:109FDE0032ECD0F02FECD0F0FDECCFF012000101FE
:109FEE0025510EECD0F052ECCEF012000101299565
:109FFE00000E286F0F0E12003D01739F000E796F39
:10A00E0078851200026E60000BF06BFD1200026E7E
:10A01E0060000BF06CFD12003D01739F7885738F0D
:10A02E001200000ECFECCAF0120032ECD0F0090E86
:10A03E00120035ECD0F0040E120035ECD0F0030E09
:10A04E001200000E3D01796F12003D016C5112009D
:10A05E003D01739B12003D01748D12003D01749DF4
:10A06E0012003D016A5112003D01738D12003D0137
:10A07E00739D12003D01799512003D0176991200F3
:10A08E003D01799F1200010E1200020E1200050E04
:08A09E001200010E1200120075
:020000040030CA
:0A0000008CD5FFF78DCFFFDFFFFF67
:00000001FF
